:020000040800F2
:1000000000060020E1020008E3020008E302000805
:10001000E3020008E3020008E3020008E30200082C
:10002000E3020008E3020008E30200086D3800085C
:10003000E3020008E3020008E3020008E30200080C
:10004000E3020008E3020008E3020008E3020008FC
:10005000E3020008E30200085D3C0008893C000858
:10006000B53C0008E13C00080D3D0008913E000849
:10007000B93E0008E53E0008113F00083D3F00087A
:10008000653F0008913F0008E3020008E302000812
:10009000E3020008E3020008E3020008393D00081B
:1000A000E3020008E3020008E3020008E30200089C
:1000B000E3020008E3020008E3020008E30200088C
:1000C000E3020008E3020008E3020008E30200087C
:1000D000E3020008E3020008E3020008E30200086C
:1000E0009D3D0008E3020008E3020008E302000867
:1000F000E3020008E3020008E3020008BD3F000835
:10010000E3020008E3020008113E0008E3020008D1
:10011000E3020008E3020008E3020008E30200082B
:10012000E93F0008114000083D4000086940000810
:1001300095400008E3020008E3020008E30200081B
:10014000E3020008E3020008E3020008E3020008FB
:10015000BD400008E940000815410008E30200081E
:10016000E3020008E3020008E3020008E3020008DB
:10017000E3020008F92F0008E3020008E302000888
:10018000E3020008E3020008E3020008E3020008BB
:10019000E3020008E3020008E3020008E3020008AB
:1001A000E3020008E3020008E3020008E30200089B
:1001B000E3020008E3020008E3020008E30200088B
:1001C000E3020008E3020008E3020008E30200087B
:1001D000E3020008E52F0008E3020008E30200083C
:1001E000E3020008E3020008E3020008E30200085B
:1001F000E3020008E3020008E3020008E30200084B
:10020000E3020008E3020008E3020008E30200083A
:10021000E3020008E3020008E3020008E30200082A
:10022000E3020008E3020008E3020008E30200081A
:10023000E3020008E3020008E3020008E30200080A
:10024000E3020008E3020008E3020008E3020008FA
:10025000E3020008E3020008E3020008E3020008EA
:10026000E3020008E3020008E3020008E3020008DA
:10027000E3020008E3020008E3020008E3020008CA
:10028000E3020008E3020008E3020008E3020008BA
:10029000E3020008E3020008E3020008E3020008AA
:1002A000E3020008E3020008E3020008E30200089A
:1002B000E3020008E3020008E3020008E30200088A
:1002C000E3020008E3020008E3020008E30200087A
:1002D000E3020008E3020008E3020008E30200086A
:1002E00002E000F000F8FEE772B6374880F30888B5
:1002F000364880F3098836483649086040F20000E5
:10030000CCF200004EF63471CEF200010860BFF36B
:100310004F8FBFF36F8F40F20000C0F2F0004EF637
:100320008851CEF200010860BFF34F8FBFF36F8F8B
:100330004FF00000E1EE100A4EF63C71CEF20001E3
:100340000860062080F31488BFF36F8F02F0C0F8B6
:1003500003F0DCF94FF055301F491B4A91423CBF76
:1003600041F8040BFAE71D49184A91423CBF41F895
:10037000040BFAE71A491B4A1B4B9A423EBF51F83D
:10038000040B42F8040BF8E700201849184A914280
:100390003CBF41F8040BFAE702F0D8F803F03AFA50
:1003A000144C154DAC4203DA54F8041B8847F9E7A6
:1003B00000F042F8114C124DAC4203DA54F8041B21
:1003C0008847F9E702F0C0B80006002000220020AC
:1003D0000000000808ED00E00000002000060020FA
:1003E00028460008002200205C2200206022002015
:1003F00080440020E0020008E0020008E00200085B
:10040000E00200082DE9F04F2DED108AC1F80CD064
:10041000D0F80CD0BDEC108ABDE8F08F002383F338
:1004200011882846A047002001F01AFBFEE701F0E2
:10043000A5FA00DFFEE7000038B500F02DFC02F061
:1004400007F8054602F03AF80446C0B90E4B9D4243
:1004500017D001339D4241F2883512BF0446002572
:100460000124002001F0FEFF0CB100F075F800F04F
:100470006FFD284600F01EF900F06EF8F9E7002540
:10048000EFE70546EDE700BF010007B008B500F053
:10049000D5FBA0F120035842584108BD07B541F2F1
:1004A0001203022101A8ADF8043000F0E5FB03B00F
:1004B0005DF804FB38B5302383F3118817480368CF
:1004C0000BB101F099FB0023154A4FF47A711348E0
:1004D00001F088FB002383F31188124C236813B1C9
:1004E0002368013B2360636813B16368013B636069
:1004F0000D4D2B7833B963687BB9022000F092FC74
:10050000322363602B78032B07D163682BB9022059
:1005100000F088FC4FF47A73636038BD60220020DD
:10052000B50400088023002078220020084B1870B2
:1005300003280CD8DFE800F008050208022000F0CC
:1005400069BC022000F05CBC024B00225A6070477C
:100550007822002080230020F8B5504B504A1C46DA
:100560001968013100F0998004339342F8D1626830
:100570004C4B9A4240F291804B4B9B6803F10063D5
:1005800003F500339A4280F08880002000F0AAFB37
:100590000220FFF7CBFF454B0021D3F8E820C3F83A
:1005A000E810D3F81021C3F81011D3F81021D3F8B4
:1005B000EC20C3F8EC10D3F81421C3F81411D3F8CD
:1005C0001421D3F8F020C3F8F010D3F81821C3F8A1
:1005D0001811D3F81821D3F8802042F00062C3F834
:1005E0008020D3F8802022F00062C3F88020D3F866
:1005F0008020D3F8802042F00072C3F88020D3F826
:10060000802022F00072C3F88020D3F8803072B6C8
:100610004FF0E023C3F8084DD4E90004BFF34F8F37
:10062000BFF36F8F224AC2F88410BFF34F8F536914
:1006300023F480335361BFF34F8FD2F8803043F6F9
:10064000E076C3F3C905C3F34E335B0103EA060C3E
:1006500029464CEA81770139C2F87472F9D2203BFD
:1006600013F1200FF2D1BFF34F8FBFF36F8FBFF3A2
:100670004F8FBFF36F8F536923F40033536100230F
:10068000C2F85032BFF34F8FBFF36F8F302383F325
:100690001188854680F308882047F8BD00000208CD
:1006A00020000208FFFF0108002200200044025839
:1006B00000ED00E02DE9F04F93B0B44B2022FF2174
:1006C00000900AA89D6800F0EDFBB14A1378A3B929
:1006D0000121B04811700360302383F3118803684F
:1006E0000BB101F089FA0023AB4A4FF47A71A948A3
:1006F00001F078FA002383F31188009B13B1A74B14
:10070000009A1A60A64A1378032B03D000231370B3
:10071000A24A53604FF0000A009CD3465646D14689
:10072000012000F077FB24B19C4B1B68002B00F0EC
:100730002682002000F082FA0390039B002BF2DB5C
:10074000012000F05DFB039B213B1F2BE8D801A299
:1007500052F823F0D5070008FD07000891080008AB
:1007600021070008210700082107000823090008C5
:10077000F30A00080D0A00086F0A0008970A00082B
:10078000BD0A000821070008CF0A00082107000859
:10079000410B00087508000821070008850B0008B8
:1007A000E107000875080008210700086F0A000823
:1007B0002107000821070008210700082107000879
:1007C0002107000821070008210700082107000869
:1007D000910800080220FFF759FE002840F0F98137
:1007E000009B022105A8BAF1000F08BF1C4641F288
:1007F0001233ADF8143000F03FFA91E74FF47A70FD
:1008000000F01CFA071EEBDB0220FFF73FFE00287A
:10081000E6D0013F052F00F2DE81DFE807F0030A92
:100820000D1013360523042105A8059300F024FAC2
:1008300017E004215548F9E704215A48F6E7042156
:100840005948F3E74FF01C08404608F1040800F04F
:100850004BFA0421059005A800F00EFAB8F12C0F10
:10086000F2D101204FF0000900FA07F747EA0B0B1D
:100870005FFA8BFB00F062FB26B10BF00B030B2B36
:1008800008BF0024FFF70AFE4AE704214748CDE7E6
:10089000002EA5D00BF00B030B2BA1D10220FFF7EC
:1008A000F5FD074600289BD00120002600F01AFA2B
:1008B0000220FFF73BFE1FFA86F8404600F022FABE
:1008C0000446B0B1039940460136A1F140025142BD
:1008D000514100F027FA0028EDD1BA46044641F212
:1008E0001213022105A83E46ADF8143000F0C4F9F9
:1008F00016E725460120FFF719FE244B9B68AB4203
:1009000007D9284600F0F0F9013040F0678104353E
:10091000F3E70025224BBA463E461D701F4B5D6033
:10092000A8E7002E3FF45CAF0BF00B030B2B7FF41A
:1009300057AF0220FFF7FAFD322000F07FF9B0F147
:100940000008FFF64DAF18F003077FF449AF0F4AD8
:1009500008EB0503926893423FF642AFB8F5807FFB
:100960003FF73EAF124BB845019323DD4FF47A7049
:1009700000F064F90390039A002AFFF631AF039A5E
:100980000137019B03F8012BEDE700BF0022002097
:100990007C23002060220020B50400088023002072
:1009A0007822002004220020082200200C220020AF
:1009B0007C220020C820FFF769FD074600283FF48D
:1009C0000FAF1F2D11D8C5F120020AAB25F003008F
:1009D00084494245184428BF4246019200F03CFA3F
:1009E000019AFF217F4800F05DFA4FEAA803C8F39F
:1009F00087027C492846019300F05CFA06460028ED
:100A00003FF46DAF019B05EB830533E70220FFF751
:100A10003DFD00283FF4E4AE00F0A2F900283FF4C9
:100A2000DFAE0027B846704B9B68BB4218D91F2F1A
:100A300011D80A9B01330ED027F0030312AA1344E6
:100A400053F8203C05934046042205A9043700F0E2
:100A5000ABFA8046E7E7384600F046F90590F2E742
:100A6000CDF81480042105A800F006F902E7002360
:100A7000642104A8049300F0F5F800287FF4B0AED8
:100A80000220FFF703FD00283FF4AAAE049800F00F
:100A90005DF90590E6E70023642104A8049300F0C3
:100AA000E1F800287FF49CAE0220FFF7EFFC00285D
:100AB0003FF496AE049800F04BF9EAE70220FFF706
:100AC000E5FC00283FF48CAE00F05AF9E1E7022083
:100AD000FFF7DCFC00283FF483AE05A9142000F0EA
:100AE00055F907460421049004A800F0C5F83946DA
:100AF000B9E7322000F0A2F8071EFFF671AEBB077F
:100B00007FF46EAE384A07EB0903926893423FF6D2
:100B100067AE0220FFF7BAFC00283FF461AE27F071
:100B200003074F44B9453FF4A5AE484609F104090F
:100B300000F0DAF80421059005A800F09DF8F1E72F
:100B40004FF47A70FFF7A2FC00283FF449AE00F0A2
:100B500007F9002844D00A9B01330BD008220AA9C8
:100B6000002000F0A7F900283AD02022FF210AA88F
:100B700000F098F9FFF792FC1C4800F077FF13B0E3
:100B8000BDE8F08F002E3FF42BAE0BF00B030B2BC8
:100B90007FF426AE0023642105A8059300F062F8D7
:100BA000074600287FF41CAE0220FFF76FFC80464A
:100BB00000283FF415AEFFF771FC41F2883000F0D9
:100BC00055FF059800F0EEF946463C4600F0B6F9B0
:100BD000A6E506464EE64FF0000901E6BA467EE677
:100BE00037467CE67C22002000220020A0860100FF
:100BF0000F4B70B51B780C460133DBB2012B11D8BB
:100C00000C4D4FF47A732968A2FB033222460E6A18
:100C100001462846B047844204D1074B00220120F8
:100C20001A7070BD4FF4FA7000F020FF0020F8E752
:100C30001022002028260020B4230020002307B51E
:100C4000024601210DF107008DF80730FFF7D0FFB4
:100C500020B19DF8070003B05DF804FB4FF0FF30B2
:100C6000F9E700000A46042108B5FFF7C1FF80F04C
:100C70000100C0B2404208BD30B4054C0A460146EE
:100C800023682046DD69034BAC4630BC604700BF9B
:100C900028260020A086010070B5104C0025104EBB
:100CA00001F000FA20803068238883420CD80025A8
:100CB0002088013801F0F2F923880544013BB5F59D
:100CC000802F2380F4D370BD01F0E8F93368054428
:100CD0000133B5F5003F3360E5D3E8E7B6230020E4
:100CE0008823002001F0ACBA00F1006000F500306C
:100CF0000068704700F10060920000F5003001F0DC
:100D00002DBA0000054B1A68054B1B889B1A8342BD
:100D100002D9104401F0C2B9002070478823002096
:100D2000B623002038B50446074D29B12868204471
:100D3000BDE8384001F0CAB92868204401F0B4F990
:100D40000028F3D038BD00BF882300200020704762
:100D500000F1FF5000F58F10D0F800087047000038
:100D6000064991F8243033B100230822086A81F83B
:100D70002430FFF7BFBF0120704700BF8C23002045
:100D8000014B1868704700BF0010005C194B013818
:100D90000322084470B51D68174BC5F30B042D0CD6
:100DA0001E88A6420BD15C680A46013C824213466B
:100DB0000FD214F9016F4EB102F8016BF6E7013A58
:100DC00003F10803ECD181420B4602D22C2203F836
:100DD000012B0424094A1688AE4204D1984284BFEC
:100DE000967803F8016B013C02F10402F3D1581A22
:100DF00070BD00BF0010005C14220020F841000804
:100E0000022803D1024B4FF400229A61704700BFC1
:100E100000100258022802D1014B08229A61704743
:100E200000100258022804D1024A536983F00803D3
:100E3000536170470010025870B504464FF47A763B
:100E40004CB1412C254628BF412506FB05F0641B0B
:100E500000F00CFEF4E770BD002310B5934203D000
:100E6000CC5CC4540133F9E710BD0000013810B563
:100E700010F9013F3BB191F900409C4203D11AB1F6
:100E80000131013AF4E71AB191F90020981A10BD26
:100E90001046FCE703460246D01A12F9011B00294E
:100EA000FAD1704702440346934202D003F8011B73
:100EB000FAE770472DE9F8431F4D14460746884668
:100EC00095F8242052BBDFF870909CB395F824303D
:100ED0002BB92022FF2148462F62FFF7E3FF95F848
:100EE00024004146C0F1080205EB8000A24228BF61
:100EF0002246D6B29200FFF7AFFF95F82430A41B2C
:100F000017441E449044E4B2F6B2082E85F82460DB
:100F1000DBD1FFF725FF0028D7D108E02B6A03EBD0
:100F200082038342CFD0FFF71BFF0028CBD10020E4
:100F3000BDE8F8830120FBE78C230020024B1A78E0
:100F4000024B1A70704700BFB4230020102200200B
:100F500010B5114C114800F0B9F821460F4800F0C7
:100F6000E1F824684FF47A70D4F89020D2F804386D
:100F700043F00203C2F80438FFF75EFF0849204639
:100F800000F0DEF9D4F89020D2F8043823F0020300
:100F9000C2F8043810BD00BFB44200082826002063
:100FA000BC4200087047000030B50A44084D914229
:100FB0000DD011F8013B5840082340F30004013BD9
:100FC0002C4013F0FF0384EA5000F6D1EFE730BD68
:100FD0002083B8ED026843681143016003B11847EC
:100FE0007047000013B5406B00F58054D4F8A43866
:100FF0001A681178042914D1017C022911D11979B8
:10100000012312898B4013420BD101A94C3002F00D
:101010003BF9D4F8A4480246019B2179206800F0EE
:10102000DFF902B010BD0000143002F0BDB80000BE
:101030004FF0FF33143002F0B7B800004C3002F02C
:101040008FB900004FF0FF334C3002F089B9000037
:10105000143002F08BB800004FF0FF31143002F072
:1010600085B800004C3002F05BB900004FF0FF3251
:101070004C3002F055B900000020704710B500F563
:101080008054D4F8A4381A681178042917D1017C47
:10109000022914D15979012352898B4013420ED170
:1010A000143002F01DF8024648B1D4F8A4484FF4B9
:1010B000407361792068BDE8104000F07FB910BD31
:1010C000406BFFF7DBBF0000704700007FB5124B9D
:1010D00001250426044603600023057400F1840200
:1010E00043602946C0E902330C4B0290143001934F
:1010F0004FF44073009601F0CFFF094B04F6944281
:10110000294604F14C000294CDE900634FF440738A
:1011100002F096F804B070BD08420008C110000843
:10112000E50F00080A68302383F311880B790B332D
:1011300042F823004B79133342F823008B7913B123
:101140000B3342F8230000F58053C3F8A4180223A0
:101150000374002080F311887047000038B5037FC6
:10116000044613B190F85430ABB90125201D02217B
:10117000FFF730FF04F114006FF00101257700F054
:101180009DFC04F14C0084F854506FF00101BDE85F
:10119000384000F093BC38BD10B50121044604303E
:1011A000FFF718FF0023237784F8543010BD0000A8
:1011B00038B504460025143001F086FF04F14C00D8
:1011C000257702F055F8201D84F854500121FFF7CF
:1011D00001FF2046BDE83840FFF750BF90F880304F
:1011E00003F06003202B06D190F881200023212AF0
:1011F00003D81F2A06D800207047222AFBD1C0E955
:101200001D3303E0034A426707228267C367012058
:10121000704700BF2C22002037B500F58055D5F867
:10122000A4381A68117804291AD1017C022917D12F
:101230001979012312898B40134211D100F14C041A
:10124000204602F0D5F858B101A9204602F01CF85A
:10125000D5F8A4480246019B2179206800F0C0F827
:1012600003B030BD01F10B03F0B550F8236085B039
:1012700004460D46FEB1302383F3118804EB850745
:10128000301D0821FFF7A6FEFB6806F14C005B69E4
:101290001B681BB1019002F005F8019803A901F049
:1012A000F3FF024648B1039B2946204600F098F818
:1012B000002383F3118805B0F0BDFB685A691268FA
:1012C000002AF5D01B8A013B1340F1D104F18002C2
:1012D000EAE70000133138B550F82140ECB1302373
:1012E00083F3118804F58053D3F8A4281368527946
:1012F00003EB8203DB689B695D6845B104216018DC
:10130000FFF768FE294604F1140001F0F3FE2046C1
:10131000FFF7B4FE002383F3118838BD7047000047
:1013200001F0AAB901234022002110B5044600F8BB
:10133000303BFFF7B7FD0023C4E9013310BD0000C7
:1013400010B53023044683F3118824224160002124
:101350000C30FFF7A7FD204601F0B0F90223002072
:10136000237080F3118810BD70B500EB8103054632
:1013700050690E461446DA6018B110220021FFF7BA
:1013800091FDA06918B110220021FFF78BFD3146B5
:101390002846BDE8704001F097BA0000836820221B
:1013A000002103F0011310B5044683601030FFF7ED
:1013B00079FD2046BDE8104001F012BBF0B40125D4
:1013C00000EB810447898D40E4683D43A469458171
:1013D00023600023A2606360F0BC01F02FBB00001B
:1013E000F0B4012500EB810407898D40E4683D439A
:1013F0006469058123600023A2606360F0BC01F092
:10140000A5BB000070B5022300250446242203700A
:101410002946C0F888500C3040F8045CFFF742FDC4
:10142000204684F8705001F0E3F963681B6823B12B
:1014300029462046BDE87040184770BD0378052B4B
:1014400010B504460AD080F88C3005230370436839
:101450001B680BB1042198470023A36010BD000056
:101460000178052906D190F88C20436802701B682A
:1014700003B118477047000070B590F8703004460B
:1014800013B1002380F8703004F18002204601F08F
:10149000CBFA63689B68B3B994F8803013F06005A9
:1014A00035D00021204601F0BDFD0021204601F08D
:1014B000ADFD63681B6813B10621204698470623DB
:1014C00084F8703070BD204698470028E4D0B4F806
:1014D0008630A26F9A4288BFA36794F98030A56FC7
:1014E000002B4FF0300380F20381002D00F0F280DA
:1014F000092284F8702083F3118800212046D4E962
:101500001D23FFF76DFF002383F31188DAE794F8BA
:10151000812003F07F0343EA022340F20232934228
:1015200000F0C58021D8B3F5807F48D00DD8012BBD
:101530003FD0022B00F09380002BB2D104F188023F
:1015400062670222A267E367C1E7B3F5817F00F01B
:101550009B80B3F5407FA4D194F88230012BA0D1B9
:10156000B4F8883043F0020332E0B3F5006F4DD099
:1015700017D8B3F5A06F31D0A3F5C063012B90D875
:101580006368204694F882205E6894F88310B4F86B
:101590008430B047002884D0436863670368A3673A
:1015A0001AE0B3F5106F36D040F6024293427FF452
:1015B00078AF5C4B63670223A3670023C3E794F80B
:1015C0008230012B7FF46DAFB4F8883023F0020332
:1015D000A4F88830C4E91D55E56778E7B4F8803091
:1015E000B3F5A06F0ED194F88230204684F88A308B
:1015F00001F05CF963681B6813B10121204698472C
:10160000032323700023C4E91D339CE704F18B03FB
:1016100063670123C3E72378042B10D1302383F3BE
:1016200011882046FFF7BAFE85F31188032163680D
:1016300084F88B5021701B680BB12046984794F8B2
:101640008230002BDED084F88B3004232370636853
:101650001B68002BD6D0022120469847D2E794F889
:10166000843020461D0603F00F010AD501F0CEF9A3
:10167000012804D002287FF414AF2B4B9AE72B4BA0
:1016800098E701F0B5F9F3E794F88230002B7FF486
:1016900008AF94F8843013F00F01B3D01A06204637
:1016A00002D501F0D7FCADE701F0C8FCAAE794F839
:1016B0008230002B7FF4F5AE94F8843013F00F01E4
:1016C000A0D01B06204602D501F0ACFC9AE701F041
:1016D0009DFC97E7142284F8702083F311882B4631
:1016E0002A4629462046FFF769FE85F31188E9E678
:1016F0005DB1152284F8702083F311880021204603
:10170000D4E91D23FFF75AFEFDE60B2284F8702072
:1017100083F311882B462A4629462046FFF760FEB0
:10172000E3E700BF384200083042000834420008B6
:1017300038B590F870300446002B3ED0063BDAB244
:101740000F2A34D80F2B32D8DFE803F037313108B5
:10175000223231313131313131313737856FB0F8A3
:1017600086309D4214D2C3681B8AB5FBF3F203FB9B
:1017700012556DB9302383F311882B462A4629462A
:10178000FFF72EFE85F311880A2384F870300EE0EF
:10179000142384F87030302383F31188002320460B
:1017A0001A461946FFF70AFE002383F3118838BD55
:1017B000C36F03B198470023E7E70021204601F0FB
:1017C00031FC0021204601F021FC63681B6813B145
:1017D0000621204698470623D7E7000010B590F869
:1017E00070300446142B29D017D8062B05D001D809
:1017F0001BB110BD093B022BFBD80021204601F094
:1018000011FC0021204601F001FC63681B6813B144
:10181000062120469847062319E0152BE9D10B2312
:1018200080F87030302383F3118800231A4619465C
:10183000FFF7D6FD002383F31188DAE7C3689B69BD
:101840005B68002BD5D1C36F03B19847002384F8A0
:101850007030CEE700238268037503691B689968BE
:101860009142FBD25A680360426010605860704732
:1018700000238268037503691B6899689142FBD84D
:101880005A680360426010605860704708B50846A7
:10189000302383F311880A7D0023052A06D8DFE868
:1018A00002F00B050503120E826913604FF0FF333F
:1018B0008361FFF7CFFF002383F3118808BD82699E
:1018C000936801339360D0E9003213605A60EDE70A
:1018D000FFF7C0BF054BD9680875186802685360E8
:1018E0001A600122D8600275FEF78CBDB823002073
:1018F0000C4B30B5DD684B1C87B004460FD02B462F
:10190000094A684600F06EF92046FFF7E3FF009BA6
:1019100013B1684600F070F9A86907B030BDFFF751
:10192000D9FFF9E7B82300208D18000838B50C4D11
:1019300004468161EB6881689A68914203D8BDE8EA
:101940003840FFF787BF1846FFF792FF0123014693
:10195000EC6020462375BDE83840FEF753BD00BF5C
:10196000B8230020044B1A68DB6890689B68984293
:1019700094BF002001207047B8230020084B10B509
:101980001C68D868226853601A600122DC602275E6
:10199000FFF76EFF01462046BDE81040FEF732BD5E
:1019A000B823002038B50123084C0025237065605A
:1019B00001F05AFD01F080FD0549064801F012FED4
:1019C0000223237085F3118838BD00BF2026002034
:1019D00040420008B823002000F044B9034A51688F
:1019E00053685B1A9842FBD8704700BF001000E0B4
:1019F0008B600223086108468B8270478368A3F1DD
:101A0000840243F8142C026943F8442C426943F8D9
:101A1000402C094A43F8242CC268A3F1200043F863
:101A2000182C022203F80C2C002203F80B2C034A7A
:101A300043F8102C704700BF1D040008B823002095
:101A400008B5FFF7DBFFBDE80840FFF741BF000026
:101A5000024BDB6898610F20FFF73CBFB8230020E2
:101A6000302383F31188FFF7F3BF000008B5014668
:101A7000302383F311880820FFF73AFF002383F314
:101A8000118808BD064BDB6839B1426818605A609E
:101A9000136043600420FFF72BBF4FF0FF30704707
:101AA000B82300200368984206D01A68026050608C
:101AB00018469961FFF70CBF7047000038B504461F
:101AC0000D462068844200D138BD036823605C6005
:101AD0008561FFF7FDFEF4E7036810B59C68A2423C
:101AE0000CD85C688A600B604C6021605960996812
:101AF0008A1A9A604FF0FF33836010BD121B1B6877
:101B0000ECE700000A2938BF0A2170B504460D46EB
:101B10000A26601901F0A2FC01F08AFC041BA54210
:101B200003D8751C04462E46F3E70A2E04D901207B
:101B3000BDE8704001F096BD70BD0000F8B5144BD3
:101B40000D460A2A4FF00A07D96103F1100182609D
:101B500038BF0A2241601969144601604860186163
:101B6000A81801F06BFC01F063FC431B0646A3427E
:101B700006D37C1C28192746354601F06FFCF2E796
:101B80000A2F04D90120BDE8F84001F06BBDF8BD73
:101B9000B8230020F8B506460D4601F049FC0F4A6F
:101BA000134653F8107F9F4206D12A46014630461D
:101BB000BDE8F840FFF7C2BFD169BB68441A2C19D1
:101BC00028BF2C46A34202D92946FFF79BFF224695
:101BD00031460348BDE8F840FFF77EBFB823002038
:101BE000C8230020C0E90323002310B45DF8044B90
:101BF0004361FFF7CFBF000010B5194C236998422D
:101C00000DD08168D0E9003213605A609A680A44A6
:101C10009A60002303604FF0FF33A36110BD026898
:101C2000234643F8102F53600022026022699A4233
:101C300003D1BDE8104001F00BBC936881680B44F0
:101C4000936001F0F5FB2269E1699268441AA242AF
:101C5000E4D91144BDE81040091AFFF753BF00BF93
:101C6000B82300202DE9F047DFF8BC8008F1100709
:101C70002C4ED8F8105001F0DBFBD8F81C40AA68B5
:101C8000031B9A423ED814444FF00009D5E90032B4
:101C9000C8F81C4013605A60C5F80090D8F810309E
:101CA000B34201D101F0D4FB89F31188D5E90331A6
:101CB00028469847302383F311886B69002BD8D0CE
:101CC00001F0B6FB6A69A0EB040982464A450DD2D1
:101CD000022001F0C7FC0022D8F81030B34208D12E
:101CE00051462846BDE8F047FFF728BF121A2244A4
:101CF000F2E712EB09092946384638BF4A46FFF792
:101D0000EBFEB5E7D8F81030B34208D01444C8F859
:101D10001C00211AA960BDE8F047FFF7F3BEBDE83B
:101D2000F08700BFC8230020B823002000207047A0
:101D3000FEE70000704700004FF0FF3070470000E2
:101D400002290CD0032904D00129074818BF00201C
:101D50007047032A05D8054800EBC20070470448C5
:101D600070470020704700BF184300083C22002045
:101D7000CC42000870B59AB005460846144601A941
:101D800000F0C2F801A8FFF785F8431C0022C6B294
:101D90005B001046C5E9003423700323023404F8C5
:101DA000013C01ABD1B202348E4201D81AB070BDF1
:101DB00013F8011B013204F8010C04F8021CF1E7CE
:101DC00008B5302383F311880348FFF725FA002371
:101DD00083F3118808BD00BF2826002090F88030CA
:101DE00003F01F02012A07D190F881200B2A03D1AA
:101DF0000023C0E91D3315E003F06003202B08D158
:101E0000B0F884302BB990F88120212A03D81F2AFA
:101E100004D8FFF7E3B9222AEBD0FAE7034A426776
:101E200007228267C3670120704700BF332200206A
:101E300007B5052917D8DFE801F01916031919208D
:101E4000302383F31188104A01210190FFF78CFAA7
:101E5000019802210D4AFFF787FA0D48FFF7A8F90C
:101E6000002383F3118803B05DF804FB302383F370
:101E700011880748FFF772F9F2E7302383F31188DE
:101E80000348FFF789F9EBE76C420008904200082D
:101E90002826002038B50C4D0C4C2A460C4904F17C
:101EA0000800FFF767FF05F1CA0204F110000949B5
:101EB000FFF760FF05F5CA7204F118000649BDE896
:101EC0003840FFF757BF00BF003F00203C220020F2
:101ED0004C420008564200086142000870B50446B2
:101EE00008460D46FEF7D6FFC6B2204601340378F9
:101EF0000BB9184670BD32462946FEF7B7FF0028D9
:101F0000F3D10120F6E700002DE9F04705460C4625
:101F1000FEF7C0FF2B49C6B22846FFF7DFFF08B126
:101F20000B36F6B228492846FFF7D8FF08B110361D
:101F3000F6B2632E0BD8DFF88C80DFF88C90234F3D
:101F4000DFF894A02E7846B92670BDE8F0872946C0
:101F50002046BDE8F04702F031B9252E2ED10722E8
:101F600041462846FEF782FF70B9194B224603F11D
:101F7000100153F8040B8B4242F8040BF9D11B8873
:101F8000073512341380DDE7082249462846FEF75C
:101F90006DFF98B9A21C0F4B197802320909C95D6F
:101FA00002F8041C13F8011B01F00F015345C95D31
:101FB00002F8031CF0D118340835C3E7013504F8E2
:101FC000016BBFE738430008614200085343000833
:101FD0004043000800E8F11F0CE8F11FBFF34F8FEA
:101FE000044B1A695107FCD1D3F810215207F8D1DC
:101FF000704700BF0020005208B50D4B1B78ABB9ED
:10200000FFF7ECFF0B4BDA68D10704D50A4A5A6098
:1020100002F188325A60D3F80C21D20706D5064A5D
:10202000C3F8042102F18832C3F8042108BD00BFBF
:102030005E410020002000522301674508B5114B86
:102040001B78F3B9104B1A69510703D5DA6842F0CF
:102050004002DA60D3F81021520705D5D3F80C21DD
:1020600042F04002C3F80C21FFF7B8FF064BDA68D4
:1020700042F00102DA60D3F80C2142F00102C3F809
:102080000C2108BD5E410020002000520F289ABF9D
:1020900000F5806040040020704700004FF40030DD
:1020A00070470000102070470F2808B50BD8FFF7C5
:1020B000EDFF00F500330268013204D104308342A1
:1020C000F9D1012008BD0020FCE700000F2838B539
:1020D00005463FD8FFF782FF1F4CFFF78DFF4FF0FB
:1020E000FF3307286361C4F814311DD82361FFF75B
:1020F00075FF030243F02403E360E36843F08003C9
:10210000E36023695A07FCD42846FFF767FFFFF70F
:10211000BDFF4FF4003100F0B3F92846FFF78EFF02
:10212000BDE83840FFF7C0BFC4F81031FFF756FFD5
:10213000A0F108031B0243F02403C4F80C31D4F8C7
:102140000C3143F08003C4F80C31D4F810315B0734
:10215000FBD4D9E7002038BD002000522DE9F84F0C
:1021600005460C46104645EA0203DE0602D0002072
:10217000BDE8F88F20F01F00DFF8BCB0DFF8BCA08E
:10218000FFF73AFF04EB0008444503D10120FFF7B5
:1021900055FFEDE720222946204601F0FFFF10B948
:1021A00020352034F0E72B4605F120021F68791C0A
:1021B000DDD104339A42F9D105F178431B481C4E16
:1021C000B3F5801F1B4B38BF184603F1F80332BF2D
:1021D000D946D1461E46FFF701FF0760A5EB040C68
:1021E000336804F11C0143F002033360231FD9F864
:1021F000007017F00507FAD153F8042F8B424CF802
:102200000320F4D1BFF34F8FFFF7E8FE4FF0FF3309
:102210002022214603602846336823F002033360FE
:1022200001F0BCFF0028BBD03846B0E714210052B3
:102230000C20005214200052102000521021005295
:1022400010B5084C237828B11BB9FFF7D5FE012340
:10225000237010BD002BFCD02070BDE81040FFF7AC
:10226000EDBE00BF5E4100202DE9F04F0D4685B068
:10227000814658B111F00D0614BF2022082211F03A
:102280000803019304D0431E03426AD0002435E0C2
:10229000002E37D009F11F0121F01F094FF001086E
:1022A000324F05F00403DFF8D0A005EA080BBBF1BC
:1022B000000F32D07869C0072FD408F101080C371D
:1022C000B8F1060FF3D19EB9294D4946A8190192DC
:1022D00001F014F9044600283AD11836019A782EF4
:1022E000F3D1494601F00AF90446002830D1019A99
:1022F0004946204801F002F9044668BB204605B073
:10230000BDE8F08F0029C9D101462846029201F0AC
:10231000F5F80446E0B9029AC0E713B178694107BD
:10232000CBD5AC0702D578698007C6D5019911B124
:1023300078690107C1D51820494600FB08A0CDE9FE
:10234000022301F0DBF80446DDE902230028B4D0C3
:102350004A460021204601E04A460021FEF7A2FD40
:10236000CCE70246002E95D198E700BF64430008F1
:102370009041002060410020784100200121FFF7BA
:1023800073BF0000F8B5144D01241827134E40F216
:10239000FF3200210120FEF785FD07FB04600134B8
:1023A0002A6955F80C1F01F095F8062CF5D1372550
:1023B0004FF4C0542046FFF7E1FF014628B1224602
:1023C0000748BDE8F84001F085B8C4EBC404013DFE
:1023D0004FEAD404EED1F8BD6443000878410020F0
:1023E000604100200244074BD2B210B5904200D1A8
:1023F00010BD441C00B253F8200041F8040BE0B2B9
:10240000F4E700BF504000580E4B30B51C6F240459
:1024100005D41C6F1C671C6F44F400441C670A4CF5
:1024200002442368D2B243F480732360074B904286
:1024300000D130BD441C51F8045B00B243F8205079
:10244000E0B2F4E7004402580048025850400058F7
:1024500007B5012201A90020FFF7C4FF019803B0CE
:102460005DF804FB13B50446FFF7F2FFA04205D068
:10247000012201A900200194FFF7C6FF02B010BDA0
:102480000144BFF34F8F064B884204D3BFF34F8FF5
:10249000BFF36F8F7047C3F85C022030F4E700BFD2
:1024A00000ED00E0034B1A681AB9034AD2F8D024B1
:1024B0001A607047084200200040025808B5FFF734
:1024C000F1FF024B1868C0F3806008BD084200208D
:1024D00070B5BFF34F8FBFF36F8F1A4A0021C2F858
:1024E0005012BFF34F8FBFF36F8F536943F4003324
:1024F0005361BFF34F8FBFF36F8FC2F88410BFF3E8
:102500004F8FD2F8803043F6E074C3F3C900C3F3B1
:102510004E335B0103EA0406014646EA8175013940
:10252000C2F86052F9D2203B13F1200FF2D1BFF371
:102530004F8F536943F480335361BFF34F8FBFF321
:102540006F8F70BD00ED00E0FEE70000214B2248D8
:10255000224A70B5904237D3214BC11EDA1C121AA1
:1025600022F003028B4238BF00220021FEF79AFCC2
:102570001C4A0023C2F88430BFF34F8FD2F880305A
:1025800043F6E074C3F3C900C3F34E335B0103EABF
:102590000406014646EA81750139C2F86C52F9D247
:1025A000203B13F1200FF2D1BFF34F8FBFF36F8F9A
:1025B000BFF34F8FBFF36F8F0023C2F85032BFF3CA
:1025C0004F8FBFF36F8F70BD53F8041B40F8041B8F
:1025D000C0E700BF844600088044002080440020FB
:1025E0008044002000ED00E0074BD3F8D81021EA2A
:1025F0000001C3F8D810D3F8002122EA0002C3F882
:102600000021D3F8003170470044025870B5D0E97A
:10261000244300224FF0FF359E6804EB4213510122
:10262000D3F80009002805DAD3F8000940F080400B
:10263000C3F80009D3F8000B002805DAD3F8000B23
:1026400040F08040C3F8000B013263189642C3F893
:102650000859C3F8085BE0D24FF00113C4F81C38E6
:1026600070BD0000890141F02001016103699B06F2
:10267000FCD41220FFF7B2B910B50A4C2046FEF781
:1026800051FE094BC4F89030084BC4F89430084C04
:102690002046FEF747FE074BC4F89030064BC4F8BF
:1026A000943010BD0C42002000000840D0430008C8
:1026B000A842002000000440DC43000870B5037805
:1026C0000546012B5CD1434BD0F89040984258D13D
:1026D000414B0E216520D3F8D82042F00062C3F8A8
:1026E000D820D3F8002142F00062C3F80021D3F8CB
:1026F0000021D3F8802042F00062C3F88020D3F894
:10270000802022F00062C3F88020D3F8803000F0EF
:10271000ADFC324BE360324BC4F800380023D5F8EF
:102720009060C4F8003EC02323604FF40413A363F9
:102730003369002BFCDA01230C203361FFF74EF9DB
:102740003369DB07FCD41220FFF748F93369002B0B
:10275000FCDA00262846A660FFF758FF6B68C4F82D
:102760001068DB68C4F81468C4F81C6883BB1D4B90
:10277000A3614FF0FF336361A36843F00103A360DB
:1027800070BD194B9842C9D1134B4FF08060D3F8FC
:10279000D82042F00072C3F8D820D3F8002142F0CC
:1027A0000072C3F80021D3F80021D3F8802042F052
:1027B0000072C3F88020D3F8802022F00072C3F8A2
:1027C0008020D3F88030FFF70FFF0E214D209EE7C9
:1027D000064BCDE70C420020004402584014004054
:1027E00003002002003C30C0A8420020083C30C05A
:1027F000F8B5D0F89040054600214FF0006620461D
:10280000FFF730FFD5F8941000234FF001128F68C6
:102810004FF0FF30C4F83438C4F81C2804EB4312DE
:1028200001339F42C2F80069C2F8006BC2F8080980
:10283000C2F8080BF2D20B68D5F89020C5F8983092
:10284000636210231361166916F01006FBD1122083
:10285000FFF7C4F8D4F8003823F4FE63C4F8003856
:10286000A36943F4402343F01003A3610923C4F890
:102870001038C4F814380B4BEB604FF0C043C4F869
:10288000103B094BC4F8003BC4F81069C4F8003988
:10289000D5F8983003F1100243F48013C5F898205E
:1028A000A362F8BDAC43000840800010D0F890202F
:1028B00090F88A10D2F8003823F4FE6343EA01133B
:1028C000C2F80038704700002DE9F84300EB81039F
:1028D000D0F890500C468046DA680FFA81F948012A
:1028E000166806F00306731E022B05EB41134FF02A
:1028F000000194BFB604384EC3F8101B4FF001011D
:1029000004F1100398BF06F1805601FA03F39169B0
:1029100098BF06F5004600293AD0578A04F15801BD
:10292000374349016F50D5F81C180B430021C5F8F7
:102930001C382B180127C3F81019A7405369611ED2
:102940009BB3138A928B9B08012A88BF5343D8F804
:102950009820981842EA034301F140022146C8F842
:102960009800284605EB82025360FFF77BFE08EBD8
:102970008900C3681B8A43EA845348341E436401B8
:102980002E51D5F81C381F43C5F81C78BDE8F883D4
:1029900005EB4917D7F8001B21F40041C7F8001BCD
:1029A000D5F81C1821EA0303C0E704F13F030B4AE2
:1029B0002846214605EB83035A60FFF753FE05EBDB
:1029C0004910D0F8003923F40043C0F80039D5F895
:1029D0001C3823EA0707D7E7008000100004000234
:1029E000D0F894201268C0F89820FFF70FBE0000BE
:1029F0005831D0F8903049015B5813F4004004D0AE
:102A000013F4001F0CBF0220012070474831D0F89A
:102A1000903049015B5813F4004004D013F4001FB8
:102A20000CBF02200120704700EB8101CB68196ABE
:102A30000B6813604B6853607047000000EB810324
:102A400030B5DD68AA691368D36019B9402B84BF1B
:102A5000402313606B8A1468D0F890201C4402EB6A
:102A60004110013C09B2B4FBF3F46343033323F098
:102A7000030343EAC44343F0C043C0F8103B2B6850
:102A800003F00303012B0ED1D2F8083802EB4110FA
:102A900013F4807FD0F8003B14BF43F0805343F021
:102AA0000053C0F8003B02EB4112D2F8003B43F068
:102AB0000443C2F8003B30BD2DE9F041D0F89060EE
:102AC00005460C4606EB4113D3F8087B3A07C3F8DA
:102AD000087B08D5D6F814381B0704D500EB810312
:102AE000DB685B689847FA071FD5D6F81438DB0710
:102AF0001BD505EB8403D968CCB98B69488A5A6821
:102B0000B2FBF0F600FB16228AB91868DA68904228
:102B10000DD2121AC3E90024302383F31188214611
:102B20002846FFF78BFF84F31188BDE8F08101236D
:102B300003FA04F26B8923EA02036B81CB68002B52
:102B4000F3D021462846BDE8F041184700EB810349
:102B50004A0170B5DD68D0F890306C692668E6608F
:102B600056BB1A444FF40020C2F810092A6802F03C
:102B70000302012A0AB20ED1D3F8080803EB42146B
:102B800010F4807FD4F8000914BF40F0805040F06A
:102B90000050C4F8000903EB4212D2F8000940F0DB
:102BA0000440C2F800090122D3F8340802FA01F106
:102BB0000143C3F8341870BD19B9402E84BF4020BA
:102BC000206020681A442E8A8419013CB4FBF6F474
:102BD00040EAC44040F00050C6E700002DE9F84349
:102BE000D0F8906005460C464F0106EB4113D3F830
:102BF000088918F0010FC3F808891CD0D6F81038DE
:102C0000DB0718D500EB8103D3F80CC0DCF81430D7
:102C1000D3F800E0DA68964530D2A2EB0E024FF00E
:102C200000091A60C3F80490302383F31188FFF77A
:102C30008DFF89F3118818F0800F1DD0D6F8343835
:102C40000126A640334217D005EB84030134D5F8A2
:102C50009050D3F80CC0E4B22F44DCF8142005EBFC
:102C60000434D2F800E05168714514D3D5F83438F3
:102C700023EA0606C5F83468BDE8F883012303FAA1
:102C800001F2038923EA02030381DCF80830002BF8
:102C9000D1D09847CFE7AEEB0103BCF810008342D8
:102CA00028BF0346D7F8180980B2B3EB800FE3D8EA
:102CB0009068A0F1040959F8048FC4F80080A0EBD3
:102CC00009089844B8F1040FF5D818440B449060F3
:102CD0005360C8E72DE9F84FD0F8905004466E696C
:102CE000AB691E4016F480586E6103D0BDE8F84F02
:102CF000FEF788BB002E12DAD5F8003E9B0705D000
:102D0000D5F8003E23F00303C5F8003ED5F804389B
:102D1000204623F00103C5F80438FEF7A1FB370570
:102D200005D52046FFF772FC2046FEF787FBB0046E
:102D30000CD5D5F8083813F0060FEB6823F4705360
:102D40000CBF43F4105343F4A053EB6031071BD581
:102D50006368DB681BB9AB6923F00803AB612378B8
:102D6000052B0CD1D5F8003E9A0705D0D5F8003ECA
:102D700023F00303C5F8003E2046FEF771FB6368AD
:102D8000DB680BB120469847F30200F1BA80B70226
:102D900026D5D4F8909000274FF0010A09EB47128E
:102DA000D2F8003B03F44023B3F5802F11D1D2F8C1
:102DB000003B002B0DDA62890AFA07F322EA0303CB
:102DC000638104EB8703DB68DB6813B13946204677
:102DD00098470137D4F89430FFB29B689F42DDD901
:102DE000F00619D5D4F89000026AC2F30A1702F06F
:102DF0000F0302F4F012B2F5802F00F0CA80B2F592
:102E0000402F09D104EB8303002200F58050DB68DA
:102E10001B6A974240F0B0803003D5F8185835D57A
:102E2000E90303D500212046FFF746FEAA0303D598
:102E300001212046FFF740FE6B0303D50221204607
:102E4000FFF73AFE2F0303D503212046FFF734FE98
:102E5000E80203D504212046FFF72EFEA90203D580
:102E600005212046FFF728FE6A0203D506212046E9
:102E7000FFF722FE2B0203D507212046FFF71CFE99
:102E8000EF0103D508212046FFF716FE700340F13D
:102E9000A780E90703D500212046FFF79FFEAA0778
:102EA00003D501212046FFF799FE6B0703D50221C8
:102EB0002046FFF793FE2F0703D503212046FFF797
:102EC0008DFEEE0603D504212046FFF787FEA806F7
:102ED00003D505212046FFF781FE690603D50621AB
:102EE0002046FFF77BFE2A0603D507212046FFF781
:102EF00075FEEB0574D520460821BDE8F84FFFF7B5
:102F00006DBED4F890904FF0000B4FF0010AD4F84A
:102F100094305FFA8BF79B689F423FF638AF09EB1E
:102F20004713D3F8002902F44022B2F5802F20D1B4
:102F3000D3F80029002A1CDAD3F8002942F0904285
:102F4000C3F80029D3F80029002AFBDB3946D4F85E
:102F50009000FFF787FB22890AFA07F322EA0303AE
:102F6000238104EB8703DB689B6813B13946204655
:102F700098470BF1010BCAE7910701D1D0F8008007
:102F8000072A02F101029CBF03F8018B4FEA1828BF
:102F90003FE704EB830300F58050DA68D2F818C0ED
:102FA000DCF80820DCE9001CA1EB0C0C00218F42AE
:102FB00008D1DB689B699A683A449A605A683A4437
:102FC0005A6029E711F0030F01D1D0F800808C4539
:102FD00001F1010184BF02F8018B4FEA1828E6E7EE
:102FE000BDE8F88F08B50348FFF774FEBDE8084058
:102FF00000F074BC0C42002008B50348FFF76AFEDD
:10300000BDE8084000F06ABCA8420020D0F890302B
:1030100003EB4111D1F8003B43F40013C1F8003B2E
:1030200070470000D0F8903003EB4111D1F800391F
:1030300043F40013C1F8003970470000D0F8903015
:1030400003EB4111D1F8003B23F40013C1F8003B1E
:1030500070470000D0F8903003EB4111D1F80039EF
:1030600023F40013C1F8003970470000090100F192
:103070006043012203F56143C9B283F8001300F0F5
:103080001F039A4043099B0003F1604303F561432A
:10309000C3F880211A60704730B50433039C017275
:1030A000002104FB0325C160C0E90653049B0363B0
:1030B000059BC0E90000C0E90422C0E90842C0E95C
:1030C0000A11436330BD00000022416AC260C0E9BA
:1030D0000411C0E90A226FF00101FEF7EFBC000005
:1030E000D0E90432934201D1C2680AB9181D704771
:1030F00000207047036919600021C2680132C26074
:10310000C269134482699342036124BF436A036125
:10311000FEF7C8BC38B504460D46E3683BB16269AA
:103120000020131D1268A3621344E36207E0237AB0
:1031300033B929462046FEF7A5FC0028EDDA38BD54
:103140006FF00100FBE70000C368C269013BC36088
:103150004369134482699342436124BF436A4361D4
:1031600000238362036B03B11847704770B53023A7
:10317000044683F31188866A3EB9FFF7CBFF054604
:1031800018B186F31188284670BDA36AE26A13F865
:10319000015B9342A36202D32046FFF7D5FF0023D1
:1031A00083F31188EFE700002DE9F84F04460E463F
:1031B000174698464FF0300989F311880025AA4632
:1031C000D4F828B0BBF1000F09D141462046FFF7E3
:1031D000A1FF20B18BF311882846BDE8F88FD4E910
:1031E0000A12A7EB050B521A934528BF9346BBF171
:1031F000400F1BD9334601F1400251F8040B9142B4
:1032000043F8040BF9D1A36A403640354033A3623A
:10321000D4E90A239A4202D32046FFF795FF8AF3A6
:103220001188BD42D8D289F31188C9E730465A4681
:10323000FDF712FEA36A5E445D445B44A362E7E7C8
:1032400010B5029C0433017203FB0421C460C0E981
:1032500006130023C0E90A33039B0363049BC0E900
:103260000000C0E90422C0E90842436310BD000029
:10327000026A6FF00101C260426AC0E904220022C2
:10328000C0E90A22FEF71ABCD0E904239A4201D110
:10329000C26822B9184650F8043B0B6070470023FF
:1032A0001846FAE7C3680021C2690133C360436965
:1032B000134482699342436124BF436A4361FEF72A
:1032C000F1BB000038B504460D46E3683BB1236905
:1032D00000201A1DA262E2691344E36207E0237A28
:1032E00033B929462046FEF7CDFB0028EDDA38BD7C
:1032F0006FF00100FBE7000003691960C268013A42
:10330000C260C269134482699342036124BF436A65
:10331000036100238362036B03B118477047000009
:1033200070B530230D460446114683F31188866A32
:103330002EB9FFF7C7FF10B186F3118870BDA36ADD
:103340001D70A36AE26A01339342A36204D3E16968
:1033500020460439FFF7D0FF002080F31188EDE705
:103360002DE9F84F04460D46904699464FF0300A35
:103370008AF311880026B346A76A4FB9494620460A
:10338000FFF7A0FF20B187F311883046BDE8F88F22
:10339000D4E90A073A1AA8EB0607974228BF17464E
:1033A000402F1BD905F1400355F8042B9D4240F8EE
:1033B000042BF9D1A36A40364033A362D4E90A232F
:1033C0009A4204D3E16920460439FFF795FF8BF355
:1033D00011884645D9D28AF31188CDE729463A4665
:1033E000FDF73AFDA36A3D443E443B44A362E5E752
:1033F000D0E904239A4217D1C3689BB1836A8BB189
:10340000043B9B1A0ED01360C368013BC360C369C1
:103410001A4483699A42026124BF436A036100230C
:1034200083620123184670470023FBE700F080BA4F
:10343000014B586A704700BF000C0040034B00224C
:1034400058631A610222DA60704700BF000C004026
:10345000014B0022DA607047000C0040014B5863BA
:10346000704700BF000C0040024B034A1A60034A39
:103470005A6070475C430020804400200000022016
:10348000074B494210B55C68201A08401968821A37
:103490008A4203D3A24201D85A6010BD0020FCE743
:1034A0005C43002008B5302383F31188FFF7E8FF61
:1034B000002383F3118808BD04480121044B0360F5
:1034C0000023C0E901330C3000F0D4B8644300207D
:1034D000A5340008CB1D083A23F00703591A521AE5
:1034E000012110B4D2080024C0E9004384600C30EC
:1034F0001C605A605DF8044B00F0BCB82DE9F84F31
:10350000364ECD1D0F46002818BF0646082A4FEA42
:10351000D50538BF082206F10C08341D91464046F7
:1035200000F0C4F809F10701C9F1000E2246246831
:103530006CB9404600F0C4F83368CBB30822494662
:10354000E8009847044698B340E9026730E004EB8E
:10355000010CD4F804A00CEA0E0C0AF10100ACF145
:10356000080304EBC0009842E0D9A0EB0C0CB5EBCB
:10357000EC0F4FEAEC0BD9D89C421CD204F10802A4
:10358000AB45A3EB02024FEAE202626009D9691C73
:10359000ED43206803EBC1025D44556043F8310000
:1035A00022601C465F60404644F8086B00F088F8D3
:1035B0002046BDE8F88FAA45216802D11160234654
:1035C000EFE7013504EBC50344F8351003F10801BA
:1035D000401AC01058601360F1E700BF6443002038
:1035E000FEE7000070B51B4B0025044686B058600E
:1035F0000E468562016300F049F904F11003A560ED
:10360000E562C4E904334FF0FF33C4E90044C4E980
:103610000635FFF70DFF2B46024604F13401204624
:10362000C4E9082380230C4A2565FEF7E1F901234C
:103630000A4AE06000920375684672680192B268B7
:10364000CDE90223064BCDE90435FEF7F9F906B0C2
:1036500070BD00BF20260020E8430008ED430008AD
:10366000E1350008024AD36A1843D062704700BFB0
:10367000B8230020C0E90000816070478368013BE7
:10368000002B10B583600CDA074BDC684368A0613F
:10369000206063601C6044600520FEF71BF9A06990
:1036A00010BD0020FCE700BFB823002008B5302380
:1036B00083F31188FFF7E2FF002383F3118808BD2D
:1036C00008B5302383F3118883680133002B8360AE
:1036D00007DC036800211A68026050601846FEF794
:1036E00025F9002383F3118808BD00004B6843606F
:1036F0008B688360CB68C3600B6943614B6903626D
:103700008B6943620B6803607047000008B53C4B4F
:1037100040F2FF713B48D3F888200A43C3F8882061
:10372000D3F8882022F4FF6222F00702C3F8882031
:10373000D3F88820D3F8E0200A43C3F8E020D3F878
:1037400008210A43C3F808212F4AD3F8083111464B
:10375000FFF7CCFF00F5806002F11C01FFF7C6FF08
:1037600000F5806002F13801FFF7C0FF00F58060CE
:1037700002F15401FFF7BAFF00F5806002F1700119
:10378000FFF7B4FF00F5806002F18C01FFF7AEFF98
:1037900000F5806002F1A801FFF7A8FF00F5806046
:1037A00002F1C401FFF7A2FF00F5806002F1E00121
:1037B000FFF79CFF00F5806002F1FC01FFF796FF28
:1037C00002F58C7100F58060FFF790FF00F07CF946
:1037D0000E4BD3F8902242F00102C3F89022D3F8A6
:1037E000942242F00102C3F894220522C3F89820E3
:1037F0004FF06052C3F89C20054AC3F8A02008BDD2
:103800000044025800000258F443000800ED00E0B4
:103810001F00080308B500F02BFBFEF7C3F8104BA0
:10382000D3F8DC2042F04002C3F8DC20D3F80421B6
:1038300022F04002C3F80421D3F80431094B1A687E
:1038400042F008021A601A6842F004021A60FEF799
:1038500029FEFEF797FDBDE80840FEF71BBB00BF41
:10386000004402580018024870470000EFF3098333
:10387000054968334A6B22F001024A6383F30988E1
:10388000002383F31188704700EF00E0302080F3BD
:10389000118862B60D4B0E4AD96821F4E061090423
:1038A000090C0A430B49DA60D3F8FC2042F080721D
:1038B000C3F8FC20084AC2F8B01F116841F00101AA
:1038C00011602022DA7783F82200704700ED00E0D3
:1038D0000003FA0555CEACC5001000E0302310B54A
:1038E00083F311880E4B5B6813F4006314D0F1EE80
:1038F000103AEFF309844FF08073683CE361094BA1
:10390000DB6B236684F30988FEF72CF810B1064BB5
:10391000A36110BD054BFBE783F31188F9E700BFF6
:1039200000ED00E000EF00E02F0400083204000882
:10393000114BD3F8E82042F00802C3F8E820D3F88E
:10394000102142F00802C3F810210C4AD3F81031BC
:10395000D36B43F00803D363C722094B9A624FF03D
:10396000FF32DA6200229A615A63DA605A600122F9
:103970005A611A60704700BF004402580010005C92
:10398000000C0040094A08B51169D3680B40D9B250
:103990009B076FEA0101116107D5302383F311887A
:1039A000FEF71AF8002383F3118808BD000C0040CD
:1039B000064BD3F8DC200243C3F8DC20D3F8042103
:1039C0001043C3F80401D3F804317047004402588F
:1039D00008B53C4B4FF0FF31D3F8802062F0004235
:1039E000C3F88020D3F8802002F00042C3F8802082
:1039F000D3F88020D3F88420C3F88410D3F884202F
:103A00000022C3F88420D3F88400D86F40F0FF4030
:103A100040F4FF0040F4DF4040F07F00D867D86FEB
:103A200020F0FF4020F4FF0020F4DF4020F07F0072
:103A3000D867D86FD3F888006FEA40506FEA5050CB
:103A4000C3F88800D3F88800C0F30A00C3F88800E0
:103A5000D3F88800D3F89000C3F89010D3F8900002
:103A6000C3F89020D3F89000D3F89400C3F89410D2
:103A7000D3F89400C3F89420D3F89400D3F89800B6
:103A8000C3F89810D3F89800C3F89820D3F898009A
:103A9000D3F88C00C3F88C10D3F88C00C3F88C20BA
:103AA000D3F88C00D3F89C00C3F89C10D3F89C107A
:103AB000C3F89C20D3F89C3000F042FBBDE80840DE
:103AC00000F0AEB90044025808B50122534BC3F8C8
:103AD0000821534BD3F8F42042F00202C3F8F4203B
:103AE000D3F81C2142F00202C3F81C210222D3F8B1
:103AF0001C314C4BDA605A689104FCD54A4A1A6072
:103B000001229A60494ADA6000221A614FF4404269
:103B10009A61444B9A699204FCD51A6842F4807207
:103B20001A603F4B1A6F12F4407F04D04FF480327A
:103B30001A6700221A671A6842F001021A60384BAD
:103B40001A685007FCD500221A611A6912F038026F
:103B5000FBD1012119604FF0804159605A67344A06
:103B6000DA62344A1A611A6842F480321A602C4BC5
:103B70001A689103FCD51A6842F480521A601A68D8
:103B80009204FCD52C4A2D499A6200225A6319638B
:103B900001F57C01DA6301F2E71199635A64284A5E
:103BA0001A64284ADA621A6842F0A8521A601C4B5A
:103BB0001A6802F02852B2F1285FF9D148229A61BE
:103BC0004FF48862DA6140221A621F4ADA641F4A9F
:103BD0001A651F4A5A651F4A9A6532231E4A1360A6
:103BE000136803F00F03022BFAD10D4A136943F057
:103BF00003031361136903F03803182BFAD14FF054
:103C00000050FFF7D5FE4FF08040FFF7D1FE4FF098
:103C10000040BDE80840FFF7CBBE00BF0080005168
:103C2000004402580048025800C000F002000001A1
:103C30000000FF01008890081210200063020901B3
:103C4000470E0508DD0BBF01200000200000011019
:103C50000910E00000010110002000524FF0B042B6
:103C600008B5D2F8883003F00103C2F8883023B1D8
:103C7000044A13680BB150689847BDE80840FFF745
:103C80002DBE00BF004400204FF0B04208B5D2F86E
:103C9000883003F00203C2F8883023B1044A9368E5
:103CA0000BB1D0689847BDE80840FFF717BE00BFCA
:103CB000004400204FF0B04208B5D2F8883003F03D
:103CC0000403C2F8883023B1044A13690BB1506968
:103CD0009847BDE80840FFF701BE00BF0044002040
:103CE0004FF0B04208B5D2F8883003F00803C2F8AC
:103CF000883023B1044A93690BB1D0699847BDE875
:103D00000840FFF7EBBD00BF004400204FF0B04279
:103D100008B5D2F8883003F01003C2F8883023B118
:103D2000044A136A0BB1506A9847BDE80840FFF790
:103D3000D5BD00BF004400204FF0B04310B5D3F80C
:103D4000884004F47872C3F88820A30604D5124A88
:103D5000936A0BB1D06A9847600604D50E4A136B7C
:103D60000BB1506B9847210604D50B4A936B0BB1EE
:103D7000D06B9847E20504D5074A136C0BB1506C21
:103D80009847A30504D5044A936C0BB1D06C9847AF
:103D9000BDE81040FFF7A2BD004400204FF0B04343
:103DA00010B5D3F8884004F47C42C3F8882062053B
:103DB00004D5164A136D0BB1506D9847230504D5F1
:103DC000124A936D0BB1D06D9847E00404D50F4AA9
:103DD000136E0BB1506E9847A10404D50B4A936E35
:103DE0000BB1D06E9847620404D5084A136F0BB12B
:103DF000506F9847230404D5044A936F0BB1D06FDA
:103E00009847BDE81040FFF769BD00BF004400209F
:103E100008B5FFF7B7FDBDE80840FFF75FBD00003C
:103E2000062108B50846FFF721F906210720FFF70C
:103E30001DF906210820FFF719F906210920FFF7CF
:103E400015F906210A20FFF711F906211720FFF7BF
:103E50000DF906212820FFF709F909217A20FFF73B
:103E600005F907213220BDE80840FFF7FFB8000040
:103E700008B5FFF7ADFD00F083F9FDF751FAFDF746
:103E800023F9FFF7F1FCBDE80840FFF7CFBA0000C7
:103E900008B5074B074A196801F03D01996053685E
:103EA0000BB190689847BDE80840FFF717BD00BF09
:103EB000000002407C43002008B5084B19688909BE
:103EC00001F03D018A019A60054AD3680BB110697F
:103ED0009847BDE80840FFF701BD00BF0000024061
:103EE0007C43002008B5084B1968090C01F03D011E
:103EF0000A049A60054A53690BB190699847BDE876
:103F00000840FFF7EBBC00BF000002407C430020EC
:103F100008B5084B1968890D01F03D018A059A60C2
:103F2000054AD3690BB1106A9847BDE80840FFF70E
:103F3000D5BC00BF000002407C43002008B5074B01
:103F4000074A596801F03D01D960536A0BB1906A84
:103F50009847BDE80840FFF7C1BC00BF0000024021
:103F60007C43002008B5084B5968890901F03D01E0
:103F70008A01DA60054AD36A0BB1106B9847BDE835
:103F80000840FFF7ABBC00BF000002407C430020AC
:103F900008B5084B5968090C01F03D010A04DA60C4
:103FA000054A536B0BB1906B9847BDE80840FFF78B
:103FB00095BC00BF000002407C43002008B5084BC0
:103FC0005968890D01F03D018A05DA60054AD36B15
:103FD0000BB1106C9847BDE80840FFF77FBC00BFED
:103FE000000002407C43002008B5074B074A1968CF
:103FF00001F03D019960536C0BB1906C9847BDE89E
:104000000840FFF76BBC00BF000402407C43002067
:1040100008B5084B1968890901F03D018A019A60C9
:10402000054AD36C0BB1106D9847BDE80840FFF707
:1040300055BC00BF000402407C43002008B5084B7B
:104040001968090C01F03D010A049A60054A536D94
:104050000BB1906D9847BDE80840FFF73FBC00BF2B
:10406000000402407C43002008B5084B1968890D04
:1040700001F03D018A059A60054AD36D0BB1106EBF
:104080009847BDE80840FFF729BC00BF0004024084
:104090007C43002008B5074B074A596801F03D01F1
:1040A000D960536E0BB1906E9847BDE80840FFF79A
:1040B00015BC00BF000402407C43002008B5084B3B
:1040C0005968890901F03D018A01DA60054AD36E19
:1040D0000BB1106F9847BDE80840FFF7FFBB00BF6A
:1040E000000402407C43002008B5084B5968090CC5
:1040F00001F03D010A04DA60054A536F0BB1906F7D
:104100009847BDE80840FFF7E9BB00BF0004024044
:104110007C43002008B5084B5968890D01F03D012A
:104120008A05DA60054AD36F13B1D2F88000984748
:10413000BDE80840FFF7D2BB000402407C430020EA
:1041400000230C4910B51A460B4C0B6054F82300A1
:10415000026001EB430004334260402BF6D1074A72
:104160004FF0FF339360D360C2F80834C2F80C34C8
:1041700010BD00BF7C43002028450008000002401D
:104180000023054A19460133102BC2E9001102F140
:104190000802F8D1704700BF0044002010B5013973
:1041A0000244904201D1002005E0037811F8014F4C
:1041B000A34201D0181B10BD0130F2E7034611F8ED
:1041C000012B03F8012B002AF9D1704753544D33CA
:1041D0003248373F3F3F0053544D333248373378EE
:1041E0002F3732780053544D3332483734332F371A
:1041F00035332F373530000001105A0003105900B5
:10420000012058000320560000000000451000085F
:10421000311000086D1000085910000865100008E2
:10422000511000083D1000082910000879100008FE
:1042300000000000010000000000000063300000EA
:104240003C420008102400202026002041726475A2
:1042500050696C6F740025424F415244252D424CE9
:10426000002553455249414C250000000200000042
:104270000000000065120008D51200084000400050
:10428000D03E0020E03E00200200000000000000C0
:1042900003000000000000001D13000800000000E3
:1042A00010000000F03E00200000000001000000AF
:1042B000000000000C42002001010200311E000835
:1042C000411D0008DD1D0008C11D0008430000005D
:1042D000D442000809024300020100C03209040070
:1042E0000001020201000524001001052401000163
:1042F000042402020524060001070582030800FFCA
:1043000009040100020A0000000705010240000044
:104310000705810240000000120000002043000851
:10432000120110010200004009124157000201026F
:10433000030100000403090425424F4152442500B3
:10434000416F636F64612D52432D48373433447598
:10435000616C0030313233343536373839414243BD
:10436000444546000000002000000200020000005A
:1043700000000030000004000800000000000024DD
:1043800000000800040000000004000000FC000021
:10439000020000000000043000800000080000005F
:1043A00000000038000001000100000000000000D3
:1043B0007914000831170008DD170008400040009C
:1043C00044430020444300200100000054430020E7
:1043D0008000000040010000080000000001000013
:1043E00000100000080000006D61696E0069646CD7
:1043F000650000000000802A00000000AAAAAAAA06
:1044000000000024FFFF00000000000000A00A00E0
:104410000000000100000000AAAAAAAA00000001F2
:10442000FFFF00000000000000000000000000404E
:1044300000000000AAAAAAAA00000040FFFF000096
:10444000000000000000000040000000000000002C
:10445000AAAAAAAA40000000FFFF00000000000076
:10446000000000004000400000000000AAAAAAAA24
:1044700000004000F7FF0000000000000000000006
:104480000000000000000000AAAAAAAA0000000084
:10449000FFFF00000000000000000000000000001E
:1044A00000000000AAAAAAAA00000000FFFF000066
:1044B00000000000000000000000000000000000FC
:1044C000AAAAAAAA00000000FFFF00000000000046
:1044D000000000000000000000000000AAAAAAAA34
:1044E00000000000FFFF00000000000000000000CE
:1044F0000000000000000000AAAAAAAA0000000014
:10450000FFFF0000000000000000000000000000AD
:1045100000000000AAAAAAAA00000000FFFF0000F5
:1045200000000000000000001000024008000240EF
:104530000008024000000B00280002400800024072
:104540000408024006010C0040000240080002403E
:104550000808024010020D00580002400800024006
:104560000C08024016030E00700002400C000240CE
:104570001008024000040F00880002400C000240B6
:104580001408024006051000A00002400C00024082
:104590001808024010061100B80002400C0002404A
:1045A0001C08024016072F001004024008040240B5
:1045B0002008024000083800280402400804024095
:1045C0002408024006093900400402400804024061
:1045D00028080240100A3A00580402400804024029
:1045E0002C080240160B3B00700402400C040240F1
:1045F00030080240000C3C00880402400C040240D9
:1046000034080240060D4400A00402400C0402409D
:1046100038080240100E4500B80402400C04024065
:104620003C080240160F46005A140000000000002B
:1046300000001A0000000000FF0000000000000061
:10464000CC41000883040000D7410008500400005A
:10465000E5410008009600000000080096000000F8
:1046600000080000040000003443000800000000BF
:10467000000000000000000000000000000000003A
:1046800000000000FFFFFFFFFFFFFFFFFFFFFFFF36
:10469000FFFFFFFFFFFFFFFFFFFFFFFFFFFFFFFF2A
:1046A000FFFFFFFFFFFFFFFFFFFFFFFFFFFFFFFF1A
:1046B000FFFFFFFFFFFFFFFFFFFFFFFFFFFFFFFF0A
:1046C000FFFFFFFFFFFFFFFFFFFFFFFFFFFFFFFFFA
:020000040801F1
:020000040802F0
:10000000000600309D0D020875CD0E085103020850
:10001000FDCC0E08F5CC0E08F9CC0E089F0D020899
:100020009F0D02089F0D02089F0D02083DBD130899
:100030009F0D02089F0D02089F0D02089F0D0208E8
:100040009F0D02089F0D02089F0D02089F0D0208D8
:100050009F0D02089F0D020839D3130865D31308BA
:1000600091D31308BDD31308E9D3130811741308EF
:10007000397413086574130891741308BD74130858
:10008000E574130811751308357013089F0D0208E5
:100090009F0D02089F0D02089F0D020815D413083A
:1000A0009F0D020879D513089F0D02088DD51308FE
:1000B00091D51308A5D51308B9D51308A17C130849
:1000C000D17C1308017D1308317D13085580130876
:1000D0006D801308EDD4130801D5130815D5130846
:1000E00079D413089F0D02089F0D0208E1D513086B
:1000F0009F0D02089F0D02089F0D02083D75130811
:100100009F0D02089F0D0208CDD5130885801308A6
:1001100029D513089F0D02089F0D02089F0D0208A4
:100120006975130891751308BD751308E9751308EF
:10013000157613089F0D02089F0D02089F0D0208F7
:100140009F0D02089F0D02089F0D02089F0D0208D7
:100150003D76130869761308957613083DD5130884
:100160009F0D02089F0D02089F0D02089F0D0208B7
:100170009F0D020829C913089F0D02089F0D020850
:100180009F0D02089F0D020851D5130865D513086D
:100190009D8013089F0D02089F0D02089F0D020805
:1001A0009F0D02089F0D02089F0D02089F0D020877
:1001B0009F0D02089F0D02089F0D02089F0D020867
:1001C0009F0D02089F0D02089F0D02089F0D020857
:1001D0009F0D020815C913089F0D02089F0D020804
:1001E0009F0D02089F0D02089F0D02089F0D020837
:1001F0009F0D02089F0D02089F0D02089F0D020827
:100200009F0D02089F0D02089F0D02089F0D020816
:100210009F0D02089F0D02089F0D02089F0D020806
:100220009F0D02089F0D02089F0D02089F0D0208F6
:100230009F0D02089F0D02089F0D020855701308BC
:100240009F0D0208DD71130805721308317213083F
:100250005D72130889721308B5721308E1721308EE
:100260000D7313089F0D02089F0D02089F0D0208D1
:100270009F0D02089F0D02089F0D02089F0D0208A6
:100280009F0D02089F0D02089F0D02089F0D020896
:100290009F0D02089F0D02089F0D02089F0D020886
:1002A0009F0D02089F0D02089F0D02089F0D020876
:1002B0009F0D02089F0D02089F0D02089F0D020866
:1002C0009F0D02089F0D02089F0D02089F0D020856
:1002D0009F0D02089F0D02089F0D02089F0D020846
:1002E000BD440208CD7D020851C00208DD28030884
:1002F0000D920308E93B04088D3C0608DD990808C7
:1003000015A00808D918090821760908E97D090807
:100310002981090879F90908E5200A08F57C0B0804
:100320006D190C08ADC60E086DDF0E089DFA110898
:10033000699E120821C61208D9DD1208C90F1308D8
:100340008D151308000000000000000000000000F0
:10035000EFF30383EFF30982EFF30881DFF814D0A2
:100360002DE9FE4F684600F0F1FFBDE8FE4F8D46D7
:10037000704700008C320030F1EE101AA0EC200A19
:1003800001607047A0EC108A704700BF81F0004107
:1003900002E000BF83F0004330B54FEA41044FEA6A
:1003A000430594EA050F08BF90EA020F1FBF54EA05
:1003B000000C55EA020C7FEA645C7FEA655C00F0A1
:1003C000E2804FEA5454D4EB5555B8BF6D420CDD72
:1003D0002C4480EA020281EA030382EA000083EAF5
:1003E000010180EA020281EA0303362D88BF30BD95
:1003F00011F0004F4FEA01314FF4801C4CEA1131EB
:1004000002D0404261EB410113F0004F4FEA033349
:100410004CEA133302D0524263EB430394EA050FD4
:1004200000F0A780A4F10104D5F1200E0DDB02FA43
:100430000EFC22FA05F2801841F1000103FA0EF2D7
:10044000801843FA05F359410EE0A5F120050EF19D
:10045000200E012A03FA0EFC28BF4CF0020C43FACE
:1004600005F3C01851EBE37101F0004507D54FF0DB
:10047000000EDCF1000C7EEB00006EEB0101B1F52B
:10048000801F1BD3B1F5001F0CD349085FEA300071
:100490004FEA3C0C04F101044FEA445212F5800F7C
:1004A00080F09A80BCF1004F08BF5FEA500C50F119
:1004B000000041EB045141EA050130BD5FEA4C0CFC
:1004C000404141EB0101013C28BFB1F5801FE9D259
:1004D00091F0000F04BF01460020B1FA81F308BF7C
:1004E0002033A3F10B03B3F120020CDA0C3208DD48
:1004F00002F1140CC2F10C0201FA0CF021FA02F123
:100500000CE002F11402D8BFC2F1200C01FA02F192
:1005100020FA0CFCDCBF41EA0C019040E41AA2BFB7
:1005200001EB0451294330BD6FEA04041F3C1CDA7F
:100530000C340EDC04F11404C4F1200220FA04F09F
:1005400001FA02F340EA030021FA04F345EA030149
:1005500030BDC4F10C04C4F1200220FA02F001FA0B
:1005600004F340EA0300294630BD21FA04F029468D
:1005700030BD94F0000F83F4801306BF81F4801126
:100580000134013D4EE77FEA645C18BF7FEA655C99
:1005900029D094EA050F08BF90EA020F05D054EA6B
:1005A000000C04BF1946104630BD91EA030F1EBF70
:1005B0000021002030BD5FEA545C05D14000494174
:1005C00028BF41F0004130BD14F580043CBF01F567
:1005D000801130BD01F0004545F0FE4141F470014D
:1005E0004FF0000030BD7FEA645C1ABF1946104628
:1005F0007FEA655C1CBF0B46024650EA013406BF29
:1006000052EA033591EA030F41F4002130BD00BFE7
:1006100090F0000F04BF0021704730B54FF48064A4
:1006200004F132044FF000054FF0000150E700BF25
:1006300090F0000F04BF0021704730B54FF4806484
:1006400004F1320410F0004548BF40424FF0000171
:100650003EE700BF42004FEAE2014FEA31014FEAB4
:1006600002701FBF12F07F4393F07F4F81F0605103
:10067000704732F07F4208BF704793F07F4F04BF4E
:1006800041F40021704730B54FF4607401F000452B
:1006900021F000411CE700BF50EA010208BF70478B
:1006A00030B54FF000050AE050EA010208BF70477C
:1006B00030B511F0004502D5404261EB41014FF4E5
:1006C000806404F132045FEA915C3FF4D8AE4FF0ED
:1006D00003025FEADC0C18BF03325FEADC0C18BFD0
:1006E000033202EBDC02C2F1200300FA03FC20FA21
:1006F00002F001FA03FE40EA0E0021FA02F114446E
:10070000BDE600BF80F0004002E000BF81F0004184
:1007100042001FBF5FEA410392EA030F7FEA226CA7
:100720007FEA236C6AD04FEA1262D2EB1363C1BF37
:10073000D218414048404140B8BF5B42192B88BFA6
:10074000704710F0004F40F4000020F07F4018BFC9
:10075000404211F0004F41F4000121F07F4118BFE9
:10076000494292EA030F3FD0A2F1010241FA03FC91
:1007700010EB0C00C3F1200301FA03F100F0004379
:1007800002D5494260EB4000B0F5000F13D3B0F141
:10079000807F06D340084FEA310102F10102FE2AB0
:1007A00051D2B1F1004F40EBC25008BF20F0010020
:1007B00040EA03007047490040EB0000013A28BFBF
:1007C000B0F5000FEDD2B0FA80FCACF1080CB2EB42
:1007D0000C0200FA0CF0AABF00EBC25052421843C0
:1007E000BCBFD0401843704792F0000F81F4000165
:1007F00006BF80F400000132013BB5E74FEA410338
:100800007FEA226C18BF7FEA236C21D092EA030FA3
:1008100004D092F0000F08BF0846704790EA010F1D
:100820001CBF0020704712F07F4F04D1400028BF4A
:1008300040F00040704712F100723CBF00F500002C
:10084000704700F0004343F0FE4040F40000704762
:100850007FEA226216BF08467FEA2363014642020E
:1008600006BF5FEA412390EA010F40F48000704721
:100870004FF0000304E000BF10F0004348BF4042C7
:100880005FEA000C08BF704743F0964301464FF003
:1008900000001CE050EA010208BF70474FF000035F
:1008A0000AE000BF50EA010208BF704711F00043A0
:1008B00002D5404261EB41015FEA010C02BF844670
:1008C0000146002043F0B64308BFA3F18053A3F5CF
:1008D0000003BCFA8CF2083AA3EBC25310DB01FA16
:1008E00002FC634400FA02FCC2F12002BCF1004F9A
:1008F00020FA02F243EB020008BF20F0010070472B
:1009000002F1200201FA02FCC2F1200250EA4C007E
:1009100021FA02F243EB020008BF20EADC707047C4
:100920007BB972B90029BEBF00204FF0004106E03C
:1009300008BF00281CBF6FF000414FF0FF3000F0EF
:100940002BBAADF1080C6DE904CE002909DB002BB0
:100950001ADB00F0B9F8DDF804E0DDE9022304B0A9
:100960007047404261EB4101002B1BDB00F0ACF80B
:10097000DDF804E0DDE9022304B0404261EB41010F
:10098000524263EB43037047524263EB430300F070
:100990009BF8DDF804E0DDE9022304B0404261EB9E
:1009A00041017047524263EB430300F08DF8DDF8DC
:1009B00004E0DDE9022304B0524263EB43037047D5
:1009C00053B94AB9002908BF00281CBF4FF0FF31B6
:1009D0004FF0FF3000F0E0B9ADF1080C6DE904CE46
:1009E00000F072F8DDF804E0DDE9022304B070479E
:1009F000430803F05533C01A830803F0333300F083
:100A00003330184400EB101000F00F3000EB0020E2
:100A100000EB0040000E704708B502460B4643EC61
:100A2000172BB5EEC07BF1EE10FA03D4BDE80840F9
:100A300000F02AB8B1EE477B51EC170B00F024F818
:100A4000404261EB410108BD9FED0B6B07EE900A40
:100A50009FED0B5BB7EEE77A27EE066BBCEEC66B3D
:100A6000B8EE464BA4EE457BFCEEC77B16EE101AA3
:100A700017EE900A704700BF000000000000F03D34
:100A8000000000000000F0419FED0B6B41EC170BE4
:100A90009FED0B5B27EE066BBCEEC66BB8EE464BCC
:100AA000A4EE457BFCEEC77B16EE101A17EE900AFB
:100AB000704700BFAFF30080000000000000F03D71
:100AC000000000000000F0412DE9F047089D0446B9
:100AD0008E46002B4DD18A42944669D9B2FA82F2F1
:100AE00052B101FA02F3C2F1200120FA01F10CFA2D
:100AF00002FC41EA030E94404FEA1C48210CBEFB65
:100B0000F8F61FFA8CF708FB16E341EA034306FBED
:100B100007F199420AD91CEB030306F1FF3080F07C
:100B20001F81994240F21C81023E63445B1AA4B2C9
:100B3000B3FBF8F008FB103344EA034400FB07F76B
:100B4000A7420AD91CEB040400F1FF3380F00A81AC
:100B5000A74240F207816444023840EA0640E41BA1
:100B600000261DB1D4400023C5E900433146BDE84D
:100B7000F0878B4209D9002D00F0EF800026C5E9EF
:100B8000000130463146BDE8F087B3FA83F6002E07
:100B90004AD18B4202D3824200F2F980841A61EB7F
:100BA000030301209E46002DE0D0C5E9004EDDE79D
:100BB00002B9FFDEB2FA82F2002A40F09280A1EB85
:100BC0000C014FEA1C471FFA8CFE0126200CB1FBDA
:100BD000F7F307FB131140EA01410EFB03F08842D3
:100BE00008D91CEB010103F1FF3802D2884200F260
:100BF000CB804346091AA4B2B1FBF7F007FB1011F2
:100C000044EA01440EFB00FEA64508D91CEB04048F
:100C100000F1FF3102D2A64500F2BB800846A4EBEA
:100C20000E0440EA03409CE7C6F12007B34022FAD5
:100C300007FC4CEA030C20FA07F401FA06F31C4304
:100C4000F9404FEA1C4900FA06F3B1FBF9F8200C11
:100C50001FFA8CFE09FB181140EA014108FB0EF057
:100C6000884202FA06F20BD91CEB010108F1FF3AA7
:100C700080F08880884240F28580A8F102086144B3
:100C8000091AA4B2B1FBF9F009FB101144EA0141C1
:100C900000FB0EFE8E4508D91CEB010100F1FF346C
:100CA0006CD28E456AD90238614440EA0840A0FB04
:100CB0000294A1EB0E01A142C846A64656D353D0DA
:100CC0005DB1B3EB080261EB0E0101FA07F722FAFE
:100CD00006F3F1401F43C5E9007100263146BDE827
:100CE000F087C2F12003D8400CFA02FC21FA03F38A
:100CF000914001434FEA1C471FFA8CFEB3FBF7F00B
:100D000007FB10360B0C43EA064300FB0EF69E422F
:100D100004FA02F408D91CEB030300F1FF382FD2C8
:100D20009E422DD9023863449B1B89B2B3FBF7F670
:100D300007FB163341EA034106FB0EF38B4208D949
:100D40001CEB010106F1FF3816D28B4214D9023E8A
:100D50006144C91A46EA004638E72E46284605E7A8
:100D60000646E3E61846F8E64B45A9D2B9EB020879
:100D700064EB0C0E0138A3E74646EAE7204694E709
:100D80004046D1E7D0467BE7023B614432E730463C
:100D900009E76444023842E7704700BF02E000F010
:100DA00000F8FEE772B6374880F30888364880F3CB
:100DB000098836483649086040F20000CCF200004D
:100DC0004EF63471CEF200010860BFF34F8FBFF3CF
:100DD0006F8F40F20000C0F2F0004EF68851CEF264
:100DE00000010860BFF34F8FBFF36F8F4FF000001B
:100DF000E1EE100A4EF63C71CEF2000108600620CA
:100E000080F31488BFF36F8F1AF1FAFF1CF18AF890
:100E10004FF055301F491B4A91423CBF41F8040B2B
:100E2000FAE71D49184A91423CBF41F8040BFAE722
:100E30001A491B4A1B4B9A423EBF51F8040B42F819
:100E4000040BF8E700201849184A91423CBF41F8CA
:100E5000040BFAE71BF112F81CF1E8F8144C154DDD
:100E6000AC4203DA54F8041B8847F9E703F07AFA36
:100E7000114C124DAC4203DA54F8041B8847F9E7D1
:100E80001AF1FABF0006003000220030000002080C
:100E900008ED00E0000000300006003018031808DC
:100EA0000022003094300030983000307C25023031
:100EB000E002020844030208440302084403020853
:100EC0002DE9F04F2DED108AC1F80CD0D0F80CD0E0
:100ED000BDEC108ABDE8F08F002383F3118828460B
:100EE000A047002019F1D0FDFEE719F13FFC00DF1B
:100EF000FEE7000070B54FF0FF0C4CF4E06C1CEA0C
:100F000011541DBF1CEA135594EA0C0F95EA0C0FFF
:100F100000F0DEF82C4481EA030621EA4C5123EA72
:100F20004C5350EA013518BF52EA033541F48011A1
:100F300043F4801338D0A0FB02CE4FF00005E1FB54
:100F400002E506F00042E0FB03E54FF00006E1FB9E
:100F500003569CF0000F18BF4EF0010EA4F1FF04E1
:100F6000B6F5007F64F5407404D25FEA4E0E6D4121
:100F700046EB060642EAC62141EA55514FEAC52032
:100F800040EA5E504FEACE2EB4F1FD0C88BFBCF5AE
:100F9000E06F1ED8BEF1004F08BF5FEA500E50F15F
:100FA000000041EB045170BD06F0004646EA010125
:100FB00040EA020081EA0301B4EB5C04C2BFD4EB57
:100FC0000C0541EA045170BD41F480114FF0000E50
:100FD000013C00F3AB8014F1360FDEBF002001F0BE
:100FE000004170BDC4F10004203C35DA0C341BDC38
:100FF00004F11404C4F1200500FA05F320FA04F00A
:1010000001FA05F240EA020001F0004221F000413D
:1010100010EBD37021FA04F642EB06015EEA430EB0
:1010200008BF20EAD37070BDC4F10C04C4F12005E0
:1010300000FA04F320FA05F001FA04F240EA020093
:1010400001F0004110EBD37041F100015EEA430E64
:1010500008BF20EAD37070BDC4F1200500FA05F284
:101060004EEA020E20FA04F301FA05F243EA020303
:1010700021FA04F001F0004121FA04F220EA020012
:1010800000EBD3705EEA430E08BF20EAD37070BD58
:1010900094F0000F0FD101F00046400041EB010138
:1010A00011F4801F08BF013CF7D041EA060195F01A
:1010B000000F18BF704703F00046520043EB0303D4
:1010C00013F4801F08BF013DF7D043EA06037047C1
:1010D00094EA0C0F0CEA135518BF95EA0C0F0CD0CC
:1010E00050EA410618BF52EA4306D1D181EA030112
:1010F00001F000414FF0000070BD50EA410606BF0C
:101100001046194652EA430619D094EA0C0F02D150
:1011100050EA013613D195EA0C0F05D152EA033695
:101120001CBF104619460AD181EA030101F00041B3
:1011300041F0FE4141F470014FF0000070BD41F0FC
:10114000FE4141F4780170BD4FEA410212F50012F0
:1011500015D211D56FF47873B3EB625212D94FEAFE
:10116000C12343F0004343EA505311F0004F23FAE8
:1011700002F018BF404270474FF00000704750EA3D
:10118000013005D111F0004008BF6FF000407047FA
:101190004FF00000704700BF4FEA4102B2F1E04358
:1011A00024BFB3F5001CDCF1FE5C0DD901F0004C4E
:1011B0004FEAC0024CEA5070B2F1004F40EB83009E
:1011C00008BF20F00100704711F0804F21D113F1CA
:1011D0003872BCBF01F00040704741F480114FEA03
:1011E0005252C2F11802C2F1200C10FA0CF320FA8C
:1011F00002F018BF40F001004FEAC1234FEAD323A9
:1012000003FA0CFC40EA0C0023FA02F34FEA430312
:10121000CCE77FEA625307D150EA01331EBF4FF09B
:10122000FE4040F44000704701F0004040F0FE40B6
:1012300040F40000704700BF01F0FF01102A2BDBD3
:1012400010F0070F08D010F8013B013A8B422DD067
:1012500010F0070F42B3F6D1F0B441EA012141EAA0
:10126000014122F007047FF000070023F0E8025656
:10127000083C85EA010586EA010685FA47F5A3FAE6
:1012800087F586FA47F6A5FA87F68EB9EED1F0BC57
:1012900001F0FF0102F0070232B110F8013B013A00
:1012A00083EA010313B1F8D1002070470138704779
:1012B000002D06BF35460338073815F0010F07D15A
:1012C000013015F4807F02BF013015F4C03F0130BA
:1012D000F0BC0138704700BFEC46A0E8F05F4FF06B
:1012E00000007047B0E8F05FE546080008BF012045
:1012F000704700BF10F8012B11F8013B012A28BFED
:101300009A42F7D0D01A7047034613F8012B002AEF
:10131000FBD1181A0138704710B5044620461CB19D
:1013200054F80C3B013300D110BD0822012100F01C
:1013300071FB54F80C0C54F8082C14F8041C121A05
:10134000B2FBF1F200F066FBE8E70000C26AD0E908
:10135000003112F0040F2DE9F04118BF0B46A6B082
:101360000021594C042601270291CDE90003D00643
:101370004CBF03F1200203F168020392DA6903997A
:10138000D2099B6902F004021B880A4303F47F43DD
:1013900003924FF0E022A3F53E41D2F8882D02F4EB
:1013A000A002B2F5A00F04BF012202924B424B41B2
:1013B0000493464D03A82C6000F02AFA0422012170
:1013C000434800F027FB0422012102A800F022FB81
:1013D00010220121019800F01DFB0098202201211C
:1013E0000C3000F017FB019804220121103000F0AE
:1013F00011FB0422012103A800F00CFB01980C2230
:101400000121143000F006FB0C220121009800F0AD
:1014100001FB029BDA071FD5009BDB6ADB064ED47B
:1014200015A8FEF7AFFFDDF804C00DF1140E0CF1A6
:1014300020030CF160081868083353F8041C724646
:10144000434503C29646F6D1DCF8603025938422EA
:10145000012105A800F0DEFA00F0C0F8FFF75CFFFC
:101460004FF0E023D3F8003D03F47023B3F5402F91
:101470000ED0184B05A88DF81C60059314338DF819
:10148000287006934FF0FF33CDE90833FFF744FF90
:101490002B68A34206D0104B0422012105A8059316
:1014A00000F0B8FA00F02AFA002882D0049B1BB1A1
:1014B000019A93690233936126B0BDE8F08105A8D3
:1014C000FEF75AFFC3E700BFED55CEAC98300030B1
:1014D0003065140828ED00E0ACCE55ED37B50E4D63
:1014E0002A78202A15D10D4C0D4823680D4918443F
:1014F000019219F101FF23680021019A2033094864
:101500002970236020F166F803B0BDE830401AF17D
:10151000DFBB03B030BD00BF8C320030B4320030CE
:10152000C01118088E32003008B5262017F1B0FD22
:10153000144BD3F8902042F40032C3F89020D3F833
:10154000902022F40032C3F89020D3F89020D3F8F2
:10155000E82042F40032C3F8E820D3F8102142F426
:101560000032C3F810216D22D3F81031064BDA6037
:101570004FF0FF321A620D221A600122034B1A70DB
:1015800008BD00BF0044025800440040C43200308F
:10159000014B1868704700BFFCFF1B08014B024855
:1015A000C01A7047C011180800001C080048704796
:1015B000C011180807490022074B5B1A9A4201D351
:1015C0000120704751F8040B013001D10432F5E7D6
:1015D00000207047C011180800001C085E4B2DE960
:1015E000F74F1A6802255D4B02F56A58DFF89491AF
:1015F0001A7808F118085A4F5A4C9044DFF888A11D
:1016000018F1D6FFA9EB070B06460EB14E2D49D9AE
:10161000A9EB0702B2EB080700F192804E2D00F211
:101620008F80DFF868C16B1C4F4E0C21DBB2ACEB36
:1016300006006943B84273DD60184FF0010C665034
:1016400090463E4480F808C04660B2EB080213D4CE
:101650004F2B11D0454E19464548AB1C351ADBB20D
:1016600095424FF00C0505FB01F163DD651801267D
:10167000024460502E726A600C2201215343E2182A
:1016800011724FF0FF31E15051603A4B1B782BB192
:10169000394B1B682360394B1B686360314803B0CA
:1016A000BDE8F08F336AF06953450ABF344BF31A33
:1016B000A3EB0A0380B101931AF10CF8019B58B116
:1016C0002A460C2101354A430121EDB2A0180172CE
:1016D000F169A1500D3141600C200121984400FBBB
:1016E00005FCD84504EB0C0244F80C6006F13C0CF8
:1016F0001172C2F804C005EB010205F10205D2B275
:10170000EDB200FB02F204EB02000172316AA1505B
:101710001944416014D2304618F15AFF064674E766
:1017200067184FF0010E8044665087F808E0C7F84C
:1017300004C08AE7621801256050157256609BE765
:101740004F2D01D82B4697E7012384F8BC334FF087
:10175000FF33C4E9ED3398E7B43200308C32003007
:10176000C011180804220030983000300000043006
:101770008025023000220030B8320030B032003014
:101780000022003000001C08000600307C250230DA
:101790000C4B1B7810B50BB9FFF7C6FE00230A49A6
:1017A0000A48CA699206FCD54A6A1C5CD2B29442C5
:1017B00005D10133DBB20E2BF3D1002010BD002385
:1017C000EFE700BFC4320030004400403465140825
:1017D00038B5084B04461B780BB9FFF7A5FEE4B2F9
:1017E000054DAC62EB695B0600D538BD1AF170FAA5
:1017F000F8E700BFC43200300044004010B5441E7A
:1018000014F8010F00B910BDFFF7E2FFF8E7000080
:1018100070B502680446EFF30581D9205369C9B257
:10182000CBF06EFA294B1B78A3B1294B94E8030047
:1018300083E803002748FFF7E1FF6368B3B1264858
:10184000FFF7DCFF2548FFF7D9FFFFF7A1FF24488A
:10185000FFF7D4FF234D2B783BB124681CB1204601
:1018600019F138FF20B900232B7070BD1E48E7E73F
:1018700020461E4E19F142FF00F2145084421FD23E
:10188000204619F13BFF30602046194E19F14AFFFE
:1018900004F5E053834217D9204619F143FF306025
:1018A0000023144A1360144A1370FFF783FE0028C4
:1018B000D9D01AF10DFA0120BDE8704019F1A4BD8C
:1018C000A4F214533360DFE73360E9E78D32003070
:1018D000BC32003044651408496514085A65140880
:1018E0001C8915080022003054651408B8320030F5
:1018F000B0320030B43200308C320030284B1A78CD
:1019000070B542B12748FFF779FF274B5868003878
:1019100018BF012070BD254A107800283CD0244E05
:10192000244C33682448254D1A1D21782D1A0A4469
:10193000AA4205D3224A4FF0FF31D1612022227002
:101940002278D2B103F120018D4205D81F2A9FBF12
:101950001B4AD3612022227020221949184419F110
:10196000CBFC3268237800211548134420222170D3
:1019700033601FF12FFE1AF1ABF933689D4207D98E
:101980000F4920220F48CB6119F1B6FC1AF1A0F9DA
:10199000002019F139FDB8E701221A70BAE700BF3B
:1019A0008D320030A0651408BC32003000220030B7
:1019B000B43200308C320030C011180800001C080E
:1019C0008E320030E0FF1B082DE9F84307460E4633
:1019D0000024DFF83890DFF83880B44201D1BDE848
:1019E000F88324B1230702D14846FFF707FF3D5D86
:1019F00001342B0905F00F0518F80300FFF7E8FE86
:101A000018F80500FFF7E4FEE7E700BF1C8915089A
:101A1000B0651408474B1B782DE9F74F07460E4673
:101A200090465BB1022925D0042938D0012902D182
:101A30001146FFF7C9FF4048FFF7E0FE3F4B1B7818
:101A4000002B4ED03E4A00253E4BA2EB030938E066
:101A500037F81430ADF8043024B1620702D12846BB
:101A6000FFF7CCFE0134022101A8FFF7ADFFA0452E
:101A7000EED1E0E70024304DF9E757F82430019328
:101A800024B1A30702D12846FFF7B8FE0421013490
:101A90000DEB0100FFF798FFA045EED1CBE7002446
:101AA000254DF9E7FFF71AFD022E1DD0042E2CD08C
:101AB000012E06D12378795D5A1C2270224AD15416
:101AC0000135A8450DD0214B214C1B6822780433E9
:101AD00013444B45E6D31C4B4FF0FF32DA61202311
:101AE000237003B0BDE8F08F2378DFF85CA05A1CA8
:101AF00022703A780AF80320FFF7F0FC23785A1C8A
:101B0000227000220AF80320DAE74FF0000ADFF81B
:101B100038B022783B78511C23FA0AF30AF1080AFC
:101B200021700BF80230FFF7D9FCBAF1200FF0D189
:101B3000C6E700BF8D3200301C8915080022003036
:101B400000001C08C01118088E320030B43200307A
:101B50008C320030036800221B6818477FB5039160
:101B600040210546B5F05CFC039A18B901242046D3
:101B700004B070BD134E039296F9163E002BF5D0BB
:101B80007EF056F9437A039A53B97EF051F9847A7C
:101B9000039A2CB90C4B40212846B5F049FCE6E7E6
:101BA0000A4BB6F9181ED3F84C3BB3F906309942EC
:101BB000DCDD074B4021284600240093054BB5F09F
:101BC00037FCD4E7C8620030C4651408C88200300E
:101BD000E3651408D1651408F0B50D469DB02021C9
:101BE0000446B5F01DFC002800F0AD80574E96F974
:101BF000163EBBB106F50052B6F9183ED2F84C2B92
:101C0000B2F90A1003F10A02914203DD40F28D326B
:101C1000934207DC4E4B2A4620212046B5F008FCB3
:101C200000208EE096F9053E022B05D1494B2A464D
:101C300020212046B5F0FCFBB6F8D83D41F65832DD
:101C4000A3F57A739BB293420FD8434F06F64462D2
:101C5000D7F8143B92ED007AD3ED097AB4EEE77A27
:101C6000F1EE10FA03DD3D4BD5E73D4BD3E706F629
:101C70004862D3ED0B7A92ED007AB4EEE77AF1EE9A
:101C800010FAF0DCB6F9123E002B01DC354BC2E74E
:101C9000A7F5405393F8FC280D2A06D8012393405A
:101CA00013F4215F01D0304BB5E7304812F0AAF9A8
:101CB000012806D1D7F8200BBEF0F6FC48B1012868
:101CC00010D02B4B93F8DD1F11F010011FD0294BC2
:101CD000A1E7294B0093294B2A4620212046B5F045
:101CE000A7FB9DE7224B93F8603B73B11921244871
:101CF00068F030FC48B1D6F8F06D1921204868F042
:101D00005BFC8642DDDD1F4BE4E71F4BE2E7602210
:101D100004A803911FF15EFC642303AA1B49D7F8B2
:101D20001C0BBCF0EFFD18B903AB0093184BD3E7C5
:101D3000642303AA1749D7F8140BB9F071FA0028E5
:101D4000F2D01DB0F0BD0120FBE700BFC86200303B
:101D5000EC651408FF651408C8A200303766140843
:101D6000276614085166140866661408A8BA00307D
:101D7000C8820030E0661408AB6614088666140852
:101D800060480030CA661408BB661408F56614087B
:101D9000F96614080B67140870B59AB00E46002156
:101DA0006022054602A801911FF114FC642201A9DA
:101DB000094896F025FA044640B99DF9043043B924
:101DC000064B074A31462846B5F03CFD20461AB07E
:101DD00070BD01ABF5E700BF7C8B003010671408C5
:101DE0007D47170807B50448C0F06EFA00F00100FF
:101DF00003B05DF804FB00BFC0AD00302DE9F04337
:101E0000DFF844910446A5B00D46D9F8C40F036825
:101E10001B69984780461AF059FB0021074660224B
:101E20000CA80B911FF1D6FB64230BAA4146384640
:101E300019F068FD064648B90BAB394A29462046D9
:101E4000B5F000FD304625B0BDE8F083354894F08C
:101E5000C1F9B8F1000F03D194F91E30012B0AD15A
:101E6000314816F0D3FA80B9304A29462046002678
:101E7000B5F0E8FCE6E710F0060FE3D0A9F5A040C6
:101E800016F0C4FA08B92A4AEFE703A9384619F050
:101E90008DF928B19DF80D305B0601D5254AE4E7A0
:101EA000DFF8A8800023D8ED007AF5EEC07AF1EED5
:101EB00010FAC7DD0DF120090893099305AA0A93CA
:101EC00007AB04A93846019306ABCDF8009019F092
:101ED0005FFF48463EF030FAD8ED007AB4EEE70AEC
:101EE000F1EE10FA01DB144ABFE79DED057AF4EE3E
:101EF000C77AF1EE10FA01D8104AB6E79DED047AE0
:101F0000F4EEC77AF1EE10FA01D80D4AADE79DED77
:101F1000067AF4EEC77AF1EE10FA93D8094AA4E7EC
:101F20006FB81608F46C0030C83200302867140807
:101F30003F671408656714087367140888671408F6
:101F40009E671408B4671408C8820030FC70003023
:101F500008B5064B93F8DD3F9B0704D5044AB5F05E
:101F600071FC002008BD0120FCE700BFC8820030E2
:101F7000C867140870B50E469AB020210546B5F022
:101F80004FFA18B9012420461AB070BDC5F080FE82
:101F900004460028F6D00021602202A801911FF11A
:101FA00019FB2046642201A9C5F034FE044600282E
:101FB000E8D101AB024A31462846B5F043FCE2E7DE
:101FC0007D47170870B50C4C05460E46D4F8C40F73
:101FD00003685B69984710B10124204670BDA4F5E1
:101FE000A04016F025FA04460028F5D1034A3146F0
:101FF0002846B5F027FCF0E7C8820030D8671408FF
:102000002DE9704E4B4E9BB082468B46D6F8E83F8A
:1020100093F8D55065B9484B1B68986A03685B6BA9
:102020009847044640B9454A59465046B5F00AFC1F
:1020300028461BB0BDE8708E7DF0FAFE20217FF0AF
:102040005BF958B17DF0F4FE1F217FF055F980B3A4
:1020500000243B4A59465046B5F0F4FB96F8BA3F87
:1020600003F01403142B05D10024364A5946504678
:10207000B5F0E8FB59465046B6F078FC00216022E6
:10208000884202A8019108BF0C461FF1A3FAD6F8B6
:10209000E80F01AA642103681B689847054680B9C8
:1020A0002C4601AB284A59465046B5F0CBFB254695
:1020B000BEE77DF0BDFEA5217FF01EF90028C7D147
:1020C000CCE7002CF3D0DAF808303BB9DAF800306E
:1020D000594650469B6B98470446E8E75946504698
:1020E000FFF77AFD814659465046FFF755FE09EA4B
:1020F00000005946C4B25046FFF72AFF5946044033
:102100005046FFF737FF594604405046FFF726FD7B
:10211000594604405046FFF755FF59460440504683
:10212000B5F0C6FC594604405046B6F037FC0440B2
:10213000BDE700BFC882003038BF0030EC6714082C
:10214000036814081D6814083568140808B5FFF7FB
:1021500057FF054A92F8B81F60F3041182F8B81FC0
:10216000024A907108BD00BFC88200302DC1003006
:10217000F7B505460F46B5F08FF9044678B1022150
:102180002846B5F04DF9064648B11548C0F09CF810
:10219000C205C0F30723C0F3002403D5344620460C
:1021A00003B0F0BD9B07F9D50D48C0F09BF80D4B6F
:1021B00003F6C423D3ED007AF8EEE77A30EE670A2F
:1021C000DFED097AB0EEC00AB4EEE70AF1EE10FADC
:1021D000E4DD064B3A4602212846B5F029F9DEE750
:1021E000C0AD0030C8A200300000C84240681408EA
:1021F000F8B504460F46B5F011FD102105462046FE
:10220000B5F00EF958B12046FFF7ECFD064630B99F
:102210003546044B3A4610212046B5F009F92846C8
:10222000F8BD00BF5468140870B505460E46B5F0F9
:1022300079F8044678B180212846B5F0F1F850B11C
:10224000074B93F8A93543B10024064B3246802151
:102250002846B5F0EDF8204670BD0446FBE700BF08
:10226000C89200306868140838B50E4C0546D4F89A
:10227000200BBEF019FA012811D0D4F8200BBEF0C3
:1022800013FA022804D02846BDE83840B5F04CB80F
:1022900004F5BF5011F0B6FE0128F4D138BD00207E
:1022A000FCE700BFC8A20030F0B5114C85B006466F
:1022B0000F46D4F8443B6A460093D4F8483B019358
:1022C000D4F84C3B0293D4F8503B0393B6F0DCFABD
:1022D000054639463046B5F005F994F8B83F284030
:1022E00060F3C303C3F3C00084F8B83F05B0F0BD8A
:1022F000C88200302DE9F843DFF8AC900646264846
:102300000F4693F067FF0446D9F8C40FDFF89C80AE
:1023100003681B699847054630B914F0060F03D1CE
:10232000D9F8F83F022B09D139463046B5F0ACF95F
:10233000054618B9002488F807400AE039463046B7
:10234000FFF75CFD04460028F4D02DB9012388F87E
:1023500007302046BDE8F88308213046B5F060F824
:102360000028F3D00D4829F073FE0028EED00C4B66
:10237000B02193F8142401FB023203F54053B2F864
:102380001E22B3F9063E9A42E0DD064B3A4608218A
:102390003046B5F04DF8CDE7F46C0030E83300304E
:1023A000C83200307C681408C88200302DC100306B
:1023B00070B588B005460E46B5F06CFA044688B391
:1023C00020212846B5F02CF860B31B4B93F85C2C09
:1023D00042B393F8383C9B0724D507AA06A91748AF
:1023E0008FF036FCF0B19DED077ADFED157AB4EE93
:1023F000E77AF1EE10FA15D8B7EEC77A002420215B
:1024000028468DED027BDDED067AFDEEE77A08A326
:10241000D3E90023CDED007ACDE90423094B324600
:10242000B5F006F8204608B070BD00BFAFF30080DD
:10243000000000403333E33FC8A200301C7200307C
:102440009A99193F8C6814082DE9F3410F46044608
:102450001AF03CF8804618F05BFE054640B9564A33
:1024600001212046B5F0EEF9284602B0BDE8F08122
:10247000524E3946D6F8C40F03689B699847054603
:1024800058B9D6F8C40F03681B6C98474C4A0346EA
:1024900001212046B5F0D6F9E6E7A368002BE3D08A
:1024A00010212046B4F0BCFF20B3D8ED937A98ED0C
:1024B000920A20EE270A1CF147F9DFED427AA6F5D1
:1024C000005320EE270ADFED407AB3F9D83D20EE25
:1024D000270A07EE903AF8EEE77AB4EEE70AF1EE53
:1024E00010FA07DD394B012210212046B4F0A0FF7D
:1024F0000025B9E720212046B4F092FF38B196F8C4
:10250000DD3FDB0603D5324B01222021EDE74021E0
:102510002046B4F085FF28B3012F1CD0232F1AD0FA
:10252000042F18D0D6F84C3B2A48B3F9083000EEF7
:10253000103AB8EEC00A00F0D3FBB5EEC00AF1EED7
:1025400010FA1DDD244B0122402120460093234B2D
:10255000B4F06EFFCCE7D6F8C40F0368DB6B984786
:102560000028DFD01E4B1B68D86A0368DB699847D8
:102570000128014619D11B4A2046B5F063F9B7E797
:10258000D6F8C40F03685B69984730B1D6F84C3B66
:10259000B3F90830002BE5DDD4E7D6F8C40F0368A3
:1025A0001B6898470B28DDD1F0E73946204602B07A
:1025B000BDE8F041B5F020BEB8681408C88200300C
:1025C000C9681408E02E65420000C842DD6814089E
:1025D000E0661408C8320030E3651408E5681408A2
:1025E00038BF0030F168140870B505460E46FFF795
:1025F00005FC084B04463146D8712846FFF7E2FC3B
:1026000000283146284608BF0024B6F0EBF82040E9
:1026100070BD00BF2DC100302DE9F041534F3B7814
:10262000002B40F0A080524C0126D4F8E85F3E70A9
:1026300095F8D5501DB13B702846BDE8F081B6F045
:1026400079FA054630B94B4A3870137843F00103E4
:102650001370F1E771F01AFA314670F041FBA4F5FE
:10266000A04007F0F3FE444B1E710B26013E60F0C4
:10267000B1FF60F0CDFE16F0FF06F7D13F4801F044
:102680006BFA19F023FF3E4AD0F80012116190F85E
:102690007C32D90754D419F0CBF971F0F7F93C2109
:1026A00071F030F904F57D6300221A60002133488F
:1026B00001F0D4FA314815F0A9FE01463148C4F0C2
:1026C000E1FF314B314E01211B68D86A03681B685A
:1026D000984796F8983CD4F8E80F6FF3410386F8D2
:1026E000983C03689B6A98470121D4F8E80FC1F031
:1026F00045F971F0CBF98046D4F8C40F03681B6824
:102700009847A6F580430146404693F8EC2B70F0BD
:10271000BFFCA6F5E04007F08BFE6EF031F86DF0DF
:1027200073FB00233B70CAF057FBB4F8BA3FC6F8FE
:102730002C0B23F4087343F02003A4F8BA3F7BE783
:102740009B07B3D43146A2F5C04005F019FF1048ED
:10275000BFF0C8FDDFED0F7A04F57D6320EE270A98
:1027600083ED000AA2E7002566E700BFC53200300E
:10277000C88200304CC100302DC10030C83200305A
:10278000C89200300C8A003038BF0030C8A2003038
:10279000C0AD00300AD7233C2DE9F043374D87B058
:1027A000D5F8E83F93F8D530002B64D062B1012909
:1027B00001D0232908D195F9B83F002B04DB002470
:1027C000204607B0BDE8F083B6F062FA0446002860
:1027D000F5D019F07BFE074622F066F880463846B1
:1027E00018F0BCFAD8B198F92830022B17D100267E
:1027F0004FF00009F1B203AA3846CDF80C900191D0
:10280000CDF81090CDF8149018F006FF019918B18A
:1028100003AA404621F0D4FC0136032EEAD101215F
:10282000174808F07FF80121154807F0B1FF002193
:10283000D5F8E80FC1F0A2F8124840F02DF971F078
:1028400025F9002170F04CFA0F4B00211B68D86A63
:1028500003681B68984795F8BA3FD5F8C41F6FF313
:1028600045130A4885F8BA3F0B1A3C305942594182
:10287000C8F0B2FCA4E70124A2E700BFC882003080
:10288000C832003024B3003038BF00302CB60030DE
:1028900010B5064CD4F8C40F03685B6A984718B1AA
:1028A000D4F8E83F93F8D50010BD00BFC8820030CF
:1028B00030B52DED028B89B0B0EE408A0C46FFF7A3
:1028C000E7FF0546002836D0B4EE488A22686368E0
:1028D00002A89FED1B0AF1EE10FA029203937DBF4E
:1028E000DFED188ADFED167A68EE288ADFED168AAA
:1028F00078BF68EEA78AD4ED027AF1EE677ACDED63
:10290000047A3DF0FBF8B4EE488A002201238DEDF5
:10291000050ACDED060A05A9F1EE10FA9FED0A0AA7
:10292000F0EE680A09488DED071ACDE9002368BF6B
:1029300013460FF09BF8284609B0BDEC028B30BD62
:102940000000C842E02E65420000000048B9003097
:1029500007B50191FFF79CFF30B10199044803B01E
:102960005DF804EB00F08EBB03B05DF804FB00BF24
:10297000C8320030014893F0B9BD00BFF46C00309C
:1029800000F5A04008B590F8B83FC3F340128A4262
:102990000BD061F3451380F8B83F31B171F076F890
:1029A0000F21BDE8084070F0ADBF08BD70B500F55F
:1029B000A04605460C46D6F8F83F8B4212D00129B6
:1029C00011D0022916D059B971F060F81B2170F0AE
:1029D00099FF0D4A05F5BA400621503073F034FCDA
:1029E000C6F8F84F70BD71F051F81A2170F08AFFE7
:1029F000064AEFE7012101F031F971F047F81D2196
:102A000070F080FF024AE5E76069140875691408F0
:102A10007069140800F5A04210B592F8DD3F0C462D
:102A200003F00101A14209D064F3000382F8DD3F05
:102A3000DB0704D407F0DCF8024B9C7210BD07F0F2
:102A4000C1FAF9E72DC1003000F5A04090F8DD3F54
:102A500061F3410380F8DD3F014B1973704700BFFC
:102A60002DC1003010B504467DF0E2F920217EF042
:102A700043FC04F5A043003893F8BA2F18BF012097
:102A800060F3820283F8BA2F10BD000010B504462F
:102A90006DF076FE436F04F5A04204F5E044D2F8F1
:102AA000E82FD360D4F8142B9366D4F81C2BC2F80B
:102AB0000833D4F8140B03685B6D9847D4F8140BF3
:102AC0000368BDE810409B6D18470000F8B500F59D
:102AD000A04504462DED028BD5F8E83F93F8D5309C
:102AE000002B7BD095F9B83F002B77DB00F5E04653
:102AF00096F8803F002B71D1D5F8C40F03685B694D
:102B0000984700286AD1374BD3F8C40F03681B6875
:102B100098470B2862D0D6F81C3B9FED337AD3ED53
:102B2000E47AF0EEE77AF4EEC77AF1EE10FA55D5D2
:102B3000D5F8E80F443072F0EFFC0346B7EE001A08
:102B40009F20DFED2A0A93ED000A37F081FBB5EEF6
:102B5000C00AF1EE10FA41DD04F5F5407830BFF01F
:102B6000CDFBB0EEC00ADFED227AB4EEE70AF1EE5B
:102B700010FA33D504F50057D6F8140BD7EDE47AE4
:102B80000368B8EEE78AD3F898309847DFED197AF2
:102B900038EE400AB0EEC00AB4EEE70AF1EE10FAE1
:102BA0001CD5D7F8943340F2E63203F2F313934284
:102BB00014D8D5F8E80F9FED100AC2F035FBD5F810
:102BC000E83F04F5D0509FED0C0AD3ED0C0A143009
:102BD000BDEC028BBDE8F840A4F0AEBFBDEC028BAB
:102BE000F8BD00BFC88200300000003400000000C3
:102BF000000070420000FA430AD7233C00F5A040D1
:102C000008B5D0F8E80F03681B699847F6EE007A1C
:102C100020EE270AB5EEC00AF1EE10FA48BF9FED8C
:102C2000010A08BD0000000038B500F5E045044683
:102C3000B7EE001A712004F5A044DFED110A2DED66
:102C4000028BD5F8143B93ED370A37F001FBD4F82B
:102C5000E80FB0EE408AD5F81C5B036805F50575F2
:102C60001B69984738EE400ADFED067A2846BDEC2E
:102C7000028B20EE270ABDE83840A1F07BBC00BFE4
:102C80000000000000007A4400F50050D2ED007A08
:102C900091ED006AD0EDFA5AD0EDFD6A26EEE77AA2
:102CA00067EEA57AA6EE257AE6EE267A81ED007A21
:102CB000C2ED007A7047000000F5A043B3F9103868
:102CC00043B900F54050B0F9120E0028B8BF404299
:102CD00080B2704783EAE370A0EBE370F8E700008E
:102CE00000F5A04370B52DED028B93F8DD1F82B087
:102CF000044611F0010605D09FED2E0A02B0BDEC8E
:102D0000028B70BD8DED010A7DF092F8037F002BE0
:102D1000F2D0DFED298A04F54055DFED260A4E207A
:102D2000B0EE681A9DED010A37F092FA4FF4C872BE
:102D30003146B5F91A0EB0EE408A37F0F1FAA5F82F
:102D40001A0E204615F0ACF8B5F91A3E07EE900AB7
:102D5000B8EEE77A07EE903AF8EEE77A77EE676A30
:102D6000B4EEE68AF1EE10FA0DD5204638EE668A0A
:102D7000FFF7A2FF07EE900AB8EEE70A20EE088AF6
:102D800088EE260ABAE777EE877AB4EEE78AF1EEA4
:102D900010FAB1DDB5F9123E38EE678A78EEE77ABF
:102DA00000EE103AB8EEC00A20EE088A88EE270A34
:102DB000A4E700BF0000000000007A447047000054
:102DC00070470000002070470020704700207047C7
:102DD0000020704700207047002070470020704797
:102DE00000207047002070477047000000F57850C1
:102DF000283070470048704764A1140800F5A040CF
:102E0000D0F8C40F03681B68184700000348086027
:102E10003821117008221A60704700BFAC6F140887
:102E200000F5E0409FED0A7AD0F8283B0120D3ED71
:102E30000E7AF4EEC77A9FED077AF1EE10FAB8BF7A
:102E4000D3ED047A67EE877AC1ED007A704700BF50
:102E5000000000340AD7233C00F5A040DFED047ADF
:102E6000D0F8C40F20EE270A03685B6E184700BF36
:102E70000000C84200F5004393F82D33002B14BF27
:102E80001B2003200B1A58425841704700F5A04000
:102E900090F8DD0FC0F380007047000000F5A040FF
:102EA000D0F8C40F03685B6D1847000000F5A04020
:102EB000D0F8C40F0368DB6C1847000000F5A04091
:102EC000D0F8C40F03689B6C1847000000F5A043BE
:102ED00000F50040D3F8C43F20301B1A5842584137
:102EE0007047000000F5A04010B5D0F8C40F0C46A4
:102EF0000368DB6D984707EE900A9FED057A012085
:102F0000F8EE677A67EE877AC4ED007A10BD00BFED
:102F10000AD7233C00F5A04010B5D0F8C40F0C46EA
:102F200003689B6D984707EE900A9FED057A012094
:102F3000F8EEE77A67EE877AC4ED007A10BD00BF3D
:102F40000AD7233C00F5A04010B5D0F8C40F0C46BA
:102F500003681B6E9847DFED047A012020EE270AF4
:102F600084ED000A10BD00BF0AD7233C86F0B4BD33
:102F7000C4F06CBE04F058BF8BF0B0B97FF0A4BBB6
:102F80006DF048BB34F08ABB70F028B81DF04ABD24
:102F90007FF078BF7CF076BB7AF022B914F0EEBBFC
:102FA00015F098B807F0F6BE16F03CB906F076BEFC
:102FB00006F0C4BB06F0EABA14F078BD88F06ABB2C
:102FC00092F014BF11F0CEBEFFF780BD14F012BD19
:102FD000B3F008BA8EF05ABE14F0B2BF03F044BF8B
:102FE00014F092BC14F010BC7CF060BE62F01EBB0A
:102FF0002AF078BD07F096BA03F020BA7FF052BFEE
:1030000014F0E0BF07F07CBE05F0A6BA07F0ECBFF5
:1030100006F04EBB07F036BB14F03CBBFFF736BDE5
:1030200035F026B900F5E04008B5D0F8280BBCF023
:10303000A3FF012008BD000010B400F5004400F516
:10304000A0402034D0F8C40FA04203D15DF8044B57
:1030500009F0BEBE00205DF8044B704700F5004348
:1030600000F5A0402033D0F8C40F984201D109F0F8
:10307000CDBE704707F024B80BF0FEBE0BF036BD96
:103080000BF0CABC1FB500F5A04304460391D3F86A
:10309000C40F03685B6A984760B10023DFED060A3E
:1030A00004F506400399B0EE600A1A46803000939A
:1030B0000EF0D0FD04B010BD0000000000F5A043EC
:1030C00010B504462DED028BD3F8C40FB0EE408A44
:1030D00003685B6A984720B900242046BDEC028B48
:1030E00010BD04F506409FED070A803028EE000A67
:1030F0000DF0DAFF04460028EED001210248FFF768
:103100003FFCEAE70000C842C83200307FB5044601
:1031100068460D46164620F085F804F5A04369463A
:10312000D3F8C40F03685B6D98476946284620F0C2
:1031300079F910B9002004B070BD6946284620F026
:103140007DF90028F6D0284620F09CF80546304648
:1031500020F098F88542EDD12368314620461B6A5D
:103160009847E8E730B50C4600F5A04105462DED3F
:10317000028BD1F8C40F89B0B0EE408A0168F0EE3E
:10318000608A0392496A0293884728B39FED140A24
:1031900005F506409DF83C1094ED006A68EE800A43
:1031A000D4ED016A803094ED027A26EE006A66EE74
:1031B000806A019127EE407A9DF8381028EE000AC7
:1031C000029B009105A9039A8DED056ACDED066A73
:1031D0008DED077A0EF05EFC09B0BDEC028B30BDC0
:1031E0000000C84200F5A04370B50646D3F8C40FEE
:1031F0008EB00D46036814465B6A9847D8B3DFED7E
:103200001F7A002395ED006A06F50640D5ED016AA8
:1032100008AA95ED027A26EE276A66EEA76ADFED28
:10322000180A27EE677A00938DED056AB0EE600A02
:1032300094ED006A05A9CDED066A8030D4ED016AEF
:1032400026EE276A8DED077A94ED027A66EEA76A7C
:103250008DED086A67EE677ACDED0B0ACDED096A50
:10326000CDED0C0ACDED0A7ACDED0D0ACDE9013395
:103270000BAB0EF0F3FD0EB070BD00BF0000C842F6
:1032800000000000F0B51C4600F5A04307460E46BE
:1032900015462DED028BD3F8C40F8FB0B0EE408AE7
:1032A0000368F0EE608A5B6A984700284CD09FED77
:1032B000280A07F5064096ED006A08AAD6ED016ACD
:1032C00068EE800A96ED027A26EE006A66EE806A63
:1032D0009DF8603027EE407A05A98DED056A8030B3
:1032E00095ED006ACDED066A8DED077A26EE006A4F
:1032F000D5ED016A95ED027A66EE806A8DED086A79
:1033000027EE407A94ED006A0293CDED096A26EE2D
:10331000006A9DF85C30D4ED016A8DED0A7A94ED77
:10332000027A66EE806A019327EE407A9DF8583063
:1033300028EE000A8DED0B6A00930BABCDED0C6A05
:103340008DED0D7A0EF08AFD0FB0BDEC028BF0BD55
:103350000000C84200F5A04370B50646D3F8C40F7C
:1033600086B00C4603685B6A9847054610B39FED2C
:10337000136A0023D4ED006A012294ED017A06F568
:103380000640D4ED027A66EE866A27EE067ADFED15
:103390000C0A67EEC67A03A9B0EE600A8030CDED64
:1033A000036A8DED047ACDED057ACDE900321A4637
:1033B0000EF05CFB284606B070BD00BF0000C8429E
:1033C00000000000F0B5144600F5A04207460D4687
:1033D0002DED028BD2F8C40F8DB0B0EE408A02689A
:1033E000F0EE608A0593526A90470646C8B39FED97
:1033F0001F0A012295ED006A07F50640D5ED016A26
:1034000068EE800A95ED027A26EE006A66EE806A22
:10341000029227EE407A9DF854208DED066A06A9A7
:1034200094ED006A8030CDED076A8DED087A26EEC6
:10343000006AD4ED016A94ED027A66EE806A019228
:1034400027EE407A9DF8502028EE000A059B009256
:1034500009AA8DED096ACDED0A6A8DED0B7A0EF0A1
:103460009BFA30460DB0BDEC028BF0BD0000C842A7
:1034700000F5A04370B506462DED048BD3F8C40FBC
:1034800088B0F0EE408A0368B0EE609AF0EE419AA0
:103490005B6AB0EE618A9847054600B39FED120A59
:1034A00000244FF07E5304A829EE801A079469EE99
:1034B000000A049328EE800A069405943AF0F2FC80
:1034C0009FED0A0A06F50640002301AA28EE000A2D
:1034D00004A980300194029403940EF0F1F8284678
:1034E00008B0BDEC048B70BD35FA8E3C0000C842BC
:1034F00000F5A04330B505462DED048BD3F8C40F7D
:1035000089B0F0EE409A0368B0EE609AF0EE418A1E
:103510005B6AB0EE618A98470446F0B14FF07E5383
:1035200004A8049300230793069305933AF03CFF05
:103530009FED0C0A01A8CDED019A8DED029ACDED1B
:10354000038A3CF02FFB05F50640B0EE480A012344
:1035500001AA04A980300EF0B3F8204609B0BDECF2
:10356000048B30BD35FA8E3C0A4A0B4692F9B82FCF
:10357000002A05DA00228A604A600A60012070474A
:1035800000F5E040D0F8142B783207CA83E8070032
:10359000F4E700BFC8820030694B70B5044640F8BC
:1035A000043B86F0B9FB002504F1100004F57556C4
:1035B0001CF060FE04F168006CF0BAFD04F5907038
:1035C00028F032FC04F5AA601BF050F904F2EC601C
:1035D00020F06EFB04F6382033F0A8FD04F5A65069
:1035E0003C36083086F046F904F5AC50183066F0E9
:1035F000D7FE04F5C25008306FF0D2FA04F5C85077
:1036000091F0E4FE04F5C8501C307FF0D5FA04F5C3
:10361000CA5018301EF052FF04F5D0501430A5F0F7
:103620000DF904F502502430B1F012FB04F50350FB
:103630006DF03EF904F50450143087F01BFD04F5DD
:10364000005304F505503F4A83F8385104F50453FC
:103650000830383313605FF0CBFC04F50650294680
:10366000183017F043F804F5225010308AF046FE67
:1036700004F52350A2F09AFA04F547500C30AAF052
:103680002FF904F54B502430A8F02CFF04F54C50D2
:103690000C30ACF041FB04F54E501830B0F032FC69
:1036A00004F54F503C30B1F067F804F55150143038
:1036B000A1F09AF904F553503C3015F0CFFF04F512
:1036C00059502830A3F068F804F55B50B2F058FC6C
:1036D00004F568501C49143065F020FA04F5685070
:1036E0002C3092F01DFC04F56B502830B2F01CFB1E
:1036F00004F56D50C9F090FB04F5405383F8EC5B82
:1037000004F56F553C3528460C3571F001FFAE428B
:10371000F9D104F576500D4D0830B2F085FB04F573
:1037200076502C3071F0F0F92B6813B10848C9F0CD
:1037300025FB2046074965F0F1F920462C6070BD55
:10374000E4A5150888CC00300080160828C2003097
:10375000846914085CA4150810B514F019FB7CF0FA
:1037600067FB0368BDE810405B681847FFF7F4BFCC
:1037700010B5044607F024F8204614F071FE2046E8
:1037800004F032FD2046BDE8104004F09BBE00006E
:10379000FFF7EEBF70B500F5C04504461435284666
:1037A0001CF032FC21F080F890F9253093B390F8AA
:1037B00044337BB304F5A04304F2EC66D3F8E80F7E
:1037C000443071F0A9FE0346B7EE001A9F20DFEDEA
:1037D000120A93ED000A36F03BFD94F9243728468F
:1037E0000021012B04F6481408BF86ED0F0A1CF0D7
:1037F000A1F9DFED0A7A94ED287A304620EE270A07
:10380000DFED077AA7EE270A84ED280ABDE87040AD
:1038100020F042BF70BD00BF00000000CDCCCC3D09
:103820006666663FFFF7B6BF10B50121044614F087
:1038300053FE60B1114BD3F8C40F03689B6A9847DD
:1038400028B9204602F000FD204602F00DFD4FF49D
:103850000011204614F040FE18B135F09FFE33F001
:1038600035FB4FF48021204614F036FE28B135F0A8
:1038700095FEBDE8104033F02DBA10BDC88200306F
:10388000FFF7D2BF7FB500F5E04604469FED660A1C
:10389000D6F8140B6C303CF031F904F5065001A950
:1038A0008DED010A1830CDED020A8DED031A16F0E8
:1038B000B1FD0221204614F00FFE70B10121204617
:1038C00014F00AFE48B9594BD3F8C40F03689B6A39
:1038D000984710B9204602F0B7FC0121204614F0A9
:1038E000FBFD48B9514BD3F8C40F03689B6A984756
:1038F00010B9204602F0B8FC0121204614F0ECFD7E
:1039000010B9204602F00AFD4FF40031204614F0B1
:10391000E3FD30B104F5A043D3F8E80F03685B6C16
:1039200098474021204614F0D7FD68B104F5C255F0
:10393000083528466EF0E6FB04F5805393F91C39F0
:1039400013B128466EF0A2FD4FF48061204614F0BA
:10395000C3FD20B104F5C25008306EF06DFC20218B
:10396000204614F0B9FD58B104F5A045D5F8C40FB0
:1039700003681B699847C8B3D6F81C0BB9F078FEEA
:103980008021204614F0A8FD00283CD035F006FE2A
:1039900033F0C4F91021204614F09EFD68B1D6F82A
:1039A000140BB6F0DFF904F57D5014308EF09EFA5A
:1039B00004F57A501830B2F087FD4FF6FF712046BB
:1039C00014F08AFD20B104F5AF407430C4F04CF916
:1039D0004FF40041204614F07FFD18B304F5F74082
:1039E000343004B0BDE870407FF0CEBB20460FF00D
:1039F00053F80028C0D1D5F8C40F03685B69984715
:103A00000028B9D0BCE74FF48021204614F064FDB3
:103A10000028BBD14FF40021204614F05DFD0028A2
:103A2000B4D1B7E704B070BDE02E6542C882003063
:103A3000FFF728BF10B50121044614F04DFD10B169
:103A4000204602F06BFC8021204614F045FD48B171
:103A50004FF48021204614F03FFD18B935F09EFD4B
:103A600033F038F94FF40011204614F035FD30B131
:103A700004F5D050BDE810401430A4F0F5B810BDE6
:103A8000FFF7D8BF10B5044606F0EAFB204606F063
:103A900039FA204606F02AFC204615F02FFC204675
:103AA000BDE8104004F09CB9FFF7ECBF70B50446C8
:103AB0004FF6FF7114F010FD04F5A04528B1D5F8BC
:103AC000B82F0721204602F05BFCD5F8E83F93F8B9
:103AD000D5309BB92046FEF7C5FFD5F8E80F04F5B1
:103AE000804304F54052016892F82E2E0E6A93F836
:103AF000FC18B047D5F8E80FC1F062FB7EF0ECFA95
:103B00007DF01EFF204615F0F7FB95F8B83F04F551
:103B1000E0440F4ADB43D4F8145BC3F3C013537182
:103B200084F89D3E2B681E6F6CF02AFE6CF092FAB2
:103B30002846B047D4F81C4B6CF022FE04F50574FF
:103B40006CF088FA2046BDE87040A0F0E5BA00BFEE
:103B50002DC10030FFF7AABFF8B500F5005600F5FB
:103B6000BF4700F5C0450446D6F8E833FB67D6F8F2
:103B7000F4332B60D6F8980300F58C40503036F0C3
:103B800035FB6860FB6F4FF6FF712046AB602B681A
:103B9000EB6014F0A1FC38B1D6F898232046092137
:103BA000BDE8F84002F0C2BBF8BD000000F5A0433C
:103BB00010B5D3F8F84F002C4FD093F8B92FD10798
:103BC0004BD56FF30002D3F8441B012C83F8B92FB7
:103BD000D3F8482BB1F90840B2F9082007EE104A93
:103BE00008BF03F6FC7406EE902A00F5C042B8EE5A
:103BF000C77A03BFD4ED007AF8EEE66AD2ED005A38
:103C0000F8EEE66A1CBFD2ED035AD2ED027A00F557
:103C1000005025EEE66AA7EE276A67EEA67AD0ED99
:103C2000FA6AE7EE257A90EDFD7A27EE877AA6EE1E
:103C3000267ABDEEC77A17EE102A0A8190EDFA7A3D
:103C4000D3F8483B67EE877A90EDFD7AE6EE477A47
:103C5000FDEEE77A17EE902A1A8110BD10B50446E2
:103C60002DED028B79B1204604F5C04413F0E6FE39
:103C700040F2E63263681B1A03F2F31393420ED844
:103C8000BDEC028B10BD00F5A043D3F8F83F022B2A
:103C9000F6D113F0B3FEB0F57A7FE4D2F0E700F589
:103CA0008C4360606420503393FBF0F300EE103AD5
:103CB0009FED0A7BB8EEC00B20EE070BB7EEC08B72
:103CC000B0EE480A19F110FD84ED020AB0EE480A80
:103CD0001AF1A6FB84ED030AD2E700BF000000A0A2
:103CE00046DF913F00F506500121183018F054BB13
:103CF000FFF7F8BF10B5044614F0D8F8102120469D
:103D000014F0EAFB98B1204602F0F4F94FF40011E8
:103D1000204614F0E1FB50B935F040FC33F0D6F802
:103D200004F5D050BDE810401430A3F09DBF10BD85
:103D3000FFF7E0BFF8B5044607F06AF8224B4FF6EC
:103D4000FF76254604F180004FF0FF3745F83C3BF5
:103D50001E4BA465C4E917341D4BC4E919341D4B2F
:103D6000E3661FF05FFA04F19C001FF05BFA04F1B8
:103D7000B8001FF057FA184B04F1D400A4F8D06033
:103D8000C4F8CC301FF04EFA144B15492846C4F83D
:103D900084721D6064F0C2FE04F52670A4F8787089
:103DA000A4F894601FF03EFA04F52D701FF03AFA63
:103DB00004F534701FF036FA0023204684F8E4320C
:103DC000C4F80833F8BD00BF1CD1140879300208CC
:103DD0007D300208813002080000FFFFFCC0003087
:103DE000705E150810B5044607F012F80A4B04F18E
:103DF000400023600123A3871FF014FA04F1500050
:103E00001FF010FA04F160001FF00CFA04F17000CA
:103E10001FF008FA204610BD84DC14082DE9F04399
:103E2000044689B0FFF7B8FBB44B04F5795004F5AC
:103E3000A04523604FF07C57103004F5F54602F0A2
:103E40006DFC04F5785304F5B64005A91C330597BD
:103E500068307836C5F8583B06234FF0010804F562
:103E6000BC4985F85C3B71F069FC04F5B740C8F0CB
:103E700049F90023049704F5B74785F8983B1923BF
:103E800004A907F1300085F8A43B09F12009C5F821
:103E9000A06B71F053FC07F1480004F5B847C8F077
:103EA00031F9182385F8E08B6837C5F8E86B85F899
:103EB000EC3B04F5B8407EF011FA3846B3F03EFA18
:103EC00006AE8F4B381D31468DF81880C5F8683C1A
:103ED00004F5BB4865F0FCFD04F5B940894F483056
:103EE00061F054FB04F5BA400830B2F05FF8864B3D
:103EF00004F5BA403146C5F8083D2030069771F008
:103F00001DFC04F5BA40314606972C3071F016FCC2
:103F100004F5BA40069704F5BA473146383071F0D7
:103F20000DFC5037794B07F10C00C5F8503DC8F037
:103F3000E9F8404608F1140876F066FEC145F8D16C
:103F40001E2340F2CC60C5F8503F0023A5F8543F33
:103F50001FF056FEC5F84C0F04F5BE405830C8F0AF
:103F6000D1F804F5BF401C30C8F0CCF8684B1A6893
:103F700002B91F6004F50848664B04F5BF404FF0D6
:103F80007E5708F16C08C5F8503D483005F6FC75C1
:103F900045F8388C04F5F949B4F0A4FE04F5C043A3
:103FA0002F6004F5C0409F604FF400715A4B1430ED
:103FB000069404F5E045079309F14409574B009333
:103FC00096E80C001BF060FB04F5CB4000262C307B
:103FD00098F0FEFD04F5F54003A90397483071F011
:103FE000D7FB04F5F54003A903975C3071F0A6FBFD
:103FF00004F5F54068301FF015F905F6F82304F5CF
:10400000F6404FF400411E605E6034309E6005F65D
:1040100004331E605E609E6004F506531833C5F8D5
:10402000103B002385F8313B1CF008FA04F5F740FB
:1040300034307EF011FF04F5F840383094F0A8FBDE
:1040400004F5F840743065F079FE354B04F5F9401D
:10405000C5F8743C083091F06BFE04F5F940314B23
:1040600024303149186064F059FDFF232F49484638
:1040700085F8D43C85F8DC3C64F050FD2C4B1F687F
:1040800017B12C48C8F07AFE04F5F940C3F8009047
:1040900004F5FB496430BAF04FFF04F5FB4009F129
:1040A00060095830BAF006FE48469FF0E3F904F57F
:1040B000FE4049461030C2F075F81F4B04F5FE4231
:1040C000DFF88CC0C5F8103F0623703285F8643FD6
:1040D0001A4BC3F800C03B46142798B2013307FBC4
:1040E00000C1097C0029F8D1154B1880154B1880A8
:1040F000154B1F6877B31548C4E700BF1C7414083C
:10410000086914080000A0404C6914089CC71508F1
:104110009CC6003000751408753002080C74140831
:104120005C69140890CC0030F8E71508347E160856
:1041300050CD00309869140830C81408E8C1003028
:10414000E6C10030BCC1003090C10030B96914082C
:1041500014BE140804F5FF401A606E4B03A9043026
:1041600004F50349039371F0E9FA04F5FF4009F1FE
:104170006409243006F04CFE674B04F5FF40C5F897
:10418000A43F643006F044FE644B04F50040C5F8DB
:10419000E43F04F500452030FFF7CCFD484606F02B
:1041A00037FE5F4B09F13C00C5F86433C5F0BAFC3B
:1041B0005C4B04F50540C5F8A033243006F028FE1A
:1041C000594B04F50540C5F82435683006F020FE4B
:1041D000564B04F5054085F8A475C5F86835A83038
:1041E00006F016FE524B04F50540C5F8A835E4303C
:1041F00006F00EFE4F4B04F50640C5F8E43505F514
:10420000C46338301E605E609E6006F001FE4A4B5B
:1042100004F50640C5F87476C5F83836803006F0E7
:10422000F7FD464B04F50640C5F8BC76C5F8803668
:10423000C43006F0EDFD424B04F50740C5F8C43626
:104240000C3006F0E5FD3F4B04F50740C5F80C3790
:104250004C3006F0DDFD3C4B04F50740C5F84C370B
:1042600005F2C473E0301E605E60FFF7BBFD4046A0
:1042700006F0CEFD354B04F50840C5F86C38A83083
:1042800010F040FE04F50940643006F0C1FD304BEB
:1042900004F50940C5F8A079C5F86439A83006F0DE
:1042A000B7FD2C4B04F50940A5F8E479C5F8A83909
:1042B000F83006F0ADFD284B04F50A40C5F8347A15
:1042C000C5F8F8393C30FFF78DFD244B04F50A4062
:1042D000C5F83C3A0123D83085F8C53A05F6CC2319
:1042E00005F664451E605E609E600BF095FF04F568
:1042F0000B40AC3012F07CF904F50C40243006F091
:1043000087FD174B204645F8403C2E606E6009B093
:10431000BDE8F083CDCC4C3D0CCD1408B4CD1408D1
:10432000C4D1140858D21408BCD3140860D414089B
:1043300004D51408A0D51408E4D7140888D81408A4
:10434000C8D9140864DA140808DB1408E8DD140876
:1043500018D314080CE2140834D9140840DD1408EA
:10436000D4E2140838B5054B0A4601461C68236898
:1043700020461D68024BA847002038BD38BF0030DA
:10438000C832003038B5037904463BB905682DB111
:10439000284631F033FE28461FF034FC204638BD55
:1043A000314B70B50360044600F5665034301EF0A2
:1043B000C1FE04F5405393F8F02342B9D3F8EC530F
:1043C0002DB1284631F01AFE28461FF01BFC04F5DB
:1043D000025004F5AA5504F5A75624300C35B0F068
:1043E0004BFC04F5E1500C360830FFF7CBFF04F529
:1043F000E150FFF7C7FF04F5E0501830FFF7C2FFA8
:1044000004F5C8501C307EF0EFFBB54204D0183DD7
:10441000284631F04DFAF8E7144B04F5766504F6BA
:104420001876C4F8383AB54204D0083D2846FFF75C
:10443000A9FFF8E704F6FC3070F032FD04F53D60AA
:1044400070F02EFD04F6A43070F02AFD04F6F8207A
:1044500070F026FD04F6CC2070F022FD04F52A60F1
:1044600070F01EFD204670BDE4A51508404D1508EE
:1044700038B5104B0446036000F5E04393F8042F71
:1044800042B9D3F8005F2DB1284631F0B7FD284678
:104490001FF0B8FB04F5A043074AD3F84C0FC3F84C
:1044A000502D08B11FF0B2FB2046FFF779FF2046E0
:1044B00038BD00BF1C7414089CC7150810B5C8F09F
:1044C000F1F8064C064B18602046FFF7A7FC204683
:1044D000044A0549BDE8104019F100B9C83200305E
:1044E00038BF0030586A013071440208012070471B
:1044F00090F8D0308B4286BF00EB8100D0F8D4001A
:104500000020704790F8D0308B4286BF00EB8100CE
:10451000D0F8D40000207047FA207047014B93F880
:10452000DE0D7047C8620030034BD3F8F80F431E0E
:1045300058425841704700BFC8820030034BD3F83F
:10454000F80F831E58425841704700BFC8820030A0
:10455000034BD3F8E80F08B1BFF01ABB014870470E
:10456000C8820030EC741408F8B5436A0446444D20
:1045700043F4E0524262826A42F4E0528262C26ACA
:1045800042F4E052C262D5F81C2BE2B143F4F84386
:104590004362D5F81C0BB8F005FB38B1A36A43F4AD
:1045A0008043A362E36A43F48043E362D5F81C0BC3
:1045B000B8F022FC38B1A36A43F40053A362E36A63
:1045C00043F40053E3622F488DF09CFB18B1636AFB
:1045D00043F0806363622B488DF040FB18B1A36AFF
:1045E00043F08063A36227488DF0BEFB18B9E36AED
:1045F00043F08063E362244B1E6846B119213046C4
:1046000065F0A8FF18B1636A43F4807363621F4FBB
:1046100097F8603B6BB1A36A43F48073A36246B121
:104620001921304665F0E4FF18B1E36A43F4807362
:10463000E36295F9E43C8BB1D4E9092343F08003AC
:1046400042F08002A362626295F9E43C33B195F8CE
:10465000CC3D1BB1E36A43F08003E362636A43F03D
:1046600080436362A36A43F08043A362D7F8E83FC4
:1046700093F8C1301BB9E36A43F08043E362F8BDAD
:10468000C8A200301C720030F4C10030C882003073
:1046900013B54FF44470CDE900211FF0ABFA044686
:1046A00028B1DDE900217AF053F8024B236020465F
:1046B00002B010BD48771408002070477047000012
:1046C0000320704708207047014B93F8E00D7047B6
:1046D000C8620030034B93F9F008003818BF01207E
:1046E000704700BFC8720030014B93F9E20D70476C
:1046F000C86200307047000008B50C4BD3F81C0BA3
:1047000070B910230A4A43F04000D2F8E82F22B1D2
:1047100092F8D5200AB143F0C00040F0010008BD76
:10472000B8F040FA0028ECD01823EBE7C8A200301C
:10473000C882003038B5C5780B4604463522352D81
:104740004FF00001184628BF35251CF143FF04F146
:104750000C012A46BDE838401CF1F2BE00B500232A
:1047600089B002930393049305930693079317F07C
:10477000ADFE02A917F07AFCA0B117F0A7FE00F574
:104780005A7005AB07C883E8070018463BF0D4FD14
:10479000F1EE047A20EE270AFCEEC07ACDED017A24
:1047A0009DF8040009B05DF804FB00001FB5184C2B
:1047B00094F8521604F2FC4015F072F978B194F8AE
:1047C000521604F2FC4015F0EBFB40B194F852167F
:1047D00004F2FC4004B0BDE8104015F025BC0023F5
:1047E00001930293039317F071FE01A917F03EFCA9
:1047F00020B101A83BF0A0FD04B010BD29F0B0F934
:10480000B02290F8F43202FB030090ED3B0AF3E78C
:10481000C862003008B50D4BD3F8E80FA8B144309A
:1048200070F07AFE0346B7EE001A9F2093ED000A5F
:10483000DFED070A35F00CFDDFED067A20EE270AE2
:10484000BDEEC00A10EE103A18B208BDC8820030A2
:10485000000000000000C8422DE9F04FDFF8D880CA
:104860008DB00446334F042508F5804617F8019BA8
:10487000B8F9383E09F1FF3A43FA0AF3D90742D5AD
:10488000207C72F013FD8346207C73F02DFC00F138
:1048900021039B4505D2207C0DB0BDE8F04F71F09F
:1048A00023BFBAF1030F2ED8DFE80AF00234393EF5
:1048B000D6F8140B03689B68984700F1A0035A6967
:1048C000D3F800A0D3F804E0D8681969D3F818C069
:1048D00008925A6A1B6ACDF825206222CDF8293049
:1048E000212306900791C221207CCDF80CA0CDF8A1
:1048F00010E0CDF814C08DF82490CDE900321923D2
:1049000003AA72F051FD013D15F0FF05AED10DB0C7
:10491000BDE8F08FD6F8140B0368DB68CCE7D6F857
:10492000140B03681B69C7E7D6F81C3B03F52D730E
:10493000C5E700BF38781408C862003007B5019099
:10494000C3F0A6F928B1019903B05DF804EBC3F0F8
:104950005BB903B05DF804FB13B504460748019149
:1049600009F0B0FF30B90199204602B0BDE810400F
:1049700073F01ABE042002B010BD00BFE8B20030D0
:10498000014809F039BD00BFE8B200300B4B70B5EB
:10499000D3F8F43805460E461446DB0703D5114616
:1049A0000748C1F0BDFF21460648C4F029F8224659
:1049B00031462846BDE8704078F0AABAC872003087
:1049C000D8B10030E08A003010B588B0044675F0E8
:1049D0006BF90C4BD3F8E80F38B90B4A0621204687
:1049E00008B0BDE8104075F047B969461E22BFF017
:1049F000D7F86B46054A0621204675F03DF908B008
:104A000010BD00BFC8820030387514087D471708F4
:104A1000034A92F8403B013382F8403B74F09AB865
:104A2000C88200300148BAF0B3BC00BFACAF003060
:104A300007B5084601911EF02DFD38B104480199D3
:104A400002F0FCFF002003B05DF804FB0420FAE74D
:104A500044BF0030F7B58B8B06460C461746CD2B6E
:104A60001DD1D1ED067AFCEEE77ACDED017A9DF805
:104A70000430022B13D10E4D95F82D1C05F6B430E1
:104A80007EF020FA58B195F82D1C05F6B4307EF072
:104A900021FA20B994ED020A064802F0AFFF3A4627
:104AA0002146304603B0BDE8F04074F0E5B800BFE1
:104AB000C8A2003044BF0030162A10B40C4605D0FE
:104AC000542A03D05DF8044B73F08ABD0323012000
:104AD00023705DF8044B704708B573F0F1FF40F4A4
:104AE0001C6040F00D0008BD1FB517F0EFFC044638
:104AF00068461EF097FB6946204617F0FBF90E4BFF
:104B000093F8B90F10F0200014D003F50053DDED39
:104B1000017AD3F81C3BF8EEE77A93ED0F7A77EE43
:104B2000877A9FED067A67EE877AFDEEE77A17EED1
:104B3000903A18B204B010BDC88200300AD7233CA6
:104B400010B504461FF05EF8204610BD10B50C4CA1
:104B500094F9B83F002B0FDBD4F8C40F0368DB6C6B
:104B6000984758B9D4F8C40F03689B6C984700283D
:104B70000CBF0220032010BD0120FCE70420FAE74F
:104B8000C882003008B5134B93F8B90F10F020001D
:104B90001ED0D3F8C40F0368DB6D984707EE900A68
:104BA000F2EE046AB8EE677ADFED0B7A27EE277A29
:104BB000DFED0A7AB4EEE77AF1EE10FA58BFB0EE04
:104BC000677AC7EE267AFCEEE77A17EE903A98B24B
:104BD00008BD00BFC88200300AD7233C00FF7F47D2
:104BE00010B44C69012C05D101465DF8044B034813
:104BF00003F010BD5DF8044B73F0C6BFC83200303F
:104C00002DE9F341B1F9043006460C461546002B58
:104C100035DB1C4F4FF000089FED1B0A4FF47A73F1
:104C2000CDE90028B1F90220D7F8441B78F0C2FC86
:104C300001239FED150A3046B4F90020D7F8481B30
:104C4000CDE900534FF47A7378F0B4FC9FED0F0A6E
:104C50004346B4F90420D7F84C1B3046CDE9005840
:104C600078F0A8FC9FED080A4FF47A73B4F9062097
:104C7000D7F8501B3046CDE9005878F09BFC02B0C5
:104C8000BDE8F081C88200300000FA4400007A4498
:104C900008B5094B93F8B90F10F020000AD0D3F8EB
:104CA000C40F03689B6D984735F0A0FAC82390FBAA
:104CB000F3F0C0B208BD00BFC8820030044B1878C2
:104CC00020B9044B93F8BA0FC0F38010704700BFAF
:104CD000CCC00030C88200307FB50023039304931A
:104CE000059317F0F3FB03A917F0C0F9D8B117F03B
:104CF000EDFBD0EDDA0A90EDDB0AF1EE600AB1EEE1
:104D0000400A19F189FDDFED097A20EE270A35F016
:104D1000E3F9F6EE007A20EE270AFCEEC07ACDED3C
:104D2000017A9DF8040007B05DF804FBE02E6542AF
:104D3000124B07B593F8B90F10F020001AD003F505
:104D40000053D3F81C0B00F565703BF0F5FADFED6E
:104D50000C7A20EE270ADFED0B7AB4EEE70AF1EECB
:104D600010FA58BFB0EE670AFCEEC07ACDED017ABA
:104D70009DF8040003B05DF804FB00BFC88200305A
:104D8000CDCC4C3D00007F430C4B93F8A9258AB94C
:104D9000A3F5805213F8233C9B060BD192F9B83F40
:104DA000002B09DB92F8B93F13F0200F14BF042049
:104DB000012070470520704703207047C8920030DB
:104DC00008B5074B93F92C3E032B03D0BDE80840F0
:104DD00074F0CABF034A022174F04EFF042008BDDC
:104DE000C862003050751408094BD3F8F4289207B4
:104DF00001D473F0E9BB03F54053DFED067A03F607
:104E0000EC2393ED000AB8EEC00A20EE270A7047A3
:104E1000C87200300AD7233C10B594B0044603A8EA
:104E20001EF000FA1C4B03A9D3F8C40F03685B6D96
:104E3000984778B3002103A81EF08CFA50B3247C65
:104E4000C7F0CAFF059B9622DDED047A572108932F
:104E5000069BF8EEE77A9FED117A0993002367EE3F
:104E6000877A07900B9320460C930D930E930F9324
:104E70001093119312934FF6F853CDED0A7AADF8D3
:104E80004C3000238DF84E303323CDE9003207AA91
:104E900072F08AFA14B010BDC88200300AD7233CE1
:104EA00030B5844C05462DED0A8BD4F8C40F99B06B
:104EB00003685B6A9847002867D004F54054D4F82B
:104EC000BC36062B00F2E180DFE803F00404046343
:104ED000A0C35F00784840F6F8540DF0C7F89FED86
:104EE000778A9FED770AF0EE489AB0EE48AAF0EE86
:104EF000488AF0EE48AAB0EE48BA90ED027B90EDF9
:104F0000005BF7EEC76BB7EEC55B90ED047B0BA8BB
:104F10008DED0B5ACDED0C6AB7EEC77B8DED0D7A9A
:104F20003AF0ECFDB0EE40CAF0EE60BAB0EE419A55
:104F30002D7CC7F051FF00238C22B1EE499A0B90D3
:104F40001593F1EE688A16930123B1EE488A552134
:104F50008DF85E30332328468DED0CCACDED0DBAA9
:104F60008DED0E9A8DED0FBACDED10AACDED118A13
:104F70008DED12AACDED139A8DED148AADF85C403B
:104F8000CDE900320BAA72F00FFA19B0BDEC0A8B12
:104F900030BD49484FF440640DF068F89FED480A71
:104FA00090ED027B90ED005BF7EEC76BB7EEC55B53
:104FB00090ED047B0BA88DED0B5ACDED0C6AB7EE8E
:104FC000C77B8DED0D7A3AF099FD3B48F0EE60BA63
:104FD000B0EE419AB0EE40CA0DF04CF89FED380AA1
:104FE0003AF08CFD3448B0EE40BAF0EE60AAF0EE34
:104FF000418A0DF043F89FED320A3AF07FFDF0EE62
:10500000609AB0EE40AAB0EE418A91E72A4840F695
:1050100007440DF02FF89FED2A0A3AF06FFD26485D
:10502000B0EE40BA9FED259AF0EE60AAF0EE418A0C
:105030000DF024F89FED220AF0EE49BA3AF05EFD39
:10504000B0EE49CAB0EE40AAF0EE609AB0EE418AE6
:105050006EE7194840F63F44DFED188A0DF00EF870
:105060009FED170A3AF04AFDF0EE68AAB0EE40AAAA
:10507000F0EE609AB0EE418AB0EE68BAB0EE689A8F
:10508000F0EE68BAB0EE68CA52E79FED0C8A0024D1
:10509000F0EE489AB0EE48AAF0EE488AF0EE48AA40
:1050A000B0EE48BAB0EE489AF0EE48BAB0EE48CA50
:1050B0003EE700BFC882003048B900300000000061
:1050C0000AD7233C2DE9F0413C4D04462DED068BDB
:1050D00095F8B93F8CB099066AD505F50057DFED14
:1050E000388A9FED380AD7F8140B6C303AF006FD79
:1050F0008DED041A21EE281AD5F8C46F8DED020A41
:1051000060EE289ACDED030A3046BDEEC11A94F840
:10511000108020EEA89A11EE103A1DB233689B6DF4
:10512000984707EE900A3046F8EEE77A67EEA87ADD
:10513000FDEEE77A17EE903A1CB23368DB6D9847C4
:1051400007EE900AD7F81C3B3046B8EE678ADFEDD1
:105150001E7A93ED0FAA336828EE288A1B6E2AEE7A
:1051600028AAB4EEE78AF1EE10FA58BFB0EE678ACB
:1051700098470023B72220EE280A3E21BCEEC88AB9
:1051800008934046CDED059A8DED069A18EE103A3B
:105190008DED07AA8DED090AADF82C301A23ADF874
:1051A0002850ADF82A40CDE9003205AA72F0FCF88B
:1051B0000CB0BDEC068BBDE8F08100BFC8820030AA
:1051C0000AD7233C9F0CB34500FF7F471C4B2DE9BA
:1051D000F04F2DED028BD3F8143B8DB0047CD3F847
:1051E0008480D3F88870D3F88C60D3F8905093ED16
:1051F000258AD3F898B0D3F89CA0D3F8DC90C7F0F8
:10520000EBFD00231622029053218DF82C3025232C
:1052100020468DED078ACDF820B0CDF824A0CDF83A
:105220002890CDF80C80049705960695CDE90032BC
:1052300002AA72F0B9F80DB0BDEC028BBDE8F08F98
:10524000C8A2003070B58A7A06464B7A0C4643EA0B
:105250000223CA7A43EA02439D2B21D1134D95F8CC
:105260002D1C05F6B4307DF02DFEC8B195F82D1C2F
:1052700005F6B4307DF03AFE022811D195F82D1CC8
:1052800005F6B4307DF026FE50B9D4ED057A9FEDD9
:10529000080AF8EEE77A074827EE800A02F0AEFB2C
:1052A00021463046BDE8704073F054BBC8A20030C0
:1052B0000AD7233C44BF0030054BD3F8E83F2BB15D
:1052C00093F8CA00002808BF0220704702207047E8
:1052D000C882003008B5034BD3F8C40F03681B68BD
:1052E000984708BDC8820030024B93F8B90FC0F34D
:1052F00040107047C882003070B52C4E05460C46F1
:10530000D6F8C40F2DED028B036886B091ED018AAB
:105310005B6A984750B9BDEEC88A18EE103ADB07B1
:1053200004D4022006B0BDEC028B70BDD4E90401A8
:1053300036F0A8FA0028F4D002A81DF073FF02AAE4
:105340002146284678F044F80028EAD0184902A8F7
:105350001EF0ACF803460028E3D1DFED160A024642
:10536000009002A9B0EE600A13480CF073FCD8B1AB
:10537000D6F8C40F03685B6A9847044608B100205A
:10538000D0E7022204210D4806F088F960B1DFED74
:10539000090A2346224602A9B0EE600A0648009494
:1053A0000CF058FC0028EAD10420BBE7C88200308A
:1053B000B0AD00300000000048B90030C832003005
:1053C00008B591F82030032B1CD1D1ED027A9FED66
:1053D0000E7AF0EEE77A91ED060A0C4BF4EEC77AFE
:1053E000DFED0B7AD3F8C40F20EE270AF1EE10FAA6
:1053F0004CBF0121002113F0BFFB002814BF002087
:10540000042008BD0220FCE700000034C882003000
:105410000000C84210B52DED028BD1ED007A82B0AC
:105420000C46F5EEC07AF1EE10FA04DA042002B070
:10543000BDEC028B10BD9FED197AF4EEC77AF1EE48
:1054400010FAF3D891ED030A9FED158AF0EEC07AB9
:10545000F4EEC87AF1EE10FA19D5D4ED037A1148BA
:10546000F4EEC87AD4ED027AD4ED010AFDEEE77AC3
:1054700094ED000AF1EE10FACDED017AACBF0122F5
:1054800000229DF9041002F01DFA0020CFE7F7EE8C
:10549000000A34F07BFD0028C8D0DEE70000B443EA
:1054A0000000003444BF003091ED010AB5EEC00A9F
:1054B00008B5F1EE10FA01DC042008BD9FED107A6A
:1054C000D1ED007A20EE070A9FED0E7A0E4BF4EE36
:1054D000C77AD3F8C40FF1EE10FA036805DDDB6E6E
:1054E00098470028E8D00020E7E79FED087AF4EE1F
:1054F000C77AF1EE10FACCBF9B6E5B6EF0E700BF8F
:105500000000C8429A993940C88200303333F33FD3
:1055100008B5D1ED007A9FED157AF0EEE77AF4EE5A
:10552000C77AF1EE10FA1CD5D1ED017AF0EEE77AE8
:10553000F4EEC77AF1EE10FA13D5022203210C48DB
:1055400006F0ACF878B10A480121FDF719FA0948CC
:1055500090F86030012B02D05C303EF04FFA002012
:1055600000E0022008BD0420FCE700BF000000347A
:10557000C8320030C8B2003010B5D1ED007AFCEE70
:10558000E77A17EE903A9CB2012C02D0022C06D09A
:105590004CB92146054886F0FBFC002010BD0448AC
:1055A00003F0EAFDF9E70420F8E700BF6CAF003034
:1055B000C83200301FB5D1ED017A0B7CFCEEE77AE2
:1055C000CDED027AD1ED007A0093FCEEE77AD1EDD1
:1055D000030A91ED020A01469DF80830CDED037AE9
:1055E0009DF80C20024811F0BBFF05B05DF804FBEC
:1055F000C832003013B513480C46C2F05DFAF0B162
:10560000D4ED017AFCEEE77ACDED017A9DF8040045
:10561000012807D002280CD088B90B4B83F8020868
:1056200002B010BD94ED020A0648C2F057FA0020FD
:10563000F6E794ED030A0348C2F090FAF7E7042076
:10564000EEE700BFBC8A0030C882003010B50A4CBB
:1056500094F8DD3FDB070CD402220521A4F5A0401D
:1056600006F01CF828B90222A4F5A040114606F065
:1056700015F8002010BD00BFC882003010B5D1ED74
:10568000007A0446FCEEE77A17EE903A13F0FF0337
:105690000FD10F4BD3F8C40F03689B6F984708B125
:1056A000002010BD0B4A2046062174F0E5FA0420C4
:1056B000F7E7012B09D1064BD3F8C40F0368DB6F62
:1056C00098470028ECD1044AEDE70220E9E700BF43
:1056D000C8820030747514088475140801F10C0335
:1056E0009FED0A7AF1EC017AF4EE677AF1EE10FAA6
:1056F0000AD6F0EEE77AF4EEC77AF1EE10FA03DCA0
:105700009942EFD1012070470020704700007A4491
:1057100030B5002305462DED028B8DB00393049325
:10572000059316F0D3FE03A916F0A0FC58B316F0AB
:10573000CDFE00F55A7306AC2D7C93E8070084E893
:105740000700DDED060A9DED070AF1EE600AB1EEF5
:10575000400A19F161F82046B0EE408A3AF0ECFDBB
:10576000089B0122DFED0A7AA8210B930C2328EE77
:10577000278A28468DED0A0ACDE9003209AA8DED67
:10578000098A71F011FE0DB0BDEC028B30BD00BF77
:10579000E02E65424029F7B505460E461ED00AD8D0
:1057A0001B290CD024290CD03146284603B0BDE873
:1057B000F04078F0A3B9A1F14203012BF4D8012401
:1057C00005E00C2170F0A2FF044618B90024204621
:1057D00003B0F0BD2846FFF79BFFF8E7262170F0E5
:1057E00095FF04460028F1D0297C10489DF098FFD1
:1057F0000F4B1F68002FEAD02621284670F086FF45
:1058000004460028E3D000230DF106023146284665
:10581000ADF8063079F0C6F80028D8D0BDF80620DB
:105820003846297C96F036FAD1E700BFA8B00030A0
:105830004CCD003038B5184C0D4694F8DD3FDB07F1
:105840000AD4D4F8E83F93F8D5303BB9012204F6E6
:1058500068401146FCF7E0FE002038BD94F9B83FDF
:105860000222002B12DA0521A4F5A04005F016FF54
:105870000028F1D095ED000A0121DFED087AD4F877
:10588000C40F20EE270A13F077F9E5E70921A4F504
:10589000A04005F003FFDFE7C88200300000C842E7
:1058A00010B5214C94F8DD3FDB070ED4D4F8E83F67
:1058B00093F8D5304BB194F9B83F002B07DA0122A9
:1058C000082104F66840FCF767FF002010BDD1ED09
:1058D000007A9FED167AF0EEE77AF4EEC77AF1EEF1
:1058E00010FA0BD502221121114805F0D7FEA0B9FC
:1058F00002220F48114605F0D1FEE6E7D4F8C40FA6
:1059000003681B6898470428DFD0D4F8C40F0368E5
:105910001B6898471428E5D1D7E740F6C41105481D
:1059200009F02CFED1E700BFC8820030000000342F
:10593000C8320030ECB7003073B58B8B05460C468F
:10594000C12B44D8BB2B0DD8202B67D02ED8113BB0
:1059500099B2052918D92146284602B0BDE8704001
:1059600079F016BBBC3B052BF5D801A151F823F00B
:10597000C15A0208CB5A020857590208575902085F
:105980004F5A02085B5A0208052BE4D801A151F8CE
:1059900023F000BFA75A02085759020857590208B6
:1059A000BB5A0208BB590208715A0208732B30D047
:1059B00006D8542B5CD0552BCDD10222092174E09E
:1059C000B22BC8D102B0BDE87040FFF76DBD4AF2FE
:1059D0001146B34258D00BD8D12B44D0B3F5967FA3
:1059E00057D0D02BB7D102B0BDE87040FFF7C4BD8F
:1059F0004AF21346B34242D04AF26866B3424DD0EF
:105A00004AF21246B342A6D102B0BDE87040FFF799
:105A100011BF02B0BDE87040FFF7FCBCD1ED007AC9
:105A2000F5EEC07AF1EE10FA54DD9FED2B7AF4EE2C
:105A3000C77AF1EE10FA4DD8FCEEE77A274ACDEDA1
:105A4000017A9DF80430A2F81A38002033E021468C
:105A500002B0BDE87040FFF74FBC214602B0BDE880
:105A60007040FFF70BBE02B0BDE87040FFF7A2BD6B
:105A70002146284602B0BDE87040FFF7A1BC02B045
:105A8000BDE87040FFF70CBF02B0BDE87040FFF703
:105A9000DDBD02B0BDE87040FFF73ABD02B0BDE821
:105AA0007040FFF7A7BD022205210D4805F0F6FD65
:105AB0000028CAD1042002B070BD02220621F4E7FA
:105AC0000221084807F012F9F2E70221054807F021
:105AD000D7F8EDE70220EEE700007F43C8820030F0
:105AE000C8320030E8B20030F6EE007A08B591ED29
:105AF000007AB4EEE77AF1EE10FA06DD0122052114
:105B00000348FCF749FE002008BD0420FCE700BF65
:105B1000308F003030B52DED028BCD7893B00C4630
:105B20002722272D4FF0000108A828BF27251BF1A9
:105B300051FD04F10C0108A82A461BF101FD424B5E
:105B4000D3F8C40F03685B6A9847002841D09DF8DA
:105B5000465068063DD400244FF07E532906049336
:105B600007940694059427D504A838F01DFCEA078D
:105B700005F006030194029403942ED4002B2ED139
:105B80000D9B01930E9B02930F9B03932F480BF0E9
:105B90008FFD9DED100A044630B3B7EE001A40F2B7
:105BA000ED40FFEE000A34F053FB234601AA04A99E
:105BB00026480BF085FD0CE0099B04A804930A9B82
:105BC00005930B9B06930C9B079338F0F3FB00287F
:105BD000CDD113B0BDEC028B30BD062BD6D0012148
:105BE0001A480BF001FDF4E7DFED190AB7EE001AD1
:105BF0004FF49E6034F02CFBF6EE000AB0EE408AC3
:105C000034F0C4F9E8B9B6EE000A124BD3F8203BE1
:105C1000B4EEC08AF1EE10FA08DD38EE400A30EE3C
:105C2000008A93ED070A28EE000ABEE730EE480A24
:105C3000D3ED087AF0EEE77A30EE000A27EEC00ADC
:105C4000B3E79FED030AB0E7C882003048B90030DF
:105C500000000000C8A200302DE9F0439DB081464D
:105C600008460EA9FEF766FD844BD3F8C40F0368FF
:105C70005B6A984750B19DF86C30012B09D0DA1F50
:105C8000022A06D901217E480BF0AEFC1DB0BDE80A
:105C9000F083BDF86840A20504F0070604F0380759
:105CA00004F4E07501D5002DF0D04FF00008CDF8D8
:105CB0001480CDF81880CDF81C803EBB9FED716A32
:105CC000083B9DED107ADDED117A012BDDED0F6AB9
:105CD00027EE067A67EEC67A66EE866A8DED067A5C
:105CE000CDED077ACDED056A04D806AA05A9664868
:105CF000FCF7CAFF9DF86C30073B022B06D86348BF
:105D0000BCF0ECFA014605A839F018FFCDF8208068
:105D1000CDF82480CDF82880F7B9DDED147A08A9F4
:105D2000129B4846F1EE677A0893139BCDED0A7AF1
:105D30000993FFF7D3FC0028A4D09FED520A08A8CE
:105D400039F030FF9DF86C30083B012B04D809AACC
:105D500008A94D48FCF798FFCDF82C80CDF830808D
:105D6000CDF83480EDB99DF86C309FED466A9DED1D
:105D7000167A083BDDED177ADDED156A27EE067A17
:105D800067EEC67A012B66EE866A8DED0C7ACDED54
:105D90000D7ACDED0B6A04D80CAA0BA93A48FCF792
:105DA00073FF14F4806233D1DFED397A9DED180A68
:105DB0009DF86C1020EE270ADFED327A08390129B0
:105DC00020EE270A8CBF0021012114F4006305BFD7
:105DD000DFED2F7ADDED190ADFED2E0A60EEA70A5E
:105DE00004BFDFED287A60EEA70AAEB9002F35D1E7
:105DF000B3FA83F3B2FA82F2029105A95B09204853
:105E0000520901930BAB009208AA0CF027F83DE76A
:105E100000219FED200AD8E77FB9B3FA83F3012070
:105E20005B090093B2FA82F30BAA5B09CDE901107A
:105E300008A913480BF0B0FD28E7002D7FF422AF2E
:105E40000120B3FA83F3B2FA82F25B095209CDE979
:105E500000100BA90A480BF035FD17E7002D3FF4A1
:105E600011AFB3FA83F3B2FA82F205485B09520923
:105E7000CDE9001605A90BF00DFE07E7C88200303A
:105E800048B900300000C842C8320030C0AD003010
:105E9000E02E6542000000002DE9F047A2B08046E8
:105EA000084614A9FEF746FC7E4BD3F8C40F0368DE
:105EB0005B6A9847C0B1BDF88040A30504F00709AC
:105EC00004F4E07700D57FB10CAE30461DF0AAF99E
:105ED000B9F1000F29D1DDE9150135F0D3FC30B956
:105EE000012171480BF080FB22B0BDE8F08709AAC0
:105EF0009DF88410404677F055FA0028F0D0DDED8B
:105F0000177A10AD9FED697A099B284667EE877A6C
:105F10000093FDEEE77ADDE9151217EE903A1DF0D9
:105F2000A1F995E80F0086E80F00002514F0380A63
:105F300006950795089514D1DDED1A7A06A9189BE8
:105F40004046F1EE677A0693199BCDED087A0793E8
:105F5000FFF7C4FB0028C3D09FED540A06A839F010
:105F600021FE09950A950B959FB99FED506A9DED0D
:105F70001C7ADDED1D7ADDED1B6A27EE067A67EEF1
:105F8000C67A66EE866A8DED0A7ACDED0B7ACDED96
:105F9000096A14F4806805BFDFED457A9DED1E0A9D
:105FA0009FED440A20EE270A04BFDFED407A20EE81
:105FB000270A14F4006405BFDFED3D7ADDED1F0A0A
:105FC000DFED3C0A60EEA70A04BFDFED387A60EE31
:105FD000A70AB9F1000F31D1BAF1000F52D1304602
:105FE000CDED050A8DED040A1DF04CF903289DED59
:105FF000040ADDED050A3FF473AF10A93046CDED7C
:10600000050A8DED040A1095119512951DF000FBFF
:1060100000283FF465AFB4FA84F4B8FA88F3DDEDF4
:10602000050A06AA64099DED040A5B0910A9CDF8CA
:1060300004A000941C480BF087FF55E7BAF1000F4D
:106040000FD10123B4FA84F409AA06A964091648F9
:10605000CDE901A3B8FA88F300945B090BF09CFC2E
:1060600042E7002F7FF43CAF0123B8FA88F209A978
:106070000D485209CDE90073B4FA84F35B090BF0C3
:1060800021FC31E7002F3FF42BAFB4FA84F3B8FAC8
:1060900088F23146CDF800905B09034852090BF0B5
:1060A000D9FD21E7C882003048B900300000C8425D
:1060B000E02E6542000000004B7ACA7A10B48C7A58
:1060C00043EA042343EA0243542B07D0562B09D05A
:1060D000522B0BD15DF8044BFFF71CBD5DF8044B50
:1060E000FFF7BABD5DF8044BFFF7D6BE5DF8044B71
:1060F00078F060B82DE9F04300F5A046044600278B
:1061000004F5E0492DED028BD6F8C40F91B0DFED18
:106110004B8A03685B699847002840F08A80D9F869
:106120001C3B93EDE07BB7EEC77BD3EDE77AFDEE4A
:10613000E77A27EE288A17EE903A1DB204F5B748A1
:1061400001A908F17008404612F054F818B96DF032
:106150009DFC3B4B01933722002102A81BF13AFA28
:10616000A3238DF8083095238DF80930C6F03CFE46
:10617000D9F8143BCDF80B00D6F8E80FD3F8DC20A3
:10618000D3F8E0304430CDF80F10CDF81320CDF81F
:1061900017306FF0C1F90346B7EE001ADFED290A98
:1061A0009F2093ED000A34F053F8D6F8E80F10EE74
:1061B000103A04F5F546CDF81B30783603681B69B4
:1061C000984710EE103A3046CDF81F3018EE103ACE
:1061D000CDF82330BCF086F820EE280A404610EEB9
:1061E000103ACDF82730D9F8C43ACDF82B30019BBE
:1061F000CDF82F3012F020F810EE103A3046CDF8DE
:106200003770CDF83330ADF83B50BCF077F8BDEEC9
:10621000C00A04F5C250372202A9083010EE103A25
:10622000ADF83D306CF074FD11B0BDEC028BBDE8F3
:10623000F083002508EE107A80E700BF0AD7233CE0
:106240002292CA7F0000000010B500F5E044D4F8A7
:10625000140BB2F061FDD4F81C1BD4F8140BBDE88C
:106260001040B2F0BFBD000070B54FF4805105463C
:1062700012F032F900284FD005F5E04605F5C2547A
:10628000D6F8140B083403689B689847692100F11D
:10629000A00220466CF086FBD6F8140B0368DB687E
:1062A00098476A2100F1A00220466CF07BFBD6F8EB
:1062B000140B03681B6998476B2100F1A00220466C
:1062C0006CF070FBD6F81C2B6C21204602F52D7269
:1062D0006CF068FB2021284612F0FEF8E0B105F5CD
:1062E000A043D3F8C40F03681B69984778B1D6F868
:1062F0001C2B20466E2190326CF054FBD6F81C2BE0
:1063000020466F21BC32BDE870406CF04BBB284684
:106310000CF0C2FB0028EAD170BD000008B516F0F1
:10632000D5F8BDE8084015F0C5BD00007FB50E46A4
:106330004FF6FF710446154612F0CEF8E8B1102270
:10634000002168461BF146F9A3238DF80030952300
:106350008DF8013003238DF80230C6F045FDCDF8ED
:10636000030004F5C250CDF807101022694608302A
:106370008DF80B6003956CF04BFD04B070BD000010
:106380007FB50E464FF6FF710446154612F0A4F88D
:10639000E8B11022002168461BF11CF9A3238DF8F7
:1063A000003095238DF8013004238DF80230C6F0BB
:1063B0001BFDCDF8030004F5C250CDF807101022E4
:1063C000694608308DF80B6003956CF021FD04B030
:1063D00070BD000030B52DED048B87B004460D462E
:1063E000182200216846B0EE409AF0EE608AB0EEC6
:1063F000418A1BF1EFF8A3238DF8003095238DF827
:10640000013006238DF80230C6F0EEFCCDF8030013
:1064100004F5C250CDF807101822694608308DF8EF
:106420000B508DED039ACDED048A8DED058A6CF04D
:106430006FFC07B0BDEC048B30BD000010B54FF40D
:106440008011044612F048F830B104F50650BDE85A
:106450001040183014F0B8B810BD00002DE9F04F0E
:106460002DED028B8DB080462F2200216846F0EE84
:10647000408AB0EE608A11EE10BA11EE90AA12EEC8
:10648000109A12EE907A13EE106A13EE905A14EEF0
:10649000104A1BF19FF8A3238DF8003095238DF847
:1064A000013009238DF80230C6F09EFC18EE903AB8
:1064B000CDF8030008F5C250CDF80710CDF80B3029
:1064C0002F2218EE103A69460830CDF813B0CDF8F7
:1064D0000F30CDF817A0CDF81B90CDF81F70CDF878
:1064E0002360CDF82750CDF82B406CF011FC0DB097
:1064F000BDEC028BBDE8F08F30B52DED088B8BB075
:1065000004460D46282200216846B0EE40BAF0EE5F
:1065100060AAB0EE41AAF0EE619AB0EE429AF0EEB7
:10652000628AB0EE438A1BF155F8A3238DF8003040
:1065300095238DF801300A238DF80230C6F054FC03
:10654000CDF8030004F5C250CDF8071028226946A3
:1065500008308DF80B508DED03BACDED04AA8DED0A
:1065600005AACDED069A8DED079ACDED088A8DED41
:10657000098A6CF0CDFB0BB0BDEC088B30BD000080
:106580002DE9F0438FB0144605468946312200219B
:1065900001A89846DDE916761BF11CF8A3238DF8B7
:1065A000043095238DF8053008238DF80630C6F0A9
:1065B0001BFC23683122CDF8070005F5C250049377
:1065C00063680830CDF80B1001A90593A3688DF816
:1065D0000F9006933B688DF81C80CDF81D307B68CA
:1065E000CDF82130BB68CDF825303368CDF829309F
:1065F0007368CDF82D30B368CDF831306CF088FB7E
:106600000FB0BDE8F083000070B52DED068B8CB0A7
:10661000144605460E462C22002101A8B0EE409AF1
:10662000F0EE608AB0EE418AB0EE61AAF0EE429AD6
:106630001AF1D0FFA3238DF8043095238DF805308F
:106640000B238DF80630C6F0CFFBDFED1A7A2C2233
:1066500094ED007ACDF8070005F5C25027EE277AB1
:10666000CDF80B1029EE279A01A968EEA78A083009
:106670008DED077A28EE278A94ED017A8DF80F6068
:1066800027EE277A8DED049ACDED058A8DED068AE9
:106690008DED087A94ED027A8DED0AAA67EE277ADD
:1066A000CDED0B9ACDED097A6CF032FB0CB0BDEC60
:1066B000068B70BDE02E6542AE20704730B50446B3
:1066C00089B0144B1E2204F5C2556946D3F8E80F71
:1066D0000835BDF065FA6A460F4928466CF0B4FCEF
:1066E00004F5A043D3F8C40F03681B68984704F56A
:1066F00040530146284693F8EC2B6CF0C9FC04F596
:106700000650183016F04AF904F5907026F05CF93E
:1067100009B030BDC88200307D471708F8B5464B38
:106720000446464A483040F8443C002340F8142CC4
:106730004FF0804240F8343C40F6683540F8303C39
:1067400040F6686640F82C3C40F80C3C3C4B40F866
:10675000102C40F8083C3B4B3B4F40F8043CAFF05A
:106760002FFC04F582708BF0ADF804F52B6079F006
:10677000C3F9364BC4F8B03A601979F027FC675179
:106780003035B542F8D104F6686004F580567BF0E8
:10679000E3FA04F5C75000212D4D1430C0F0A6FCDB
:1067A00004F5CD500430C1F077F904F5CE50C6F8A9
:1067B000C4590830C1F0F4FEA5F5E76304F5D350E1
:1067C000C6F8583A043091F0E7FCA5F50C7304F5CF
:1067D000E150D435C6F81C3C9FED1E1A0C30DFED9D
:1067E0001E0A9FED1E0AC6F8285CB3F057FA9FED0B
:1067F000191A04F5E2509FED1A0AF0EE410A04302E
:10680000B3F04CFA9FED131A04F5E2509FED140A11
:10681000F0EE410A1C30B3F041FA04F5E5500C30BB
:10682000B8F0C0F820460F4962F078F920460E49CA
:1068300062F074F92046F8BD904700300000C8416E
:106840000AD7233C0000E040F8C714080CC814081D
:10685000A0BD0030000000009A99993E0000B443AA
:1068600000804A4394BA140884BD140870B5ADF58D
:106870000E7D4B4DD0224B4906465AA81AF160FEB8
:106880000EAC0FCD0FC40FCD0FC40FCD0FC495E8C4
:106890000F0084E80F0000245AABB7EE000A002175
:1068A0001819103461F012FCD02CF5D13E4B02AC1B
:1068B0000FCB84E80F0001A9204661F0BBFB90B12B
:1068C0009DF90430F0EE007ADFED386AB7EE000A89
:1068D00007EE103AE068B8EEC77AE7EE267A80EE67
:1068E000270A62F0AFFC00240EAB00211819103407
:1068F000B7EE000A61F0EAFB402CF5D190222C495A
:1069000036A81AF11DFE0022092136A861F088FC84
:1069100096F9846BD6B9274D1EAC0FCD0FC40FCDA1
:106920000FC40FCD0FC495E80F0084E80F00324666
:1069300004211EA861F074FC9FED1F0A1F4862F03D
:1069400081FCB7EE000A1E4862F07CFC1D4C06ADCF
:106950009FED1D0A0FCC0FC594E80F0085E80F00CE
:10696000002106A861F0B2FB00219FED170A28461E
:1069700061F0ACFB04F11001002460221EA81AF1A2
:10698000DFFD1EABB7EE000A00211819103461F0CC
:106990009DFB602CF5D17AF03BFF0DF50E7D70BDAF
:1069A000185C1408485B1408585C1408CDCCCC3D26
:1069B000685C1408F85C1408000000007CB9140836
:1069C0008BB91408385D14080000344210B5B4B017
:1069D0000024D022074968461AF1B2FD0DEB0400ED
:1069E0001034B7EE000A002161F070FBD02CF5D115
:1069F00034B010BDB85D14082DE9F04790B01D20EB
:106A00000DF106017AF0F6FF002800F09E809DF857
:106A100006301121604A0BA80133DBB28DF8063035
:106A2000C5F096FB00220DF107010BA861F0A6F856
:106A30009DF80630594A112105460BA8C5F088FB80
:106A400000220DF107010BA861F098F89DF80630BF
:106A5000534A112106460BA8C5F07AFB00220DF11E
:106A600007010BA861F08AF89DF806304D4A112104
:106A700003F03F0307460BA8C5F06AFB00220DF1A7
:106A800007010BA861F07AF88046002D5DD0002E3A
:106A90005BD0002F59D0002857D0284661F068FA03
:106AA000002852D1304661F063FA00284DD13846B3
:106AB00061F05EFA002848D1404661F059FA00289A
:106AC00043D1394C0DF10C0C0DF11C0994E80F0069
:106AD00010348CE80F0094E80F0089E80F0002A939
:106AE000604661F0A7FA98B3BDF8084002A948468D
:106AF00061F0A0FA00284AD0BDF8083054BB23B397
:106B000040F2E2449C420FFA84FA0FFA83F927D844
:106B10000DF10A013046ADF80A9063F059F80DF115
:106B20000A012846ADF80AA063F052F80DF10A01F7
:106B30003846ADF80AA063F04BF800230DF10A01C6
:106B40004046ADF80A3063F05DF810B0BDE8F0875C
:106B50000024CBE740F2D662002B08BF1346D1E7F2
:106B60000DF10A013046ADF80AA063F031F80DF1DD
:106B70000A012846ADF80A9063F02AF80DF10A01DF
:106B80003846ADF80A9063F023F80123D6E7002CCD
:106B9000DBD040F2D663B5E79CB91408A8B9140855
:106BA000B4B91408C1B91408885E140837B500F5E3
:106BB00077510446782201251C316AF003F900223E
:106BC0000C21274861F02CFB2046FFF715FF04F548
:106BD0007750B7EE000A00220221303061F0A8FBA6
:106BE00004F56851002345202C311E4A009561F0C0
:106BF0001BFB1D490B68D8070BD404F559521B4BDE
:106C00000D6028321A6004F56D52DA6004F5C8523E
:106C10009A6104F57950032214490125103061F07E
:106C200055FB04F5C2510023114A0831FD2000959F
:106C300061F0FAFA0F4B01210F481A68D2075FBFC3
:106C40000D4A04F503541D60146061F05BFB62F0B3
:106C500057F90A4A138843F00103138003B030BD8B
:106C6000D4B91408707616083CBF0030C425003033
:106C70000CAD150840BF0030E8250030C8C1003019
:106C80000F299DBF302303FB0100B830002070475F
:106C9000014B93F9230E7047C8620030024B93F802
:106CA000DD0F00F001007047C8820030044BB3F8DC
:106CB000E83DDB075ABF0069C0F340100020704771
:106CC000C8620030014BD3F8500B7047C8820030C7
:106CD00008B503689B68984730B9044B93F9DC0FFB
:106CE000B0FA80F0400908BD0020FCE7C8820030FF
:106CF00038B50C1E2EDB184DE3B295F85C2B9A428A
:106D000028D3D5F8583B0122A5F5A040195D04F021
:106D1000C5FCF8B179F08CF803217AF0EDFAC8B926
:106D200079F086F80D217AF0E7FA98B9A5F50052C6
:106D3000A5F5A04092F9083EE340DB0756BF92F963
:106D4000221E0221E140BDE8384058BF01F0010198
:106D5000FBF72CBE38BD00BFC8820030022910B539
:106D6000044606D1014635220948BDE8104004F02A
:106D700095BC084BD3F8C40F03681B68984784423E
:106D800005D179F055F8BDE8104078F0CBBF10BDC3
:106D9000C8320030C882003029B1022907D1044B23
:106DA000C3F8BC1F7047024B0122C3F8BC2F7047C9
:106DB000C882003031B1022907D1044B012283F887
:106DC000C02F7047014B83F8C01F7047C882003046
:106DD00000F5A043DFED186A9FED187A012110B588
:106DE000D3F8482B0446D3F8443B00F50650B2F9DB
:106DF0000820B3F90830183007EE902AF8EEE77A49
:106E0000C7EEA60A07EE903AF8EEE77A87EEA60AF2
:106E100060EE870A20EE070A15F0FAFB6CF036FEEA
:106E200026216CF06FFD04F5BA40054A062150306A
:106E3000BDE810406FF008BA0000C84235FA8E3C39
:106E4000D0C5140800F5E042002300F5BA40062141
:106E500082F8303B024A50301372024A6FF0F4B9A4
:106E60002DC10030DCC51408F8B500F5E045044636
:106E700095F8301B002955D02B4B2C4AD3F8C40F62
:106E8000904204D1D3F8E83F93F8D53023B9204697
:106E9000BDE8F840FFF7D6BF254E012004F5A0431A
:106EA00095F8317B307293F9B82FC7BB002A39DBD4
:106EB00085F8310B0139DFED1F6A9FED1F7A04F56C
:106EC0000650C9B2183085F8301BB1FA81F1D3F8F9
:106ED000482BD3F8443B4909B2F90820B3F90830EC
:106EE00007EE902AF8EEE77AC7EEA60A07EE903A88
:106EF000F8EEE77A87EEA60A60EE870A20EE070A28
:106F000015F086FB95F8303B63B904F5BA4033724F
:106F10000A4A06215030BDE8F8406FF095B9002AC2
:106F2000C8DAB4E7F8BD00BFC882003034BB003017
:106F30002DC1003000007A4535FA8E3CF0C51408AA
:106F40006D2900F3E380012901DC79F0B5BF8B1EC8
:106F50006B2BFAD80FF2040C5CF823F06B7102086B
:106F6000657102086B7102086B7102084B6F0208B1
:106F70006B7102084B6F02084B6F020865710208C3
:106F80004B6F02086B710208657102086571020897
:106F90004B6F02086B7102086B7102086B7102087B
:106FA0004B6F02084B6F0208657102086B71020893
:106FB000657102084B6F020865710208657102086D
:106FC0004B6F02084B6F02084B6F02084B6F0208B1
:106FD0004B6F0208657102086B7102084B6F020863
:106FE0004B6F02084B6F02086B7102084B6F02086F
:106FF000657102084B6F02084B6F02086B71020843
:1070000065710208657102086B7102084B6F020816
:107010006B7102086B7102086B7102084B6F0208FA
:107020004B6F02086B7102084B6F02084B6F02082E
:107030006B7102086B7102086B7102084B6F0208DA
:107040004B6F02086B7102086B7102084B6F0208EC
:107050004B6F02084B6F02084B6F02084B6F020820
:107060004B6F02086B7102086B7102086B710208AA
:107070006B7102086B7102086B7102084B6F02089A
:1070800065710208657102084B6F02084B6F0208B8
:107090004B6F02084B6F02084B6F02084B6F0208E0
:1070A0006B710208657102084B6F02084B6F020892
:1070B0004B6F02084B6F02084B6F02084B6F0208C0
:1070C0004B6F02084B6F02084B6F02084B6F0208B0
:1070D0004B6F02084B6F02084B6F02084B6F0208A0
:1070E0006B7102084B6F02084B6F02084B6F02086E
:1070F0004B6F02084B6F02084B6F02084B6F020880
:107100004B6F02084B6F020865710208A12921DC50
:1071100096297FF71AAFA1F197030A2B3FF615AF17
:107120000FF2040C5CF823F06B7102086B7102081B
:107130004B6F02086B7102084B6F02084B6F02081D
:107140004B6F02084B6F02086571020865710208F7
:107150006B710208B42908D0DB2903D0B2297FF46F
:10716000F4AE7047002379F06FBE7047632970B5A5
:1071700014468AB000F3D280012905DC22460AB009
:10718000BDE8704079F06ABB8B1E612BF6D801A276
:1071900052F823F097730208AB730208CB7302080E
:1071A000D57302087D710208057402087D7102081A
:1071B0007D710208B57402087D7102087D710208B4
:1071C000B9730208D97402087D710208AF7402080D
:1071D00015750208257502087D7102087D71020887
:1071E0003D7502084B750208597502087D71020849
:1071F0007F750208917502087D7102087D71020891
:107200007D7102087D7102087D710208A375020874
:10721000BD7502087D7102087D7102087D7102084A
:10722000C37502087D710208C97502087D710208E4
:107230007D710208E37502087D710208E975020894
:107240009B7302087D7102087D7102087D7102083E
:107250007D7102087D7102087D7102088F76020837
:107260007D7102087D7102082B75020831750208D4
:10727000377502087D7102087D71020809760208DF
:10728000457602087D7102087D7102087D71020851
:107290007D7102087D7102087D7102087D76020809
:1072A0008376020889760208957602089B760208A2
:1072B000A17602087D710208E5760208A776020829
:1072C0007D7102087D7102087D7102087D710208DE
:1072D0007D7102087D71020819770208377702086C
:1072E0007D7102087D7102087D7102087D710208BE
:1072F0007D7102087D7102087D7102087D710208AE
:107300007D7102087D7102087D7102087D7102089D
:107310007D7102087D7102084D770208A0291FDCEB
:1073200096297FF72BAFA1F19703092B3FF626AFE4
:1073300001A252F823F000BF5377020859770208E0
:107340007D7102086D7702087D7102087D71020867
:107350007D7102087D710208457702089177020865
:10736000B42900F0DA80DB2917D0B2297FF406AF08
:10737000002A00F0CA81022A0FD1A54BD3F8C40F0E
:1073800003689B6F984740B976F070FAA14A0421D0
:107390006EF05AFF01E0022C01D001242FE03522CB
:1073A0000E219D4804F07AF9F7E7211E18BF01214C
:1073B0009948FBF7FBFAF0E7012C04D0022C14BF2C
:1073C00000210221F4E72146F2E721460620FFF7DB
:1073D000C5FCE2E7022CE0D18D4DD5F8C40F03685F
:1073E000DB6A984704460028D7D0D5F84C3BB3F960
:1073F0000830002BD1D1A5F5A040FFF7E9FC2046CD
:107400000AB070BD022CC8D1814D844BD5F8C42F71
:107410009A42C2D0D5F8E83F93F8D530002BBCD0C3
:1074200005F54054B4F990302BB9D5F84C3BB3F97D
:107430000830002BB1D005AE1C22002103A81AF1A0
:10744000C9F830461BF0EEFEB4F99030744C93B995
:10745000162303A97348ADF80E30D4F8EC3A642B28
:10746000B8BF6423069339F099FD20B16CF00EFB90
:1074700027216CF047FA04F6E8230FCB86E80F00CB
:10748000D5F84C3B03A96748B3F90830002BCCBFB3
:1074900010231523ADF80E3039F080FD00283FF49D
:1074A0007CAF6CF0F3FA27216CF02CFA75E72146DB
:1074B00003208CE7022C564D03D0002385F8603B57
:1074C0006BE71921584863F045F804460028F4D0CA
:1074D000012385F8603B92E7012C0BD0022C12D0DF
:1074E000002C7FF45AAF514B83F84C4E6CF0CEFA1F
:1074F0002B21D9E74D4B83F84C4E6CF0C7FA2C2169
:107500006CF000FA7BE7494B83F84C4E6CF0BEFA06
:107510002D21C9E721460F2059E711464448C4F000
:1075200023F83AE72146092051E7214604204EE797
:10753000214605204BE72146172048E7A01E41427F
:1075400041413C4884F024FD27E7022C7FF425AF1D
:10755000314801F011FE20E7012C06D0022C09D0A1
:10756000002C7FF41AAF2146EBE72146314884F026
:107570000FFD44E701212F4884F00AFDE8E7A21E31
:10758000274B5442D3F8143B544183F8204004E77E
:10759000A31E59425941224BD3F8140BB3F0AAFC55
:1075A000FBE6013C1A4B012C93F8BA2F8CBF002448
:1075B000012464F3041283F8BA2FEEE62146112069
:1075C00005E72146122002E7012234B1022C7FF4A4
:1075D000E4AE194B83F84827DFE6174B83F848479A
:1075E000DBE621461520F2E6012C08D9022C7FF4B7
:1075F000D4AE9FED120A1248C0F0B0FACDE6044BAB
:10760000002283F80228C8E621461820DFE600BFE2
:10761000C88200302BC61408C8320030E8B20030EF
:10762000C8A2003024B3003060480030C862003087
:1076300068B600306CAF0030C8B200300000000007
:10764000BC8A0030594BD3F8C40F594B98427FF491
:10765000A4AE01900FF050FB012C019808D0022C31
:107660000AD0002C7FF499AE21460FF0F5FB94E68A
:1076700000210FF059FBC2E60121F6E72146002068
:10768000A5E621461020A2E6214602209FE62146DB
:1076900001209CE62146162099E62146072096E621
:1076A00021460B2093E6022C424B0ED1012483F895
:1076B000804F6CF0EBF94A216CF024F976F0D6F8A3
:1076C0003D4A06216EF0C0FD99E6002283F8802F26
:1076D0006CF0DCF94B216CF015F976F0C7F8374AFD
:1076E000062155E6012C09D0022C0CD0002C7FF489
:1076F00054AE0121324810F0B5FD4EE6002130486D
:1077000010F0B0FD7BE62146F4E7284BD3F8C40F18
:107710000368DB6F984740E6244BD3F8C40F244B33
:1077200098427FF43AAE022C02D10FF09FFC34E66F
:107730000FF086FB31E62146FFF72EFB214804F0CF
:10774000F3FC2AE62146FFF735FB26E621461B20FF
:107750003DE621461C203AE6022C7FF41EAE1A4874
:10776000FCF7FAF976F082F8184AB9E7214678F082
:10777000D5FE1748AFF048FE044600283FF40DAE92
:107780000A4A92F8BB3F43F0020382F8BB3F36E659
:10779000012234B1022C7FF400AE044B83F8282B75
:1077A000FBE5024B83F8284BF7E500BFC8820030A9
:1077B00074BE0030C8A2003008C6140819C61408E8
:1077C000B88E00306CB20030C832003044C61408A5
:1077D000308F003010B504460448BAF081FD04F142
:1077E0000801BDE8104033F0CBBF00BFC0AD003092
:1077F00038B5044612482DED028BBAF077FD0546E8
:1078000037F06CFD0F48B0EE408A10F0FFFD90B1EC
:10781000DFED0D7AB4EEE78AF1EE10FA0BDDD5ED6F
:10782000000A95ED010A16F1F7FFDFED087A20EE68
:10783000270A84ED080A94ED080ABDEC028B38BDD6
:10784000C0AD0030C832003000401C46E02E65421A
:10785000074B93F9090E022805D0032806D00038FB
:1078600018BF0120704781F0010070470420704765
:10787000C862003003688B4214D00429C0E90013A9
:1078800002D007290CD07047074B9FED087AD3ED43
:10789000E67AF8EEE77A67EE877AC0ED087A704705
:1078A00000238362704700BFC85200300AD7233CD0
:1078B000024608B5FFF7CCFF01461046BDE8084078
:1078C000FFF7D8BF70B5044616460D462DED048B64
:1078D000F0EE408A9FED339AB0EE608ADFED329A87
:1078E000C5F07AFAE0615EB3236833B92F4BD3ED6C
:1078F000E67AF8EEE77AC4ED097A68EE898A002D17
:10790000B7EE000AFFEE007A20FE270A68EE808AB2
:10791000C4ED058AB4EEE98A254BD3F8140BF1EED9
:1079200010FA30DAB2F0A0FA20EE090A84ED060A65
:1079300020460321BDEC048BBDE87040FFF79ABFE1
:1079400094ED090A98EE890A32F01AFC002D84EDB4
:10795000050A0BDAB4EEE90AF1EE10FADADBDFED34
:10796000157A30EE670A84ED050AD3E7D2D0DFED51
:10797000127AB4EEE70AF1EE10FACBD8DFED0D7A09
:1079800030EE270AEFE7B2F06FFAB4EE480AF1EEF4
:1079900010FA48BFB0EE408A28EE098A84ED068AC4
:1079A000C6E700BF0000C84200000034C8520030E3
:1079B000C8A2003000A00C47000000B410B52DEDA7
:1079C000028BF0EE408A0446B0EE608AC5F004FAFD
:1079D000DFED090A0621E061204668EEA08A68EE24
:1079E000200AC4ED098AC4ED0A0ABDEC028BBDE889
:1079F0001040FFF73FBF00BF0000C84210B504466B
:107A00002DED028BB0EE408AC5F0E6F994ED090A3F
:107A1000DFED097AE061A8EE270A32F09BFB002334
:107A2000204684ED090AA3620621BDEC028BBDE865
:107A30001040FFF71FBF00BF0000C84270B54B6881
:107A400006460C46144D73B98B6863B9C96851B9C1
:107A50001248FFF72DFF95F82D1C05F6B430BDE850
:107A600070407BF0D7BB95F82D1C0D487BF032FAA7
:107A700048B906F1080120461BF0CAFD18B10221E1
:107A80000648FFF7F7FE224695F82D1C0448BDE88E
:107A900070407BF0B3BB00BFC8A2003044BF0030D1
:107AA0007CAE0030072108B5FFF7E4FE80ED0A0A3E
:107AB00008BD000008B50368032B21D1D0ED057A7D
:107AC0009FED117AF0EEE77AF4EEC77AF1EE10FA54
:107AD00018D50E4B90ED090AD3EDE67AF8EEE77A69
:107AE00037EEC00A32F04CFBB0EEC00ADFED087A88
:107AF000B4EEE70AF1EE10FA94BF0120002008BDB1
:107B00000120FCE70020FAE700000034C8520030F2
:107B10000000484330B5036885B00446023B082B9B
:107B20006DD8DFE803F0050D30374B613F61610030
:107B3000FFF750FE84ED090A94ED090A05B030BD47
:107B4000C5F04AF9E369DFED310AC31AE06194ED4B
:107B5000050AF12007EE903AF8EE677A67EEA07A10
:107B6000D4ED060A20EEA71A67EEE00A32F070FBA9
:107B7000D4ED057A77EEC07AC4ED057AD4ED097AB2
:107B800037EE800AD6E7FFF733FEDFED217A20EEED
:107B9000270ACFE71F4BD3ED047AF8EEE77AC0ED62
:107BA000097AC9E71C4DD5F8280BB8F005FA00286A
:107BB000C2D0D5F8283B1B6C6362BDE7C5F00CF959
:107BC000E3699FED127AC31AD4ED0A6AE06107EE09
:107BD000903AF8EE677A67EE877A94ED097AA6EE26
:107BE000A77A84ED097AA7E70B4B9FED0C0AD3F82F
:107BF000140B6C3037F082FF84ED091A9CE7064BBA
:107C0000D3F81C3BD3F85033D6E700BF6F12833A4A
:107C10000000C842C8920030C8A200309F0CB34593
:107C20000368092B08D8DFE803F0050A05050505F8
:107C3000070705100023836290ED0A0A7047044B82
:107C4000D3F81C3BD3F85433F5E7C36AF3E700BF1E
:107C5000C8A20030F0B5304D04460E46D5F8C40F2A
:107C60002DED028B036889B0D3F880309847002847
:107C70003FD005F50057D5F8C40F03F06FFB08EEB1
:107C8000100AD7F81C3BD7F8140BD3EDD28A03683F
:107C9000D3F898309847D7F81C3BD5F8C40F78EE46
:107CA000C00A93EDD31A0368CDED050A9B6C8DEDE8
:107CB000041A98470390D5F8C40F0268D26C904715
:107CC000B8EEC88A9FED150A3246009007A928EE43
:107CD000000A039B9DED041A05F6FC20DDED050A64
:107CE000B6F078FE48B10A212046FFF7C3FD079B96
:107CF000A36209B0BDEC028BF0BD23680A2BF8D15A
:107D0000002361682046A36211B9FFF7D1FDF0E7B7
:107D1000FFF7B0FDEDE700BFC88200300AD7233C73
:107D2000F8B50023264F04460D46CB6297F8DD3F99
:107D3000244E13F0010F37D1D7F8C40F03685B6FDF
:107D4000984788B3D7F8C40F03F068FE85ED0B0A97
:107D5000B0EEC00ADFED1C7AB4EEE70AF1EE10FADD
:107D600003D409213046FFF785FDD5ED0B7A28466F
:107D7000FDEEE77A17EE903A19B2FFF76BFF114864
:107D8000FFF7C8FE0F4884ED000AFFF749FF33688C
:107D900084ED010A0A2B0FD8DFE803F00C10101055
:107DA0001010100C100C0C003368092BDDD10021D1
:107DB0000448D8E70223A3602046F8BD0123FAE770
:107DC000C882003044BF003000000034034B012261
:107DD0001A6000229A60DA601A61704744BF00306E
:107DE00013B5044601A910F06FF904F5E04320B97A
:107DF000012283F85D2C02B010BD03F54562DDED74
:107E0000017ADFED086AB8EEE77AD2ED007A67EE24
:107E1000A67AB4EEE77AF1EE10FA54BF01220022FE
:107E2000E7E700BF0000C84210B5044600F5FB407C
:107E300060309BF077FE04F5FE40BDE81040103046
:107E4000BEF044BD08B50F22084803F027FC60B916
:107E50000F220621054803F021FC30B90F22092129
:107E60000248BDE8084003F019BC08BDC832003024
:107E700070B5154E04460D4696F8DD3FDA0622D55C
:107E80006FF3041386F8DD3FA6F500566BF0FEFD98
:107E9000002214216BF056FD96F8EC3B0E2B12D10C
:107EA000022D0AD0032D0AD0012D0CD194F85410C4
:107EB0002046BDE87040FFF7C5BF0621F8E794F8FB
:107EC00054100329F4D070BDC882003010B50E4C98
:107ED00049B9D4F8C40F03681B689847A0F113038D
:107EE0005842584110BDD4F8C40F03681B68984726
:107EF0001328EED00E221321A4F5A04003F0CEFBF0
:107F00000028E6D1EEE700BFC882003030B50D464C
:107F100089B01146FFF7DAFF0446F0B104A81BF060
:107F200081F914F0D3FA04A913F0E4FF28B1286909
:107F3000059B8342D4BF002001209FED127A124B93
:107F40008DED017AD3F8202B8DED027A40B1D36903
:107F5000039301A90D4807F01DFA204609B030BD72
:107F6000D2ED087AA3F58041D3F8EC2AF0EEE77A57
:107F7000D1F8F03D9A42F1EE677A67FE877ACDED4F
:107F8000037AE6E700000000C8A200302CBC0030F5
:107F9000F0B50F4685B011460646FFF797FF044639
:107FA00058B1002501AA394630460195029503953E
:107FB000BEF098FD044618B90024204605B0F0BD77
:107FC000DDED017A9FED177AF0EEE77A0395F4EE96
:107FD000C77AF1EE10FA08D5DDED027AF0EEE77A15
:107FE000F4EEC77AF1EE10FAE6D401A838F0A4F95D
:107FF00001A837F0EBFD0C4B9DED017A01A9D3F8F8
:10800000203BDDED027AD3ED066A084827EE267A9A
:1080100067EEA67A8DED017ACDED027A07F0BAF916
:10802000CBE700BF00000034C8A200302CBC0030F9
:1080300070B50E46114605462DED028B84B0FFF754
:1080400045FF044680B39FED238A01AA31462846A6
:108050008DED018A8DED028A8DED038ABEF042FD21
:10806000044608B31C4B9DED017AD3F8202BDDEDBF
:10807000027AD2ED066A27EE267A67EEA67A8DEDB1
:10808000017A9DED037ACDED027AB4EEC87AF1EE75
:1080900010FA0EDDD2ED077A67EE877A01A90F4854
:1080A000CDED037A07F076F9204604B0BDEC028BE3
:1080B00070BDD2ED087AA3F58041D3F8EC2AF0EE3A
:1080C000E77AD1F8F03D9A4267EE877A67FE887AC0
:1080D000E4E700BF00000000C8A200302CBC003064
:1080E0002DE9F0413D4F14460646884697F8DD3F9E
:1080F000DA0616D4D7F8C40F43F01003012587F829
:10810000DD3F03681B68984786F85400D7F8C40F12
:1081100003681B689847092805D100242046BDE85C
:10812000F0810025F2E7D7F8C40F03681B68984771
:108130001228F2D0D7F8C40F03681B6898470E289E
:10814000EBD0012C12D8062C38D801A353F824F018
:108150001D810208BD810208AF810208C3810208A7
:10816000CF81020885810208A58102081C4801F020
:1081700061FE0028E7D001220A211A48FAF70CFB19
:1081800000241BE0002DC9D00E220621144803F064
:1081900085FA00B900246BF079FC224614216BF0BB
:1081A000D1FBBBE7002DB9D00E220521EEE72A4610
:1081B00041463046FFF7AAFE0028E1D0002DADD0A1
:1081C000E9E72A4641463046FFF7E2FEF4E72A4651
:1081D00041463046FFF72CFFEEE700BFC882003073
:1081E000C8320030308F003000F540532DE9F04F99
:1081F00000F50659054600F5E04409F118092DED92
:10820000068B93F95A3E8BB043B100F5A047D7F8DF
:10821000E83F93F8D580B8F1000F0FD10021A4F802
:10822000741F484614F0ECFB94F8751F48460BB0D9
:10823000BDEC068BBDE8F04F14F0ECBBC4F0CCFDF8
:108240008346D4F81C0B07AE9FED968A90EDE4AA06
:10825000B4F0A8FC002800F0CD80D4F81C3B03F556
:10826000657393E8070086E8070030468DED098ABC
:1082700038F062F8B0EE409A05F5F54A284610F05D
:10828000C5F80AF1780A002800F0B7805046BAF025
:108290002DF807C886E8070030468DED098A38F0CA
:1082A0004BF8F0EE409AD7F8C40F03681B68984764
:1082B000122840F0AB80002384F8743FD7F8C40F35
:1082C00003685B69984728B1D7F84C3BB3F908308D
:1082D000002B0CDC97F9B83F002B08DA5046C4F8A5
:1082E00078BFB9F0FFFF04F67C7383ED000A94F8C1
:1082F000743F5BB1D4F8780F41F28833ABEB000BDD
:108300009B4540F29180002384F8743FD4F8140B0D
:108310009FED650A6C3037F0F1FB04AB8DED070A79
:10832000CDED080A8DED091A9FED600A96E8070069
:1083300001AE83E8070086E80700304637F0DEFB31
:108340002846B0EE408A8DED040AF0EE608ACDED4D
:10835000050A8DED061A10F059F8002876D0DFEDE9
:10836000547AF4EEE79AF1EE10FA94BF0125002555
:10837000D4F81C0BB4F016FC30B1DFED4D7AB4EE3E
:10838000E79AF1EE10FA0AD9002D66D1D7F8C40F9A
:1083900003681B689847022866D04FF00008D4F89D
:1083A0001C0BB4F029FD0546002876D0B5EEC0AA16
:1083B000F1EE10FA70D5DFED3F7AB4EEE7AAF1EEF8
:1083C00010FAACBF012600265046B9F097FF66B9F7
:1083D000B0EEC00ADFED387AB4EEE70AF1EE10FA3B
:1083E0005DD8002D08BF4FF0000894F8741F84F882
:1083F000758F16E7B0EE489A3EE728460FF0CEFF9D
:1084000000287FF443AFDFED279A4CE7D7F8E83F29
:1084100093F8D530002B3FF451AF97F9B83F002BBC
:10842000BFF64CAF012347E75046B9F05BFF04F6B7
:108430007C73D3ED007A30EE670ADFED207AB4EE7C
:10844000E70AF1EE10FA3FF75EAF5FE728460FF05C
:10845000A5FF0546002882D18AE7D4F81C0BB4F0AA
:10846000A1FB002892D19AE7B0EE680A15F13CF919
:10847000F0EE408AB0EE480A15F136F9DFED107AD9
:1084800020EE280AB4EEE70AF1EE10FACCBF4FF066
:1084900001084FF0000882E700252E4694E7B04619
:1084A000A3E700BF000000009F0CB345D30237399B
:1084B0000000FA420000C8C20000704200004842BA
:1084C00055CF7D3F38B504460FF0A0FF04F50655A3
:1084D000183548B920460FF061FF014620B92846FB
:1084E000BDE8384013F024BC04F5A044D4F8C40F10
:1084F00003689B6C984720B9D4F8C40F0368DB6C01
:1085000098470146EBE7000030B5044689B004F512
:10851000065568461AF086FE04A818351AF082FE41
:108520006946284613F0E6FCA0B104A9284613F0DA
:10853000B5FD78B1059B002269462046019323686A
:10854000D3F8B030984728B104F5AE40012144304B
:10855000BFF098F809B030BD00F5005292F814242D
:10856000D2070CD400F5A042D2F8E82F92F8D5102B
:1085700009B1FFF7C9BF0368D3F8AC30184770479B
:1085800030B587B0044602A801911AF04BFE04F5FD
:10859000065002A9183013F0ADFC019A18B9002555
:1085A000284607B030BD236802A92046D3F8B03072
:1085B000984705460028F2D004F5AE40012144302A
:1085C000BFF060F8ECE70000F0B5044685B00F4658
:1085D000154604F5065668461AF024FE6946183614
:1085E000304613F05BFD10B9002005B0F0BD3946F0
:1085F000304613F00FFB0028F6D0002DF5D004F51F
:108600000054284694F8143443F0020384F81434D8
:10861000EBE700002DE9F04F2DED0A8BBDB00446CD
:1086200024220E4618A8002118F1D4FF242200218C
:1086300021A818F1CFFF242200212AA818F1CAFF8F
:108640002422002133A818F1C5FF04F5A04500231A
:10865000CDE90D330F9395F8B93F13F0080837D1E2
:1086600043F0080395F8402B079285F8B93F1CF0BA
:108670001BF990F9253003B390F84433EBB104F2C1
:10868000EC67C24638461CF007F85FFA8AF194F8A6
:1086900012378B421FD938460AF1010A1BF0DAFF64
:1086A00081460028F1D1C94A0221304671F0E4FA2E
:1086B00095F8B93F69F3C30308E0C54A0221304683
:1086C00071F0DAFA95F8B93F6FF3C30385F8B93F53
:1086D0004FF001083CE304F5B84301216833184624
:1086E0000BEE903AF9F7E0FD814608B9B94ADBE7AD
:1086F00020460FF04DFBD5F84C3BB3F90890B9F18B
:10870000000F01D0B44AD9E795F9B83F002B01DB3F
:10871000B24AC9E720469FEDB28A01F097FE04F500
:10872000C0434A460CA9143318460CEE103A17F011
:1087300051FA00284FF08F0113AA14BF022301231E
:10874000307C0393F123ADF85490CDE913390A231B
:108750004FF00009CDE9003103234D216EF024FED6
:10876000A04B0122062130465A729F4A71F084FACA
:10877000039B06213046022B0CBF9C4A9C4A71F099
:108780007BFA04F540534946384683F8169E1BF0A1
:10879000C5FE5FFA89F194F812378B420CD913AAFF
:1087A00038468DED138A09F101098DED148A8DED9E
:1087B000158A1BF031FDECE74FF0000A4FF07C0BFF
:1087C00038461BF069FF5FFA8AF994F812274A4588
:1087D00019D9494638461BF011FC3CAAC0B20C23FB
:1087E0000AF1010A0BFB004003FB092C00F5F060C5
:1087F000ACF1900C07C88CE807003CAA02EB890991
:1088000009ED2F8ADFE741F288310AA82DF09CF9A3
:10881000D5F8E80F9FED729A0368F0EE499A9FED44
:1088200075AA9B6A9847D5F8E80F01210025BBF08F
:10883000A5F8714BDFED71AA01211B68D86A02937C
:1088400003681B689847C4F0C7FA0590C4F0C4FADF
:10885000069004F5A049079A99F8403B934240F0EE
:10886000D58094F8321A38461BF0F4FE002800F048
:10887000CD80D9F8E83F93F8D5300493002B00F071
:10888000C58041F288310BA82DF05EF9C4F0A4FA3E
:10889000059BC01A132840F2D680C4F09DFA0590BB
:1088A00020460FF075FA79F017FC824679F09EFBAE
:1088B000D9F84C3BD9F8E80FB3F9083000EE103A7C
:1088C000B8EEC00A20EE0A0ABCF0A0FE504679F0CD
:1088D00095FB38461BF0E0FE1CEE100A17F094FBE7
:1088E000D9F84C3BA220B7EE001AB3F90830DFEDFF
:1088F0003C0A00EE103AB8EEC00A20EE0A0A31F047
:10890000A7FCB4EEE90A00220CA91CEE100AF0EE56
:10891000408AF1EE10FA58BFF0EE409A17F05AF97B
:1089200008B900230C939DED0C8ADFED357AB4EE87
:10893000498AF1EE10FAF4EEE78A48BFB0EE498AB0
:10894000F1EE10FA80F28D804FF0000A9FED2D9A23
:10895000DFED2D8A5FFA8AFB94F812375B4540F20F
:1089600094814FF00C0918ABB0EE490A0AF1010AE4
:1089700009FB0BF903EB090037F0C0F859463846FC
:10898000CDED110A8DED121A8DED100A1BF036FB9C
:108990007C23C0B2B0EE680A03FB004000F5F06033
:1089A00037F0ACF83CAB13A910A899448DED130A2D
:1089B000CDED140A8DED151A37F074F809ED240A7F
:1089C00049ED230A09ED221AC4E700BF49C814087B
:1089D00038C814085FE5140857C8140869C8140893
:1089E000000000002DC1003074C8140889C81408A4
:1089F000E36514086F12833A38BF00300000C842A4
:108A000000000034A4707D3F0AD7233CD9F8E80F5A
:108A100003689B6A98470021D9F8E80FBAF0AEFFC7
:108A2000029B0021D86A03681B689847002D40F01C
:108A30005F813046C94A052171F01EF92946384642
:108A40001BF06CFD70E1029BB0EE498A0521986A2B
:108A500003685B6898470BA82DF082F8B0EE489A3F
:108A6000F7E64FF000094FF00C0B04F22C7A5FFA96
:108A700089F394F812279A4222D919463846089366
:108A80001BF0BCFA089B4FF07C0CC0B209F1010945
:108A90000BFB03F13CAB0CFB00A05A185430A2F1C5
:108AA0006C03CDE9083218AB194437F011F8089B74
:108AB000099A02ED1B0AC3ED010A83ED021AD6E7FB
:108AC000039B4FF0000A012B46D14FF00C0B9FED9A
:108AD000A4BA9FEDA49A94F812375FFA8AF5AB42D4
:108AE00040F286800BFB05F53CABB0EE680A0AF15C
:108AF000010A03EB0509A9F14803089321AB5819B2
:108B000037F00CF8089B09ED120AB0EE4B0AC3EDE2
:108B1000010A83ED021A33AB581936F0EFFF2AAB86
:108B20008DED100AB0EE490A5819CDED110A8DED00
:108B3000121A36F0E3FF13A910A88DED130ACDED3C
:108B4000140A8DED151A36F0C3FF09ED090A49ED37
:108B5000080A09ED071ABEE7F0EE088A9FED809A31
:108B60009FED80BA94F812375FFA8AF94B4564D9C1
:108B70009DED0C0AB4EEE80AF1EE10FA35DB0C2399
:108B800003FB09F93CAB03EB090521AB03EB09003F
:108B900036F0C4FF33AB05ED120AB0EE490A45EDDD
:108BA000110A03EB090005ED101A36F0A7FF2AABF6
:108BB0008DED100AB0EE4B0A03EB0900CDED110A62
:108BC0008DED121A36F09AFF13A910A88DED130A35
:108BD000CDED140A8DED151A36F07AFF05ED090A70
:108BE00045ED080A05ED071A049D0AF1010AB9E7E7
:108BF0004FF000094FF00C0A94F812375FFA89F52C
:108C0000AB4241D933AB09F101090AFB053037F01A
:108C100093FB1BEE900AF0EE408AAEF0F1FB07EEFC
:108C2000900A3CABB8EE677A03EB8505C8EE877A0D
:108C300067EEAA7A45ED2F7ADEE74FF0000A4FF093
:108C40000C0B94F812375FFA8AF94B451DD933ABF8
:108C50000AF1010A0BFB093037F06EFBC8EE297AE6
:108C60001BEE900A67EE808AAEF0CAFB07EE900A10
:108C70003CABB8EE677A03EB8909C8EE877A67EEFA
:108C8000AA7A49ED2F7ADCE7049DC4F0A5F8069B8B
:108C9000C01AB0F5FA7F27D9C4F09EF804F5A043B6
:108CA0000C9AB121D3F84C3BDDED0D7A1B89139260
:108CB000FCEEE77A339AADF85C30149217EE903AF6
:108CC000349AADF85E3014231592359A06901692B8
:108CD000F022307CCDE9003213AA6EF065FB9DF0E6
:108CE0001FFD317C9DF0D2FB0BA82CF039FFB5E6BF
:108CF00000254FF00C0A039938461BF00FFCE9B22F
:108D000094F812378B4207D933AB384601350AFB4A
:108D100001321BF081FAF2E738461BF08FFA124A53
:108D20000621304670F0A8FF104B002520465D72EA
:108D300001F07EFB04F5785016305FF0BBFF99F828
:108D4000B93F0AA865F3C30389F8B93F2CF008FFBF
:108D500040463DB0BDEC0A8BBDE8F08FA10017087E
:108D6000A4707D3F0AD7233C91C814082DC1003060
:108D7000F0B5534F85B00446D7F8D83ADA0700F17A
:108D80009C8000F5A045D5F8E83F93F8C120002A63
:108D900040F0938093F8D530002B00F08B8095F94C
:108DA000B83F002BC0F2868000F5E04696F8803F81
:108DB000002B40F08280D6F8140B9FED420A6C30F5
:108DC00036F09CFECDED020A60EEA00ADFED3E7AA1
:108DD0008DED010A8DED031AE0EE000AF4EEE70ACC
:108DE000F1EE10FA66DCD6F8143B9FED387AD3ED3D
:108DF000377AF4EEC77AF1EE10FA04D5D5F8E83FE9
:108E00001B7A002B56D0B5EE007AF4EEC77AF1EE5D
:108E100010FA4FD404F5F5407830B9F06FFADFED71
:108E20002C7AB4EEE70AF1EE10FA43D8D6F8143BE8
:108E30009FED287AD3ED367A67EE877AB3EE0E7A15
:108E4000F4EEC77AF1EE10FA34DA234AB4F9A4103A
:108E5000138801339BB2138019B9B4F8A210A4F897
:108E6000A410B4F8A410994227D8002616806AF0FE
:108E70000DFE012219216AF065FDD5F8E80F03689F
:108E80005B699847431C04F5BA40144A3146503098
:108E90006DF0DAF9D5F8E83F012283F8C120D7F860
:108EA000D83A5B0709D504F5C85005B0BDE8F040D5
:108EB0008CF0D0BA084B00221A8005B0F0BD00BF7C
:108EC000C88200309F0CB3454054094A6666663F2D
:108ED000000000B4E02E65427EBF0030A8C8140830
:108EE000494B70B52DED028BD3F8D83A84B00446C7
:108EF0009B071FD400F5E045DFED448AD5F8140B3D
:108F000003681B699847D0ED017AF4EEE87AF1EE38
:108F100010FA0FDB04F5A04304F5FF46D3F8E82F61
:108F2000043692F8C11049B1002303A930460393D7
:108F30006CF0F4FA04B0BDEC028B70BD92F8D52051
:108F4000002AF1D093F9B83F002BEDDB95F8803F74
:108F5000002BE9D1D5F8140B03681B699847D0F8AA
:108F6000B030D5F8140B039303681B69984704F5D8
:108F70008C7200F1B00130466CF0F2FBDDED037A4B
:108F8000B0EEC08AF0EEE77AF4EEC87AF1EE10FAAD
:108F900003D503A930466CF0C1FAD5F8140B036869
:108FA0001B699847D0ED040AF4EEE80AF1EE10FAD6
:108FB000C0DBF6EE087A60EEA77AF4EEC87AF1EE3E
:108FC00010FA1AD5C3F008FFD5F8903F42F210729C
:108FD000C31A9342AED99FED0E0A0021C5F8900F37
:108FE00004F5BA4028EE000A0A4A5030B7EEC00A2B
:108FF0008DED000B6DF028F99CE79DED030A30F034
:10900000C5FF0028DED195E7C8820030000000349B
:109010000000C842C4C8140810B5044600F5F94061
:10902000243082F0C7FF04F5F94001214430BDE847
:10903000104093F005B80000F8B500F5E04504468F
:1090400095F9A43C4BB300F5A04695F8B82C00F573
:10905000F94700F5F54096F8B83F78302437DB4300
:10906000C3F3C01363F3C30285F8B82CB9F046F913
:10907000DFED3D7A384620EE670A83F01BF895F85D
:10908000803F53B9384682F0C1FFD6F8E83F93F8E5
:10909000D5301BB9354B00221A80F8BD95F8B83C85
:1090A000DB07FAD4D6F8C40F03689B6B98470028F7
:1090B000F0D096F9B83F002BECDB2C4E33884BB93F
:1090C000B5F9AA3C33B1642213FB02F3D5F8EC2ABC
:1090D0009A42E2DB384683F009F8D5F8143B9FED5D
:1090E000247AD3ED367A67EE877AB3EE0E7AF4EE11
:1090F000C77AF1EE10FA05D83388002BCDD0013BAA
:109100003380CAE7B4F9A4301BB9B4F8A230A4F88C
:10911000A4303388B4F8A420B4F9A40093421549CC
:10912000D5F8C42A3CBF013333803388012B01D1E9
:109130000A60B2E709689142ACDD18B9B4F8A22020
:10914000A4F8A420B4F8A4209A42A6D8002333801F
:109150006AF09CFC02220C216AF0F4FB2046BDE878
:10916000F840FFF759BF00BF0AD7233C7CBF00304F
:10917000E02E654278BF003000F5E04208B592F974
:10918000A43C6BB300F5A04393F9B83F002B0EDA73
:1091900000F5BA40134A062150306DF055F86AF0D8
:1091A00075FC03220F21BDE808406AF0CBBBB2F981
:1091B000AA3C8BB16421D2F8EC2A13FB01F39A424A
:1091C0000ADA00F5BA40084A012150306DF03CF847
:1091D0006AF05CFC0222E5E7BDE80840FFF71CBF2F
:1091E00008BD00BFDCC81408EEC81408F0B500F5CF
:1091F000A0450446574E2DED028BD5F8E83F8DB0C3
:1092000093F8D53043B195F9B83F002B04DB00F556
:10921000405393F9323E2BB9002333800DB0BDEC9F
:10922000028BF0BD00F5E04797F8803F002BF3D1AB
:1092300001F072FB002874D1D5F8C40F03689B6B52
:1092400098470028E8D004F5F54048306CF0BCF9A8
:1092500037F072F8F0EE087AF0EE408AB4EEE70AE2
:10926000F1EE10FAD8DA04F500539FED3B8AD3ED06
:10927000F97A93EDF80A20EE270A15F165FAF2EE75
:109280000E7A20EE080AB4EEE70AF1EE10FAC3D91E
:10929000D7F8143BF3EE0E7A93ED367A27EE088A70
:1092A000B4EEE78AF1EE10FAB6D904F506500023C1
:1092B00009A9183009930A930B9312F0FBFE0028BA
:1092C00037D13388B4F9A42001339BB23380002A0C
:1092D0003AD0B4F8A420B3EB420F9FDB6AF0D6FB80
:1092E00001220C216AF02EFB00221C4BB7EEE80A8B
:1092F000B7EEC88A04F5BA4000215030CDE9062304
:10930000174B00228DED040BCDE902238DED008B70
:10931000144A6CF099FF01220C211348F9F73CFA2A
:109320007CE7D5F8C40F0368DB6C9847002883D12D
:1093300072E709A837F000F8F2EE047AB4EEE70A13
:10934000F1EE10FABDDB67E7B4F8A220A4F8A42080
:10935000BFE700BF74BF0030E02E65420000084048
:1093600000003E4004C91408308F0030F0B50023DF
:109370008BB0044600F50650079302AA089304F543
:10938000A046099305AB03A91830019307AB0093DE
:1093900004AB12F0FDFC054686F8440D18B9002513
:1093A00028460BB0F0BDC3F00FFDD6F8483D9FED49
:1093B000337A0746C31A04F5BA4006AA02A907EE93
:1093C000903A2030F8EE677A67EE877ACDED067A2C
:1093D0006CF0C6F904F5BA4006AA03A98DED020A9D
:1093E0002C306CF0BDF904F5BA4004F5785406AAA7
:1093F00004A938308DED030A6CF0B2F9C6F8487D47
:10940000D4ED0D7AF5EEC07AF1EE10FAC7D9DDEDA4
:10941000086A9DED077AD6F8C82C87FE267ADDED1E
:10942000096A87FE267AF4EEC77A9DED037AF1EE9B
:1094300010FA94BF012300231AB196F8CC2CD2075E
:1094400012D477EEA76AF4EEC76AF1EE10FA0BD8E1
:109450000233DBB29DED027AF4EEC77AF1EE10FA38
:1094600009D8002B9BD09BE7F4EEC77AF1EE10FAF7
:10947000F0D80133EDE7012B92D890E7BD37863560
:1094800070B500F5A045044695F8DD3F43F00403B0
:1094900085F8DD3F6AF0FAFA012211216AF052FAEA
:1094A000D5F8E83F93F8D530002B43D0D5F8C40F5A
:1094B00003681B68984709280AD1204609F0ECFA8E
:1094C00030B104F50640BDE87040C43009F0CCBAB4
:1094D000194BD3F8C40F03681B69984704F5405330
:1094E00040B993F9313E032B24D10621204609F0DF
:1094F000BFFA0DE093F9311E0229F6D195F8DD3F50
:10950000DB07F2D40622204602F0C8F80028ECD08F
:109510000122D5F8C40F094B5A7303681B6C984796
:10952000034604F5BA40064A02215030BDE87040B7
:109530006CF08ABE70BD00BFC88200302DC1003003
:1095400038C9140800F5A04208B592F8DD3F590764
:1095500017D56FF3820382F8DD3F0A4B5A7B42B185
:10956000002200F5BA4002215A735030064A6CF0CE
:109570006BFE6AF08BFA00221121BDE808406AF008
:10958000E1B908BD2DC100305CC91408F0B505462D
:1095900085B005F50657684619F044FE6946183748
:1095A000384612F07BFD80B105F57853384CD3ED89
:1095B0000D7AF5EEC07AF1EE10FA08D80023354A9C
:1095C00028462380D373FFF7BDFF05B0F0BD2846C2
:1095D000FFF7CCFE064628460EF0E0FE10B92846FE
:1095E0000EF0B6FE002EA37818BF00200343DBB2B6
:1095F000A370002BE9D06378A8BB83BB2378013329
:10960000DBB2082B237003D14EB3384612F046FC70
:109610002378092B02D1384612F038FC2378092B25
:109620001DD94FF4857323806AF030FA022210218D
:109630006AF088F9C3F0D0FB6368C01A47F2305370
:10964000984209D905F5BA40134A022150306CF00E
:10965000FBFDC3F0C1FB60602846FFF711FF627895
:109660000C4BDA73B1E72678002EF8D0013EF6B243
:109670002670002BF3D0002EF1D166706AF006FA46
:10968000324610216AF05EF92846FFF75BFFE6E7F5
:1096900080BF00302DC1003074C9140800F5A0430C
:1096A00093F8DD3F5B0701D5FFF7EABE7047000086
:1096B00073B5044600F5065001A904F5A04518301D
:1096C00012F09EF90646D5F80C3D83420CD004F505
:1096D000E043D3F8140BB1F0CFFFC5F80C6D6AF07E
:1096E000D5F93E216AF00EF904F5005695F9101DE2
:1096F00096F9A82496F8A83491421BD0FF2B19D0D4
:1097000004F5E043D3F8140BB1F0B6FF96F8A83493
:1097100085F8103D6AF0BAF995F8102D18216AF015
:1097200011F904F5BA4095F9103D0421024A503070
:109730006CF08AFD02B070BD84C914082DE9F043B5
:109740008FB00546C3F048FB002305F506580646D2
:10975000059308AA069308F11808079305A908932A
:10976000404609930A930B930C930D9304AB01931A
:1097700003AB00930BAB12F0E9FADFED477A9DEDF6
:10978000077A0746B4EEE77AF1EE10FA30DB9DED8A
:109790000A7AB4EEE77AF1EE10FAACBF01240024A5
:1097A00005F5A049404699F8443D002B08BF002725
:1097B00012F0E0FA8046EFB9444699F9703A012B6D
:1097C00029D164B1D9F8E83F93F8D5403CB1D9F834
:1097D000C40F03685B69984780F00100C4B299F830
:1097E000143DCBBBCCB9C9F8186D0FB0BDE8F08300
:1097F0000024D5E7002CDFD005F5BA402C306BF003
:109800008BFEF7EE007A90ED007AB4EEE77AF1EE97
:1098100010FAD2DCD0E70024E1E7D9F8180D301AAD
:10982000B0F57A7FE1D9C9F81C3D012405F5E04384
:1098300089F8144DD3F81C3B83F848446AF026F9A4
:1098400022461D216AF07EF8144A05F5BA4002212D
:1098500050306CF0F9FCC8E714B1C9F81C6DC4E7CE
:10986000D9F81C0D43F69823361A9E42BDD905F54A
:10987000E043C9F8184D89F8144DD3F81C3B83F820
:109880004844C9F81C4D6AF001F922461D216AF0CE
:1098900059F8034AD9E700BF000000349CC91408F6
:1098A000B6C914080B4B012210B504465A72C3F016
:1098B00093FA04F5E042D2F86C3FC31A142B08D98E
:1098C000C2F86C0F04F50550BDE81040083059F09F
:1098D0009FBD10BD2DC100302DE9F743044600F5B2
:1098E000785000230DF1070104F5A0462C308DF8C7
:1098F000073060F01BF9D6F8E80F90F9C030026825
:1099000083B3083B9569DBB2012B2BD93221A847E1
:1099100004F1100004F5BA4816F000FD1F4B4FF09B
:10992000000908F150081F68F86A0368DB69984766
:1099300001281ED1C3F050FA41F28733A0EB09028F
:1099400005469A4205D9A946154A062140466CF0BB
:109950007BFC2046FFF7A6FFB86A032103685B681B
:109960009847E1E704F540539269B3F8401E9047E9
:10997000CEE70121D6F8E80FBAF000F8D6F8E80FE4
:109980000368DB6A984777F0ADFEF86A0121036847
:109990001B6803B0BDE8F043184700BF38BF003074
:1099A000D4C9140870B5044600F5BA40184A062117
:1099B0005030184E2DED028B9FED178A6CF044FC51
:1099C0002046FFF789FF2046FFF76CFF20460EF088
:1099D000DFF933680321986A03685B68984778F079
:1099E0007BFB054678F002FB04F5A043D3F84C2B33
:1099F000D3F8E80FB2F9082000EE102AB8EEC00A3A
:109A000020EE080ABBF002FE284678F0F7FADAE703
:109A1000F8C9140838BF00306F12833A2DE9F047B7
:109A2000044600F5BA402B4A0621503004F5A04602
:109A3000DFF8A89041F2873A2DED028B6CF004FC20
:109A40002046FFF749FF78F047FB054678F0CEFA4D
:109A5000B7EE000AD6F8E80FBBF0D8FD284678F03C
:109A6000CDFAC3F0B9F90746C3F0B6F9C01BD9F86F
:109A70000080504517D99FED188A284678F0B6FA2D
:109A8000B0EE480AD6F8E80FBBF0C0FD284678F0E3
:109A9000B5FA2046FFF706FFD8F82800032103682F
:109AA0005B689847E9E7284678F0A0FAB7EE000A25
:109AB000D6F8E80FBBF0AAFD284678F09FFA2046BA
:109AC000FFF7F0FED8F82800032103685B68984789
:109AD000CAE700BF28CA14080000000038BF0030E1
:109AE0002DE9F34100F5A0460446D6F8E83F93F986
:109AF000C030032B2BD0652500F5E048344F013DE5
:109B000015F0FF050CD0D8F8683F4BB93B6814211D
:109B1000986A03685B68984720460EF039F9EEE7CB
:109B200004F5B84001216830F8F7BEFB04F5405356
:109B300093F92C3E70B953B1092B08D08DF807006A
:109B400004F578500DF107012C305FF0EFFF02B003
:109B5000BDE8F081032B34D8DFE803F002252D3077
:109B6000D6F84C3BB3F9082040F2B5339A422ADDCF
:109B700004F5785001250DF107012C308DF80750C0
:109B80005FF0D4FF04F5BA40124A022150306CF065
:109B90005BFB114B5D720E4B1C68A06A05210368CC
:109BA0005B689847F9E7D6F84C3BB3F9082040F2D8
:109BB000B5339A4207DD2046FFF7F4FE2046FFF753
:109BC0002DFF092BC3D000238DF80730B8E700BF65
:109BD00038BF00304CCA14082DC1003000F5BA401F
:109BE0000B46024A042150306CF02EBB6CCA14089C
:109BF00010B5044669F04AFF0022052169F0A2FE73
:109C000004F5BA40034A04215030BDE810406CF01E
:109C10001BBB00BF78CA14080B4613B54AB100F548
:109C2000BA4000920421054A50306CF00DFB02B09E
:109C300010BD02B0BDE81040FFF7D0BF90CA1408B5
:109C400000F5BA40064A0421503008B56CF0FCFA21
:109C500069F01CFF00220821BDE8084069F072BECF
:109C6000A4CA140838B504460D46C3F0B5F804F587
:109C7000A0433DB9D3F8D42FC3F8D80F0AB9C3F81D
:109C8000D40F38BDD3F8D82F801A642882BF0022A1
:109C9000C3F8D82FC3F8D42FF3E7000037B5044634
:109CA00000F5F5407830B8F00FFB04F5A042C0F3A2
:109CB000803592F8BA3FC3F34001A9421DD065F345
:109CC000410304F5BA4482F8BA3F50346DB169F0EB
:109CD000DDFE02220B2169F035FE094A02212046F1
:109CE00003B0BDE830406CF0AFBA69F0CFFE2A4651
:109CF0000B2169F027FE034AF0E703B030BD00BF37
:109D0000BCCA1408D8CA140838B50A460C4606213D
:109D1000054601F0C3FC28B1054A137843F0080357
:109D2000137038BD21462846BDE8384008F0A0BE73
:109D30004CC1003038B50A460D461521044601F0E5
:109D4000ADFC28B1094A137843F00803137038BDFD
:109D500004F5BA400421064A50306CF075FA2946E1
:109D60002046BDE8384008F083BE00BF4CC100303B
:109D7000E8CA140838B50A460D461521044601F014
:109D80008DFC28B1094A137843F00803137038BDDD
:109D900004F5BA400421064A50306CF055FA2946C1
:109DA0002046BDE83840FFF7AFBF00BF4CC10030D0
:109DB00010CB140838B50A460D461B21044601F0A5
:109DC0006DFC28B1094A137843F00803137038BDBD
:109DD00004F5BA400421064A50306CF035FA2946A1
:109DE0002046BDE83840FFF78FBF00BF4CC10030B0
:109DF00026CB140838B50A460D461121044601F059
:109E00004DFC28B1094A137843F00803137038BD9C
:109E100004F5BA400421064A50306CF015FA294680
:109E20002046BDE8384008F023BE00BF4CC10030DA
:109E300038CB140810B500F5A04494F8BA3F9A0640
:109E400023D4D4F8C40F03681B689847032808D0AC
:109E500005D802280ED194F8B80FC00914E01B28C9
:109E6000F9D194F8B80F00F0A000A0F18003584297
:109E7000584109E0B4F8B80F20F4FE4020F07F000C
:109E800080B2003818BF012010BD0120FCE700009F
:109E900038B500F5A045044600F5BA40184A95F8D3
:109EA000DD3F0221503043F0080385F8DD3F6CF0C0
:109EB000CBF969F0EBFD0122172169F043FD204643
:109EC000FFF7B8FF40B104F5B84001221521683012
:109ED000BDE83840F8F760BCD5F8C40F03681B68CC
:109EE0009847062806D104F50740BDE83840E03021
:109EF0000AF06EB820460B21BDE83840FFF704BFDA
:109F00004CCB140870B500F5A0450646D5F8D42F03
:109F1000D5F8D83F9B1A41F28832934211D9D5F82F
:109F2000C40F03681B6D9847044695F8DD3FC3F3E3
:109F3000C003A34213D034B13046BDE87040FFF7F0
:109F4000A7BF0024F1E769F0A1FD2246172169F0BF
:109F5000F9FC95F8DD3F64F3C30385F8DD3F70BD80
:109F60000B46114610B50446072B07D8DFE803F06F
:109F700029041215181B232608F07AFD04F5A043C6
:109F8000D3F8743A9B061CD504F5C850BDE81040C0
:109F90008BF060BAFFF7B8FEF0E7FFF7EBFEEDE7F6
:109FA000FFF7C8FEEAE700F5B84001221421683047
:109FB000F8F7F2FBE2E7FFF7FDFEDFE7FFF71AFF36
:109FC000DCE710BD70B5044669F060FD0122052193
:109FD00069F0B8FC04F54053204693F8163E072B71
:109FE00096BF304A0125D55CFFF724FF68B12E4AA1
:109FF00020462E49FFF710FE04F5B840012210213B
:10A000006830F8F7C9FB002516E004F5A046D6F83D
:10A01000C40F0368DB6C9847A8B104F5C04393F8FC
:10A02000A92582B193F9A835012B0CDC204A2149DE
:10A0300001252046FFF7F0FD294620460322BDE812
:10A040007040FFF78DBFD6F8C40F0368DB6C9847EC
:10A0500018B1D6F8743A190715D4D6F8C40F0368A6
:10A060001B689847032803D1D6F8743ADA070DD451
:10A07000D6F8C40F03685B6A984768B90B49204655
:10A08000FFF7ACFDD8E70A4A0849D1E70A4A074971
:10A090002046FFF7C1FDB6E7D6F8743A5B07EDD569
:10A0A000064AF4E718CC14086CCB1408CDE8150860
:10A0B00076CB140889CB140899CB1408A9CB1408C3
:10A0C00070B50446154669F0E1FC0122062169F0ED
:10A0D00039FC2046FFF7AEFE98B104F5B8400122E6
:10A0E000072100256830F8F757FB134A134920462B
:10A0F000FFF792FD294620460422BDE87040FFF795
:10A100002FBF04F5A046EDB2D6F8C40F0368DB6C90
:10A11000984758B1D6F8743A1B0707D535B1084AA5
:10A12000204606490125FFF777FDE3E7034920466E
:10A13000FFF754FDDEE700BF6CCB1408C6CB140854
:10A1400076CB1408F8B5044669F0A0FC012208217A
:10A1500069F0F8FB04F5A04675F05AFD04F540538C
:10A1600093F8053E072B96BF364A0225D55CD6F8F4
:10A17000E83F93F8D5705FB933492046FFF72EFDCD
:10A180000025294620460522BDE8F840FFF7E8BE35
:10A190002046FFF74FFE60B104F5B84001221221BE
:10A1A0006830F8F7F9FA294A27492046FFF734FDC5
:10A1B000E6E7D6F8C40F0368DB6C984778B104F57E
:10A1C000C04393F8A92552B193F9A835012B06DCB9
:10A1D0001F4A204920460125FFF71EFDD1E7D6F88A
:10A1E000C40F0368DB6C984718B1D6F8743A1907A6
:10A1F00013D4D6F8C40F03681B689847032803D10B
:10A20000D6F8743A9A070BD4D6F8743ADB0609D418
:10A210000D492046FFF7E2FCB3E70D4A0A49D9E7AA
:10A220000D4AC1E7D6F8C40F0368DB6998470646B4
:10A230000028EDD1094A204603493546FFF7ECFCDA
:10A240009FE700BF20CC14085EB614086CCB14083E
:10A2500076CB1408C0CB1408CECB1408E3CB14087B
:10A2600000F5405370B593F9053E0446BBB300F5C5
:10A27000A045D5F8486F96B3C2F0AEFD05F52D6345
:10A28000DFED177A861B93ED000A8D209FED151ADE
:10A2900020EE270ADFED140A2FF0DAFFBCEEC00A29
:10A2A00010EE103A9E420CD295F8DD3F9A0716D573
:10A2B00020460021F8F7C8FB2046BDE87040FFF7B4
:10A2C000BFBC0CD995F8DD3F9B0708D4204601217F
:10A2D000F8F7BAFB2046BDE87040FFF733BF70BD0A
:10A2E00000007A440000804F000000002DE9F34197
:10A2F000074600F5F54007F5A0447830B7F0E4FFD5
:10A30000C0F380480190C2F067FD94F8E03F4546F5
:10A31000064643450DD007F5BA4084F8E08F50302B
:10A32000002D3FD03A4B3B4AC4F8E46F02216BF05A
:10A330008BFF94F8E03F43B394F8E13F2BBBB4F9B3
:10A34000E63A40F257109FED340A07EE903A9FED3F
:10A35000331ADFED330AF8EEE77A27EE800A2FF0A2
:10A3600077FFBCEEC00AD4F8E40F10EE103A361AAC
:10A370009E420AD9012307F5BA402A4A022184F8ED
:10A38000E13F5030224B6BF05FFF94F9E53A002B30
:10A3900094F8DD3F0DDC6FF3451384F8DD3F02B028
:10A3A000BDE8F0811A4B204AC4F8E48F84F8E18FAD
:10A3B000BCE7C3F34012AA42F1D065F3451384F819
:10A3C000DD3F9B06EBD5194BD3F8C40F03681B691F
:10A3D00098470028E3D069F059FB01221F2169F05A
:10A3E000B1FA3846FFF726FD48B107F5B84001221B
:10A3F0002121683002B0BDE8F041F8F7CDB9322232
:10A4000094F8E51A384602B0BDE8F041FFF7A8BD60
:10A41000FCCB1408D4E0150800007A440000804FFB
:10A42000000000000BCC1408AFE01508C882003013
:10A4300008B50122034B1A70C2F0C6FC024B18602B
:10A4400008BD00BF89BF00308CBF0030014B002227
:10A450001A70704789BF00302DE9F0410446C2F000
:10A46000B3FC2A4B0546B4F8BE201988284E914209
:10A470000ED01A80274B18603378A3B100243470B3
:10A4800069F004FB22461321BDE8F04169F05ABA95
:10A490003378214FDBB93B782BB11E4B1F4A1B6829
:10A4A000C31A934201D8BDE8F0810123337004F54B
:10A4B000A043D3F8E80F90F8D53013B103689B6A36
:10A4C000984769F0E3FA0122132169F03BFA3B78DF
:10A4D000002BE8D03378002BE5D00E4A10491368E2
:10A4E000EB1A8B42DFD904F5A0441560D4F8E80FCD
:10A4F00090F8D530002BD6D00021B9F03FFAD4F82F
:10A50000E80F0368BDE8F0415B6A18478ABF003076
:10A5100088BF00308CBF003089BF003080841E00AF
:10A5200040420F002DE9F84300F5A04500F54058E2
:10A530000446D5F8C40F98F8687A0368DB6C98472E
:10A54000014650B995F9B83F002BA9BFD5F8E83FAF
:10A55000012193F8D50080F0010104F5685909F153
:10A560002C0948468CF066F9D5F8E83F064693F882
:10A57000D530002B7BD0002865D03E4B93F9B83FF7
:10A58000002B04DB02463C4948468BF02BFD98F932
:10A59000327A57B195F9B83F002B0EDA04F5B8407E
:10A5A00001220F216830F8F7F7F869F06FFA3246A8
:10A5B0000921BDE8F84369F0C5B9D5F8C40F0368AF
:10A5C0005B69984758B195F9B93F002B07DA95F8C0
:10A5D000DD3FDA0703D498F8683ADB07DED5314669
:10A5E00048468CF08DF9DFED257AB4EEE70AF1EEFE
:10A5F00010FA05DD0A220921204601F04FF8D4E7C0
:10A60000023F032F11D801A353F827F0F5A5020844
:10A610001DA602083BA6020841A602080A2215212F
:10A62000204601F03BF80028BFD10A22062120462F
:10A6300001F034F80028B8D1DCE70A221121F6E74E
:10A640000A221521F3E797B198F8683A7BB9094BCC
:10A6500093F9B83F002B06DB04F5BA40084A052100
:10A6600050306BF0F1FD69F011FA0022A0E7BDE86F
:10A67000F88300BFC882003028CC14080000C8420C
:10A6800031CC140870B500F5F54500F5A04386B04F
:10A690000446783593F8141D2846B7F0C3FD02A888
:10A6A00018F0C0FD04F5065002A9183011F022FC84
:10A6B00004F5E043049A2846C3F8F02A059AC3F843
:10A6C000F42AB7F001FE82061AD5284604F5F545AE
:10A6D000B7F008FEFDEEC07A683504F5005402229A
:10A6E00017EE901A284617EE906A18F0A1FD94F81C
:10A6F0001434DB0706D401223146284618F098FDB1
:10A7000006B070BD0121284618F024FE0028F2D0C2
:10A71000F6E7000070B500F5E04486B00D46164639
:10A72000B4F89C3F8B4203D1D4F8983F934221D098
:10A73000C2F052FBD4F8943FC31A132B1AD9C4F8B1
:10A74000986FA4F89C5FC4F8940F69F09FF90446D1
:10A75000C2F04AFB084B094A1B68CDE90453084B79
:10A760000193084BCDE9020100932046064B0749AF
:10A7700068F018FF06B070BD90BF003048CC1408D8
:10A7800060CC1408EA9E1408A17E14085BCC14085F
:10A7900038B500F5A0440D4694F8B93FC3F38013D3
:10A7A0008B420BD021B169F071F9112169F0AAF83F
:10A7B00094F8B93F65F3861384F8B93F38BD0000BB
:10A7C000F0B500F5A045064600F5E0442DED048BFC
:10A7D000D5F8E83F8BB093F8D530002B67D095F9CA
:10A7E000B83F002B63DBD5F8C40F03685B6998475B
:10A7F000002861D1D4F8140B01AF9FED430A6C30EF
:10A8000035F07CF90AAACDED080A04AB8DED091AE2
:10A810008DED070A12E9070083E8070087E80700C3
:10A82000384634F065FD06F5F540D4F8143BB0EE3B
:10A83000409A4830D3ED368A6AF0C6FE35F07CFD8A
:10A84000D4F81C3BD5F8C40FB0EE408AD3EDE49A9F
:10A850000368DB6C9847DFED2D7AB4EEE79AF1EEF2
:10A8600010FA02DC95F8C03F0BB1002838D0DFEDBC
:10A87000287A68EEA78AF3EE0E7AF4EEE78AF1EE14
:10A8800010FA2DDCF0EE087AB4EEE78AF1EE10FA59
:10A8900026DCF5EEC09AF1EE10FA21DAD4F8140BAA
:10A8A00003689B6F98470BB0BDEC048BF0BDD4F8E8
:10A8B000140B03689B6F0DE0D5F84C2BD4F8140BE8
:10A8C000B2F908200368002A03DCD5F8BC2F022A5D
:10A8D000F0D1DB6F0BB0BDEC048BBDE8F040184746
:10A8E000D4F8145BB7EE001A40F2AB10DFED090AA2
:10A8F0002B68D3F88060D4F81C3B93EDCC0A2FF082
:10A90000A7FC2846B047CEE79F0CB3450080BB4468
:10A91000E02E65420000000000F5A04090F8C00F56
:10A92000704700002DE9F04100F5A04506460C46B1
:10A9300095F8B83FB1EBD31F48D0254B00221A60E1
:10A9400000293FD069F0A2F8122168F0DBFF95F8EA
:10A95000B83F84F0010806F5405764F3C71385F843
:10A96000B83F9CF01DF841469BF0F6FFB8F1000F90
:10A9700006D097F8EE3B1BB9C2F02EFAC7F8F00BE1
:10A9800087F8EE8B14B3B7F8E83D5B071ED5D5F812
:10A99000E83F93F8D530CBB1D5F8C40F03685B69B5
:10A9A000984798B9D5F8C40F202103689B69984748
:10A9B00060B106F5B84001220D216830BDE8F041D4
:10A9C000F7F7EABE69F062F81C21BEE7BDE8F08146
:10A9D00090BF00302DE9F04F00F5A045044600F58A
:10A9E000E0472DED0A8BD5F8E83F8DB093F8D560A0
:10A9F0001EB90121FFF796FF0BE095F9B82F002A49
:10AA000065DAD5F8C40F03689B6C984706460028A2
:10AA100041D04FF0000B95F9B82FB24E002AC0F28A
:10AA20005481D6ED007AB4F9A420B8EE677A1AB949
:10AA3000B4F8A220A4F8A420B4F8A430DFEDAA6AE8
:10AA400007EE903AF8EEE77A67EEA67AB4EEE77A88
:10AA5000F1EE10FAACBF012100212046FFF798FE6D
:10AA600095F9B82F002A95F8B92FB8BF4BF0010B14
:10AA7000530697F8802F48BF4BF0020B0AB14BF0FA
:10AA8000080B3268594620460DB0BDEC0A8BBDE874
:10AA9000F04FFFF73FBED5F8E83F204693ED0C8A14
:10AAA000F8F7ACF8B4EEC80AF1EE10FAB1D5D5F863
:10AAB000E83F93F8A130032BABD167F0B7F94FF41F
:10AAC0008011422267F06AF93146204692E797F8F2
:10AAD00080AFBAF1000F03D00023824A136098E7D9
:10AAE000D7F8140B93F8079003685B6F984780467C
:10AAF0000090D5F8C40F03685B69984720B1D5F87A
:10AB0000BC3F022B00F0E380B9F1000FB7EE00BAB2
:10AB10000CBF4FF0000B4FF4007BB8F1000F02D0D8
:10AB20004BF4806B009604F5F9489FED70CAF3EE84
:10AB30000EBADFED6F8A08F14408404691F0A0FAA2
:10AB40000130D7F8140B0CBF012302239FED690AD3
:10AB50006C3008EE103A34F0D1FF0CAB0DF10C0E56
:10AB60000DF1180CCDED0A0A8DED0B1A8DED090AC9
:10AB700013E907008CE807008EE80700704634F000
:10AB8000B7FBD7F8142BDFED5C7AB4EECC0A92ED6C
:10AB900036AA04F5F540F0EE40AA2AEE27AA48307E
:10ABA000F1EE10FAB4EEEBAAC8BF4BF4807BF1EEE5
:10ABB00010FAC8BF4BF4807B6AF006FD35F0BCFB91
:10ABC000B8EEC88A04F5F540F0EE409AB4EEC80A33
:10ABD0007830F1EE10FA98BF4BF0800BB7F08EFB97
:10ABE00068EE288A2046B0EEC09AB4EEE89AF1EEFC
:10ABF00010FA48BF4BF0400B0DF0D8F9002846D1B1
:10AC00004BF0200B0196404691F03AFA01284FD1C3
:10AC10004BF0100BB2463349B9F1000F53D0009BF3
:10AC2000002B50D0F4EECCAAF1EE10FA4BDCB4EECF
:10AC3000EBAAF1EE10FA46DCF4EEC89AF1EE10FA47
:10AC400041D8B4EEE89AF1EE10FA3CD5019BD3B3AB
:10AC5000BAF1000F37D00A68B4F9A40007EE902AC1
:10AC6000B8EE677A18B9B4F8A200A4F8A400B4F852
:10AC7000A43007EE903AF8EEE77A67EE8B7AB4EEFE
:10AC8000E77AF1EE10FA19D501320A60C3E604F54D
:10AC9000B64068306AF040FCDFED187A90ED007A3B
:10ACA000B4EEE77AF1EE10FAAAD400230193AAE7F2
:10ACB000404691F0E5F90130ADD1A9E701212046E8
:10ACC000FFF730FEA7E60022DFE70121C5E6B9F174
:10ACD000000FB0EE08BA0CBF4FF0000B4FF4007B32
:10ACE0001EE700BF90BF0030CDCC4C3E0080BB447F
:10ACF0000000C8429F0CB345E02E65420000484367
:10AD000000F513539FED217A30B5283389B00446FE
:10AD100002AD93E8070085E80700DDED047A04F54D
:10AD2000F54077EE877A9FED1A7A4830CDED047AB8
:10AD3000D4ED2B7AF0EEE77AF4EEC77AF1EE10FA62
:10AD40000BD5B4F9A230F7EE006A07EE903AF8EEB0
:10AD5000E77A86EEA77A84ED2B7AD4F8AC3001AA94
:10AD6000294601936AF022FD2046FFF733FE204674
:10AD7000FEF762F92046FEF739FA2046FDF7F8FFA4
:10AD80002046FEF7ADF809B030BD00BF0AE81C410F
:10AD90000000003410B504461D202DED028B76F026
:10ADA000A3FE68B304F5A043D3F8C40F00F0D6FAAD
:10ADB00008EE100A04F5AC50192118305FF0C0FB02
:10ADC00002281AD00338012808D804F5B6406830A4
:10ADD0006AF0A2FB90ED008ABDEEC88AB8EEC88A80
:10ADE0009FED090A04F5F94028EE000A4430BDEC55
:10ADF000028BBDE8104091F0C9B99FED048AEDE7E0
:10AE0000BDEC028B10BD00BF0AD7233C0000000040
:10AE1000104A0260104A02F17401426002F5755254
:10AE200081604261243A0D4982610D4AC16004315A
:10AE3000C2610C4A016102620B4A4262A2F2A44260
:10AE400082620432C2620432026304324263074AFD
:10AE50008263704744E71408A4700030E8AD003006
:10AE600060540030DCAD0030B0920030E033003090
:10AE70001C2969D8DFE801F0130F171B27232F1FA8
:10AE8000682B68336868373B3E4245484B4F535800
:10AE90005C606868650000F5FF402430704700F58D
:10AEA00008406C30704700F5FF406430704700F593
:10AEB00000402030704700F505406830704700F5CD
:10AEC00007400C30704700F506408030704700F5B1
:10AED0000640C430704700F50740E030704700F589
:10AEE0000540A830704700F50540E430704700F594
:10AEF0000340DAE700F507404C30704700F50540A5
:10AF0000CBE700F50940ECE700F50940CDE700F597
:10AF10000940F830704700F50A403C30704700F5B2
:10AF2000A040D0F81408704700F50640383070474C
:10AF300000F50B40AC30704700F5A040D0F86C0A2B
:10AF4000704700F50C40A8E70020704773B50B6808
:10AF5000054608460C461B6C16469847034605F501
:10AF6000BA400F4A0421009650306BF06DF968F03A
:10AF70008DFD2368054620461B6898470A21024636
:10AF8000284668F0DFFC074B93F8B93F9B0641BFAA
:10AF9000054A137843F00403137002B070BD00BF7C
:10AFA00064CC1408C88200304CC1003038B50C4A5B
:10AFB000182305460C4666F067FC78B12146284602
:10AFC000FFF756FF30B10146064A2846FFF7BEFF9D
:10AFD000002038BD284666F005FBF9E70120F8E7B8
:10AFE000E4CC140884CC140810B5002300F5A04468
:10AFF00000F5E04084F8FC3B074BD0F8140B93F8C5
:10B00000B81FC909AEF09EFFD4F8C40F0368BDE8AD
:10B010001040DB68184700BFC882003070B5054695
:10B0200008680C46164603685B69984790B130681B
:10B0300003685B69984768B905F5A043D3F8E82F22
:10B0400092F8D52032B193F9B83F002B02DB2846A5
:10B05000F7F7EAFD04480DF0EDFD20680368BDE850
:10B0600070409B68184700BF88C0003070B500F57D
:10B07000A04504460C4ED5F8C40F0368DB69984719
:10B080003074D5F8C40F03681B689847F070D5F882
:10B09000C40F03685B6C9847014604F50550BDE892
:10B0A0007040083058F04ABA2DC10030254B70B5B9
:10B0B0002DED028B93F8DD3FB0EE408AF0EE608A12
:10B0C00082B0DB0706460D46144606D500232B60EA
:10B0D000236002B0BDEC028B70BD74F0A9FE037F4B
:10B0E000002BF3D0F36A01A99FED171A68461B687D
:10B0F0009FED160A68EE811AB3F9083028EE011A9E
:10B1000007EE103AB36A1B68B8EEC77AB3F9083095
:10B1100067EE000A07EE903AF8EEE77A27EE800A2B
:10B1200030F050F9DFED0A6A9DED007ADDED017A2D
:10B1300027EE267A67EEA67A85ED007AC4ED007ACE
:10B14000C7E700BFC88200300AD7233C53046939DF
:10B150000000C84270B5002306462DED028B88B072
:10B16000B0EE408A029306AD039302AC324B93F8E3
:10B17000DD3F13F0010F03D174F05AFE037F5BB97A
:10B1800094E8030085E803009DED060ADDED070A5B
:10B1900008B0BDEC028B70BDB36ADFED286A1B6896
:10B1A000B3F9083007EE903AF36A1B68F8EEE77AD5
:10B1B000B3F9083067EEA67A07EE103AB8EEC77A10
:10B1C000CDED037A27EE267AF1EE476AB0EEC77A24
:10B1D000CDED026ADFED1A6AB4EEE67AF1EE10FA0E
:10B1E00006D5F0EEE77AF4EEE67AF1EE10FAC7D47F
:10B1F00003AA21461348F7F747FDDDED027A9DEDDE
:10B20000037A2046F0EEE77AB0EEC77AF4EE477A9A
:10B21000F1EE10FA37FE870A33F0B8FF04A88DED7F
:10B22000040ACDED050A34F063F8204688EE000AE2
:10B2300033F0DCFFA4E700BFC88200305304693953
:10B2400000000034C8320030094B93F9B82F002AAF
:10B250000CDAB5EEC00AF1EE10FA07D9D3F8E83FE0
:10B2600093F8A100C31E5842584170470020704710
:10B27000C8820030436A1B6893F8D53043B1054B50
:10B2800093F8B80F00F0A000203818BF01207047D5
:10B2900001207047C882003010B5436A0446186820
:10B2A000D1B10221B8F07AFB236A9FED0C1A18681D
:10B2B000F0EE410A0368B0EE410ADB6A9847236A60
:10B2C000074A00211868D2ED000A03689FED030ABF
:10B2D0005B6EBDE8104018470121E3E70000000065
:10B2E000AC70003010B5436A04461868002930D0AD
:10B2F0000221B8F053FB236A1868AEF0F3FD636ACD
:10B300001B6893F8A130012B04D8236A0121186827
:10B31000AFF09EFB63691868B2F078FE6369186845
:10B32000B2F01EFF63699FED0C0A1868B3F050F984
:10B3300063691868B3F0C8F9236A9FED071A1868A3
:10B34000F0EE410A0368B0EE410ADB6ABDE8104046
:10B3500018470121CDE700BF0000000013B50446E7
:10B3600001A90C480CF0B0FE10B1019802B010BD5C
:10B3700063691868B1F016FC18B9074BD3F8EC0AEA
:10B38000F4E701AA0321054817F088FF0028F4D04C
:10B39000EBE700BFC8320030C8A20030B0AD0030CB
:10B3A000F0B504462DED048B89B0002940F0FC80F7
:10B3B00083687F4E03F58053B3F9C259642DB8BF3B
:10B3C0006425FFF7CBFF6268A8422046B2F934300B
:10B3D000AABF96F8B95F0125C5F38015002BD5BF2C
:10B3E00063695B421B6807EE903AD4BF93EDC78A4E
:10B3F000B8EEE78AB2F93230002BB8BF5B429BB29D
:10B400005B4207EE903AA368F8EEE77A03F58053C3
:10B41000B3F9C279F4EEC87AF1EE10FA38FE278A51
:10B42000642FB8BF6427FFF799FF6369391AA26BCD
:10B430001B6800EE101AD2ED001A93EDC91AD3ED75
:10B440000E0AB8EEC00A2FF0A7FB6368F0EE480AB8
:10B4500040F29720B3F93230002BB8BF5B429BB269
:10B460005B4201EE103AB8EEC11A2EF0F1FE6369AC
:10B47000B0EE408A1868B1F095FB96F8BA3F0746DF
:10B480001A077ED44B48B3F075FE002879D0002F00
:10B4900077D09FED499A01A946488DED019A8DED2F
:10B4A000029AB3F0EFFE00287BD0A069B6F018FF37
:10B4B00003AB03C883E80300194601A833F04AFE32
:10B4C00005A88DED050ACDED060A33F011FFF0EE6B
:10B4D000409A3A4E05A9DFED3A7AD6ED008AA6F1F8
:10B4E00024008DED059AA6F6085668EEA78A8DED24
:10B4F000069A8DED079AB3F0EFFEF4EEE89AF1EEBE
:10B5000010FA08DDF0EEE88ADFED2E7AF4EEE78A35
:10B51000F1EE10FA49D5DDED077A9FED2B7AF4EEC6
:10B52000C77AF1EE10FA2CDD9FED287AF4EEC77A97
:10B53000F1EE10FA25D5B6F8203D5B0721D46368FB
:10B54000F2EE0E7AB3F93230002BB8BF5B429BB2F9
:10B5500008EE103ABAEEEF8A88EE277A67EE297A7B
:10B56000F5EEC07AF1EE10FA48BFDFED137A37EE50
:10B57000C88AFAEE047AB4EE678AF1EE10FA37FE62
:10B58000888A6369B0EE480A29461868B1F0AAFBB8
:10B590006369186809B0BDEC048BBDE8F040B3F0F6
:10B5A00093B8F0EE499A94E700259FED038AE8E707
:10B5B000C8820030ACAF003000000000D0AF0030D7
:10B5C0000000C8420000003400000C420000484364
:10B5D000436A186803681B691847000038B52DEDE9
:10B5E000028B03680446D3F884309847236B2A48BB
:10B5F000F0EE408A1B68B3F908500CF051FC041EB1
:10B600004FF47A724FF000012846D8BF4FF4FA7415
:10B610002EF086FEB6EE000A84422ADD07EE900A7E
:10B62000B8EEE77A07EE904AF8EEE77A27EE007A6E
:10B6300087EE278A4FF46D7038EEC00AF5EE087A6F
:10B64000B7EE001AB1EE400AFEEE000A80EE270ABD
:10B650002EF0FEFDF7EE007A77EEC07A28EE000AB3
:10B6600020EE080A20EE080AA7EE880ABDEC028B3D
:10B6700038BD031BC4F57A7407EE103A07EE904A02
:10B68000B8EEC77AF8EEE77A27EE007A87EE278AD7
:10B6900038EE008ACEE700BFC83200302DE9F04F07
:10B6A00000F5E04900F5A04605460F4690462DED11
:10B6B000028B99F8A04F83B089F8A02FD6F8C40F59
:10B6C00003681B689847B84222D105F54055B8F188
:10B6D0001A0F85F8EC8B07D130B906F6AC26D9F8ED
:10B6E000143B3268C3F8FC20904B93F8B93F9D0699
:10B6F00006D40124204603B0BDEC028BBDE8F08FD8
:10B700004445F6D08A4A137843F002031370F0E7F9
:10B71000B8F1020F0CD01B2F12D105F500404146A5
:10B72000203003B0BDEC028BBDE8F04F01F014BB3C
:10B7300039462846FFF73AFC04460028EBD1D9E702
:10B7400039462846FFF794FB0446019018B928466D
:10B7500065F048FFCEE7D6F8E83F93F8D5B0036828
:10B760008BF0010A5B69984705F50543019AA833F8
:10B770009A4208BF0120BBF1000F08D10198514641
:10B7800003685B689847044648BB6A4A22E096F91A
:10B79000B83F002B80F2BC80002800F0B980DFF8B1
:10B7A0008CB1DBF8C40F03685B6998470446002836
:10B7B00040F0AE800198FFF711FFB0EE408AABF584
:10B7C000A040F7F71BFAB4EEC08AF1EE10FA40F38E
:10B7D0009F80594A01992846FFF7B8FB8AE705F58B
:10B7E000BF4101AA284605F5405A4431FFF716FC2F
:10B7F0000198C6F8C40F8AF8EC8B03681B68984759
:10B80000014605F5C2504246083067F041FC05F597
:10B81000BA400021503073F093FBFB1E012B02D97C
:10B82000B91F4C424C4189F89E4E9AF9323A23B1E5
:10B8300005F568502C308BF087F8D6F8C40F0368F4
:10B840001B689847C21ED9F8143B5042504106F677
:10B850007C22012F89F8A40B1268C3F8F82006F6A1
:10B86000AC22D9F8143B1268C3F8FC2001D00B2F8E
:10B8700006D106F69426D9F8143B3268C3F8FC20AA
:10B880002846FFF7F3FB294B93F8B93F9B063FF59A
:10B8900039AF2EE705F5405393F82C2A002A3FF4E0
:10B8A0006DAFB3F8482AD0077FF568AF93F8682AE0
:10B8B000002A3FF463AFD6F8E82F92F8D520002A8B
:10B8C0003FF45CAF93F8EC3B0A2B7FF457AF96F94B
:10B8D000B83F002BFFF652AF184A284601990024C2
:10B8E000FFF734FB06E716480CF0A2FD0028D1D183
:10B8F000D6F8C40F03685B6998470028CAD001983E
:10B9000003685B69984704460028C3D10D4A61E784
:10B91000019803681B6998470028E4D008480CF098
:10B9200075FD04460028DED1074A53E7C88200307F
:10B930004CC1003096F91608ACCC1408D0CC1408D1
:10B94000C8320030BECC1408827516080148FFF7D3
:10B95000A5BE00BFC832003013B504468DED010A04
:10B960008EF0AAFB01A96369A26B1B6892ED001A15
:10B9700093ED0E0AD3EDC90A8DF0AAF99DED010AE7
:10B9800002B010BD436A186803685B6A184700007C
:10B9900038B5436A05461C6894F8D51061B920464D
:10B9A000B7F0FCFF6B6A1B6893F8A10018B101287F
:10B9B00014BF0320022038BD164803783BBBFFF7B5
:10B9C00043FC20BB144A92F8B83F03F0A003202B9D
:10B9D00017D0B5EEC00AF1EE10FA10D592F8BA3FC2
:10B9E0005B070CD401212046B7F0D8FF6B6A1B68B7
:10B9F00093F8A130012B0CBF02200320DBE70221CA
:10BA0000F1E720460221B7F0C9FF0420D3E7012067
:10BA1000D1E700BF88C00030C8820030134B10B59A
:10BA20002DED028B93F8DD3F0446DB0704D59FED37
:10BA3000100ABDEC028B10BD74F0FAF9037F002BE5
:10BA4000F5D0636B186874F0B3FBA368DFED097A77
:10BA500003F5E35292ED008AD2ED010A28EE278A1F
:10BA60002FF06AFC28EE000AE3E700BFC88200302E
:10BA7000000000000000C8420148F7F731B900BFDC
:10BA8000C83200300148F8F791B800BFC832003022
:10BA90000148FFF703BE00BFC8320030F0B55F4E6B
:10BAA00004460D4696F8DD3F2DED028B13F0010F95
:10BAB0008FB005AF5FD143689B899A071CD5584862
:10BAC00069F02AFDDFED577A90ED007AB4EEE77A5F
:10BAD000F1EE10FA10DD67F0D9FF3D2167F012FF9B
:10BAE00009220521A6F5A040FFF7D8FD20B90922BB
:10BAF00002212046FFF7CCFF636893F95430002BF6
:10BB000039D000230593089323691868B6F04CF9DF
:10BB1000236AB0EE408A186803689B6E984708AAAB
:10BB2000F0EE400A3946B0EE480A2046FFF7BEFA6A
:10BB3000DDED057A9FED3C7AF0EEE77AF4EEC77A18
:10BB4000F1EE10FA08D5DDED087AF0EEE77AF4EEC2
:10BB5000C77AF1EE10FA0ED496F8BA3F1B0704D458
:10BB600067F094FF492167F0CDFE96F8BA3F43F0A5
:10BB7000080386F8BA3F95ED027A08A895ED005AB9
:10BB8000B1EE477A95ED016AB7EEC55AB7EEC66ACF
:10BB9000B7EEC77A9FED1F0B8DED085B8DED0A6B3D
:10BBA0008DED0C7B34F00AFF636908A98DED0A1B4B
:10BBB0008DED0C2B8DED080BDFED1C0A9FED1C0AA3
:10BBC0001868B2F093F863691868B2F0C9FA63694B
:10BBD0001868B2F079FD236A1D6863691868B1F0CE
:10BBE00009FB384613498DED020ACDED030A8DEDB0
:10BBF000041AFCF795F8079B02A92846009397E8DA
:10BC00000C00AEF01FFA0FB0BDEC028BF0BD00BF10
:10BC1000AFF300800000000000005940C8820030EF
:10BC2000A4AD003000002F440000003400007A442E
:10BC30000000000044BF00302DE9F041AA4D00266D
:10BC4000044695F8B93F2DED028B5A0692B0059641
:10BC5000069603D543691868B0F004FE95F8DD3FF9
:10BC6000DB0755D463689B899F071BD59F4869F004
:10BC700053FCDFED9F7A90ED007AB4EEE77AF1EEB7
:10BC800010FA0FDD67F002FF3D2167F03BFE09224D
:10BC900005219848FFF702FD20B90922022120461C
:10BCA000FFF7F6FE636893F954308BB39148F7F7CA
:10BCB0007DFFE3689FED908AB6EE000A1B68204680
:10BCC0009FED8E7AD3ED0A7AF4EEC87AF1EE10FA8F
:10BCD00067FE877A27EE800AFFF73CFACDED060A69
:10BCE0008DED050AB0EEC00AB4EEC80AF1EE10FA06
:10BCF00040F1AC80F0EEE00AF4EEC80AF1EE10FA82
:10BD000040F1A4807E4BB3F8203D980700F1AE804F
:10BD100095F8BB3F6FF3820385F8BB3F95F8BA3FB8
:10BD20001A0700F1A8807748B3F024FA95F8BB3FD2
:10BD30000EAF60F3820313F0040F85F8BB3F40F0B1
:10BD40009C80606901230E963A460F9605A900680B
:10BD5000B0F0FCFD63691868B2F002FA6369186814
:10BD6000B1F048FAA3688DED0B0ACDED0C0A8DED0C
:10BD70000D1AD3ED007AF5EEC07AF1EE10FA52DD2D
:10BD8000614B20469FED618AB3F9D83D00EE903AB1
:10BD9000F8EEE00ACDED030AFFF7E0FAA368B7EE8C
:10BDA000002A07EE900ADDED030AD3ED001AB8EE83
:10BDB000E71A9FED4F0A31EE822A61EE881A22EED1
:10BDC000082A2EF05FF9DFED527A20EE270ADFED28
:10BDD000517A20EE270A12F123FBDFED4F7A0BA8F0
:10BDE00020EE270A20EE088A33F082FAB4EEC08AE9
:10BDF000F1EE10FA17D5C8EE006A9DED0B7ADDED75
:10BE00000C7A636927EE267A67EEA67A8DED0B7AB7
:10BE1000CDED0C7A1B68D3F8AC23C3F8B823D3F864
:10BE2000B023C3F8BC23236A38463C491C68FBF79F
:10BE300077FF109B0BA92046009397E80C00AEF00B
:10BE400001F912B0BDEC028BBDE8F08195F8BA3F64
:10BE5000190704D467F01AFE492167F053FD95F8DD
:10BE6000BA3F43F0080385F8BA3F51E795F8BA3F67
:10BE70006FF3C303F7E7002058E70DF11C082148D2
:10BE800007964146089609960A96B3F0FBF928B939
:10BE9000A069B6F025FA03C888E80300A069B6F0E7
:10BEA00027FA09AA01461748B3F052FA9DED087A1D
:10BEB0009DED076A0123B7EEC77A6069B7EEC66ADF
:10BEC00000930B960BAB0C9609AA39468DED0E6BC1
:10BED0008DED107B0068B0F071FD95F8BB3F5B07FE
:10BEE0007FF52FAF36E700BFC8820030A4AD003029
:10BEF00000002F44C83200300000003400007A43B4
:10BF0000C8A20030ACAF0030C86200300000C842A8
:10BF10000AD7233C35FA8E3C0AE81C4144BF003066
:10BF200013B504460191FFF787FE0199204602B040
:10BF3000BDE81040FFF734BA1FB5194B044693F81B
:10BF4000BA3F1B0729D4002301A916480193029385
:10BF50000393B2F0A5FF032807D8DFE800F0150E21
:10BF6000020801A92046FFF799FD04B010BD0D4855
:10BF7000B2F0B8FF30B10128F7D100212046FFF719
:10BF8000CFFFF2E70121F9E765F050FF40F286327A
:10BF90004FF4801165F002FFEFE70021EFE700BFEB
:10BFA000C8820030A0B0003008B5034619B9064A6F
:10BFB00092F9E42C1AB91846FFF7B2FF08BDBDE8A4
:10BFC0000840FFF7B9BF00BFC8A200300148FEF724
:10BFD000A9BC00BFC832003000487047189000303C
:10BFE0000148F6F769BE00BFC832003030B5174DC2
:10BFF0008BB000230022044604A9D5F81C0BCDE920
:10C000000423CDE90623CDE90823B1F00BF908A9F3
:10C01000D5F81C0BB1F066F9022201A920469DED6E
:10C02000067B9DED045BF7EEC76BB7EEC55B9DED40
:10C03000087B8DED015ACDED026AB7EEC77B8DED21
:10C04000037A17F0DFFC20460BB030BDC8A20030E9
:10C05000014B01221A70704794BF003000207047D6
:10C060000020704700207047002070470020704774
:10C070000020704700207047002070470020704764
:10C08000002070479FED010A704700BF00000000CC
:10C090000020704700207047002070470120704743
:10C0A0000020704700207047002070470120704733
:10C0B0000020704701207047012070470020704722
:10C0C00001207047012070470020704700487047EA
:10C0D000FCCC140800487047FCCC1408836803F5B6
:10C0E000805393F8743CDB0706D50023022280F8C6
:10C0F0003C30024BC3F8BC2F01207047C88200308F
:10C1000090F83C3053B9836803F5805393F8743C3E
:10C11000DB0742BF034B0122C3F8BC2F002380F88A
:10C120003C307047C8820030012380F83C307047B3
:10C130002DE9F0432DED0C8BF0EE409A97B020EEF8
:10C14000000A0025F0EE60AA0446B0EE41CA894616
:10C15000A0EEA00A9046F7EE00CA1F460195029590
:10C1600003950495B7EEC00A0595069512F1C2FA3B
:10C17000B7EEC00BA3689FEDCFDA03F58053B4EEA2
:10C18000EC0A03F5436203F63443F1EE10FAD3ED03
:10C19000000A92ED009AC8BFCCEE807A29EE0D9A83
:10C1A000C4BF69EEA79A6AEEA7AAB0EE690A2FF09B
:10C1B000C3F8A36829EE009A03F58053B0EE6A0A2B
:10C1C00003F5436203F63443D3ED000AD2ED008A4F
:10C1D0002FF0B2F8A36868EE8D8A03F5805303F65A
:10C1E000484203F64C4368EE808A92ED008AB0EE36
:10C1F0004C0AD3ED000A2FF09FF8636828EE0D8AF1
:10C2000093F9703028EE008A002B00F0D980236A61
:10C210009FEDA90A18686C3033F070FCB0EE60AA8C
:10C22000CDED080A8DED091A8DED070A2DF0A8FF56
:10C23000BDEEC0BA40F6B832A0491BEE100A2EF08F
:10C240005FF84342B0EE4A0A07EE903A6368F8EEB0
:10C25000E77A93ED1A7A67EE877ACDED017A2DF0C1
:10C260008FFFFDEEC0BA40F6B83294491BEE900A3B
:10C270002EF046F84242636807EE902A039593ED4C
:10C280001B7AF8EEE77A93F97030022B67EE877A23
:10C29000CDED027A6ED18A4BB8EECBBAB3F9D83D68
:10C2A0000AEE103A236AB8EECAAA1A68B4EECABAFD
:10C2B000F1EE10FA3DDDA3683AEE4B0ADFED810A9C
:10C2C00003F5E153A16B92ED051A93ED047AD1EDDC
:10C2D000001A27EE0D7AC7EE200A2EF05DFCDDED88
:10C2E000017A37EE800A8DED010AB8EEEB0A236A77
:10C2F0001A68B4EECA0AF1EE10FA34DDA3683AEE19
:10C30000400AA16B03F5E15392ED061AD1ED001A34
:10C31000D3ED040A20EE8DDADFED6A0ACDEE200AB5
:10C320002EF03AFCDDED027A37EE800A8DED020A3E
:10C3300020E0B1EE4A0AB4EEC0BAF1EE10FAD4D55C
:10C34000A36830EE4B0AA16B03F5E153DFED5D0A04
:10C35000D1ED001A93ED047A92ED051A27EE0D7ACD
:10C36000C7EE200AB9E7B1EE4AAAB4EECA0AF1EE66
:10C3700010FAC3D4236A12AD0EAED3F800C00CF18C
:10C3800084030FCB85E80F000AAD86E80F0085E82F
:10C390000F0004AB01AA29466046AEF00DFB6368AE
:10C3A00093F97030022B16D1DDED047A39EE279A1D
:10C3B000DDED057A78EEA78ADDED067A38EE278A7C
:10C3C00089ED009AC8ED008A87ED008A17B0BDECB0
:10C3D0000C8BBDE8F083F0EEE99ADFED3B0AF0EE5E
:10C3E000EAAAAD20B0EECCCACDED009AB7EE001AA5
:10C3F000F4EEE9AACDED0AAA8DED0ECAF1EE10FA1F
:10C4000048BF6D46D5ED007AF4EECC7ADFED2F7A99
:10C41000F1EE10FAD8BF354695ED007A87EE270A7F
:10C420003CEEC00A2DF014FFE36904A8D3ED937A23
:10C4300020EE270A33F062FB8DED061AB0EEC91A22
:10C44000B520F0EEC07A8DED040ACDED050A39EE87
:10C45000000A31EE671AB0EEC11AF1EE410A2DF072
:10C46000F7FEB0EE409A9DED050AB0EEE81ABA204C
:10C47000F0EEC07A38EE800A31EE671AB0EEC11ADB
:10C48000F1EE410A2DF0E4FEF0EE408A9DED060A41
:10C49000B0EEC81ABF20F0EEC07A38EE000A31EED6
:10C4A000671AB0EEC11AF1EE410A2DF0D1FEB0EEDE
:10C4B000408A85E70000C8429F0CB34548F4FFFF5F
:10C4C000C862003000007A440000000000A08C45E3
:10C4D00010B52DED028B836A044686B0186873F0A0
:10C4E00067FEE36AB0EE408A186873F061FE636B22
:10C4F0008DED010A186873F05BFE05ABB0EE401AD3
:10C5000003A92046B0EE480A04AADDED010AFFF7B0
:10C510000FFE636A186890F8D51000293CD1B7F077
:10C520003DFA2046FFF75AF8636AB0EE408A1B686E
:10C5300093F8A11001293FD0032946D051B9236AAD
:10C5400001211868AFF066F9236A1868ADF0B4FCF1
:10C550009FED218A236A9DED030A1868A36802688B
:10C5600003F58053DDED040A9DED051A93F8743C44
:10C570009B074CBFD36B936B9847236A174AB0EE67
:10C58000480A18680021D2ED000A03685B6E9847DC
:10C5900006B0BDEC028B10BD114B93F9B92F002AE8
:10C5A00006DBD3F8BC3F022B04D190F8A1300BB9C5
:10C5B0000121B4E70221B2E7236A1868AFF02AF933
:10C5C000236A1868ADF08EFCC2E7D9790029C1D181
:10C5D0002046FFF7FBFCBDE700000000AC70003018
:10C5E000C8820030836803F6A82393ED000AB5EEF5
:10C5F000C00AF1EE10FA01DCFEF7EABF7047000056
:10C6000070470000002070470120704702207047EB
:10C6100000207047002070470120704700207047BD
:10C6200081F0010070470000012070470120704731
:10C630000048704798CD140800487047A4CD1408EE
:10C6400038B5436904461868B0F0D6FB18B9636979
:10C650001868B1F0D5FE636920461D68FFF7C0FC7D
:10C660006368B3F93820B3F9363001EE102A00EED2
:10C67000903A4342B8EEC11A284600EE103AF8EE5E
:10C68000E00AB8EEC00AB0F09BFA636920461D6864
:10C69000FFF7A6FC6368B3F93820B3F9363001EE32
:10C6A000102A00EE903A4342B8EEC11A284600EE36
:10C6B000103AF8EEE00AB8EEC00AB0F0F7FA01203E
:10C6C00038BD000030B504462DED028B436985B0BE
:10C6D0001D68FFF785FC6368B3F93820B3F936307D
:10C6E00001EE102A00EE903A4342B8EEC11A2846F5
:10C6F00000EE103AF8EEE00A5C4DB8EEC00AB0F079
:10C700005FFA2046FFF7BEF9B5F9D83D08EE103ABA
:10C71000236A1868B8EEC88A03689B6E984702AA15
:10C72000F0EE400A01A9B0EE480A2046FEF7BEFC32
:10C730002046FFF773F9236BF0EE408A20461B6812
:10C74000B3F9083000EE103AB8EEC00AFFF794F9DA
:10C750002046B0EE408A8DED030AFFF741FC636886
:10C76000B3F93630B0EE480A01EE103A43422B20BE
:10C7700000EE903AB8EEC11AF8EEE00A2DF068FD2E
:10C7800020468DED030AFFF703F9042813D8DFE8EC
:10C7900000F0032F252A4B00236A1868ADF08CFBAC
:10C7A000236A00211868AEF053F963699FED300ADF
:10C7B0001868B1F00DFF236AB0EE681ADDED020AC9
:10C7C00018689DED010A0368DB6A98476369186879
:10C7D000B1F07AFF05B0BDEC028B30BD236A0121B8
:10C7E0001868AEF035F9236A1868ADF07BFBDCE71A
:10C7F000204D2B7863B9636845209FED1F1ADFED4C
:10C800001C0A93ED040A2DF023FD28460CF0F8F9DC
:10C8100020469DED030AFFF79FF803A915488DED0B
:10C82000030A0CF029FAC6E7636A02211868B7F018
:10C83000B5F8B5F9D83D02AA01A900EE103A0F48A3
:10C84000B8EEC00A8DF0B2FB20469DED030AFFF75B
:10C8500083F80B488DED030A0BF052FC63699DEDE4
:10C86000030A1868B0F02EFAA5E700BFC8620030CE
:10C870000000000088C0003000007A4400AF0030A3
:10C88000B88E00300020704790F80D33002B14BF95
:10C890001B200320704700000020704701207047D4
:10C8A00090F8E402062804D0A0F10A035842584147
:10C8B0007047012070470000012070470120704739
:10C8C00090F80D03034A044B002814BF1046184685
:10C8D000704700BF40CE1408E98B160890F80D038E
:10C8E000034A044B002814BF10461846704700BF87
:10C8F0004CCE1408E98B160890F8E4020B3818BFE8
:10C900000120704790F80D332BB9044BD3F8C80AB7
:10C9100000F0010070470020704700BFC88200305F
:10C92000024BD3F8C80AC0F3C0107047C882003069
:10C9300090F8E43223B9034B187880F00100704777
:10C940000020704760C0003038B590F8E4420546DA
:10C95000012C01D0002038BDC368186803681B692A
:10C9600098470028F6D1EB6820461B6883F8B84842
:10C97000F1E70000C368002201201B6883F8B82893
:10C9800070470000002370B52DED028B80F80D3349
:10C9900084B0B0F8703004460D46012B01D8002950
:10C9A00049D0636A264E1B6893F8D5308BBB0723AA
:10C9B000244884F8E4320368022B02D10021FAF7FC
:10C9C00059FF9FED218A0125E368F0EE480A1868B7
:10C9D000B0EE481AF0EE481AB0EE480AB4F03AFC4D
:10C9E00004F5227084EDCE8A84EDCF8A84EDD08A5E
:10C9F00084F80C5334F0CAF8144805F0B7FA96F8E6
:10CA0000BA3F13486FF3C30386F8BA3FB2F052F946
:10CA100011E096F9B83F002BC9DA04F13C0036F07A
:10CA20009DFB05460028C2D12046FFF7D5FA094AEA
:10CA3000022169F009FC284604B0BDEC028B70BDF0
:10CA4000C882003044BF00300000000048B9003008
:10CA5000A0B0003054CE140810B50446094890F830
:10CA60006030012B02D15C3034F0FAF8064890F8BF
:10CA70002D1C00F6B43076F043FA002384F80D3311
:10CA800010BD00BFC8B20030C8A200300A4B10B5BC
:10CA900004462DED028BB0EE408AD3F8200BB3F0A4
:10CAA0003FFF9FED060A012028EE008A84EDCF8A21
:10CAB000BDEC028B10BD00BFC8A200300AD7233CDA
:10CAC0000A4B10B504462DED028BB0EE408AD3F828
:10CAD000200BB3F035FF9FED060A012028EE008AF7
:10CAE00084EDD08ABDEC028B10BD00BFC8A200301F
:10CAF0000AD7233C0A4B10B504462DED028BB0EE4D
:10CB0000408AD3F8200BB3F029FF9FED060A0120DD
:10CB100028EE008A84EDCE8ABDEC028B10BD00BFEA
:10CB2000C8A200300AD7233CC3681B681869B0F05C
:10CB3000B3BC000038B5D0F8E83204460D461BB946
:10CB4000C0F04AF9C4F8E802C0F046F9D4F8E83277
:10CB5000C01A4FF47A73B0FBF3F0B4F8E63298429F
:10CB600009D32046FFF738FA2B88044A062169F0DA
:10CB70006BFB012038BD0020FCE700BF70CE14081D
:10CB800090F8E432052B05D1054BD3F8283BD86843
:10CB9000B0F0F2BBC36818680368DB68184700BFD1
:10CBA000C8A2003008B590F8E432052B0BD1094B30
:10CBB000D3F8283BD868243032F09AFBBCEEC00A88
:10CBC00010EE100A08BDC368186803689B68984790
:10CBD000F4E700BFC8A2003090F8E4328B4206D0E0
:10CBE0000B2B80F8E41202D10148FCF757BD7047C7
:10CBF000C832003073B501231E4E05460A4680F840
:10CC00007530D6F8C43F834214D10124019285F8CF
:10CC10000D43D6F8C40F03681B689847019A014674
:10CC2000154866F035FA96F8B93F9A061BD42046A7
:10CC300002B070BD01910321FEF72AFF019A04465C
:10CC40000028E2D185F8750066F020FF1B220A213A
:10CC500066F078FE96F8B93F9B06E8D5074A137848
:10CC600043F0040303E0054A137843F00203137012
:10CC7000DDE700BFC8820030104B00304CC10030EF
:10CC800030B585B004460D4601466846FFF7AEF95B
:10CC9000694604F13C0036F0C5FEC8B966F0F6FE00
:10CCA0001B220A2166F04EFE0D4B93F8B93F9B06FE
:10CCB00004D50C4A137843F0040313702046FFF7A1
:10CCC0008BF9094A042169F0BFFA002005B030BD94
:10CCD0002946204605B0BDE83040FFF78BBF00BFB6
:10CCE000C88200304CC1003084CE140830B585B005
:10CCF00004460D4601466846FFF778F9694604F197
:10CD00003C0036F0B3FEC8B966F0C0FE1B220A2113
:10CD100066F018FE0D4B93F8B93F9B0604D50C4AFC
:10CD2000137843F0040313702046FFF755F9094ABE
:10CD3000042169F089FA002005B030BD294620465B
:10CD400005B0BDE83040FFF755BF00BFC8820030D6
:10CD50004CC10030C0CE14087FB505460E460146D2
:10CD6000684605F13C04FFF741F96946204636F074
:10CD70007DFEC0B92046694636F054FE044690B99F
:10CD800066F084FE1B220A2166F0DCFD0D4B93F851
:10CD9000B93F9B060FD42846FFF71EF90A4A042123
:10CDA00069F052FA04E031462846FFF723FF0446B3
:10CDB000204604B070BD054A137843F00403137095
:10CDC000E9E700BFC8820030F8CE14084CC100303B
:10CDD00010B590F8E4420A2C16D1B0F812430C803A
:10CDE00090F818131170D0F81C231A60029BD0F829
:10CDF00020231A60039BB0F924231A80049BB0F906
:10CE0000262301201A8010BD0020FCE790F8E432B0
:10CE10000A2B06D1B0F812338B4204BF012380F8ED
:10CE20001033704730B5044685B00F480BF0EEFA6A
:10CE30000546B0B1072301A984F8E4320023019329
:10CE400002930393E3681868B3F0F6FCE36801A962
:10CE50000022186803685B68984700210348FAF7C6
:10CE600009FD284605B030BDC832003044BF00304F
:10CE7000F0B5414F05460C46D7F8F42AD7F8F03AFA
:10CE80001343D7F8EC2A13432DED028B87B00CD156
:10CE900064F0CCFF40F275124FF4801107B0BDEC86
:10CEA000028BBDE8F04064F079BF8069B5F01AFAF2
:10CEB0002046B0EE408A16F0E5F9032839D1EB6838
:10CEC00001A91868B3F0BEFD064690B3DDED017A06
:10CED000636838EE678A0093284B0021DFED287ADB
:10CEE00093F9B83F9FED270A002B009B264827FEA9
:10CEF000800A38EE008ABDEEC88A18EE102A9342E6
:10CF0000ACBF00930092FAF7B5FC6B691868B1F0FA
:10CF100077FADDED007A31461C48B8EEE70A0CF0EE
:10CF200035F900212846FFF757FE07B0BDEC028B0C
:10CF3000F0BD94E80F0002AE86E80F00D7F8F03A93
:10CF40006A46022130460493D7F8F43A059316F066
:10CF5000A5F978B966F09AFD0222152166F0F2FC77
:10CF6000DDED037AF8EEE77A77EE887AFDEEE77A80
:10CF7000CDED007A0026AFE7C8A20030C8820030AD
:10CF8000000000000000C84244BF003060C0003014
:10CF900030B52DED028BC3688BB004460D46186882
:10CFA000B3F026FD00285CD1002301930293039384
:10CFB00094F8E432F3B90022002304A93848CDE9FB
:10CFC0000423CDE90623CDE908230CF011F988B13B
:10CFD0009DED067B9DED045BF7EEC76BB7EEC55B81
:10CFE0009DED087B8DED015ACDED026AB7EEC77B52
:10CFF0008DED037A94EDCE0A9FED2A8AE368B4EEB4
:10D00000C80ADDED010A9DED021ADDED031AF1EE0D
:10D0100010FA1868AABFDFED247A9FED240A20EEEB
:10D02000270AB4F017F9D4EDCF7AF4EEC87AF1EE0E
:10D0300010FA07DBE3689FED1C0A186827EE800AE8
:10D04000B3F06EFCD4EDD07AF4EEC87AF1EE10FABB
:10D0500007DBE3689FED140A186827EE800AB3F037
:10D060006FFCE36829461868B4F01EF8054688B1DD
:10D070000F4B1B68022B09D0032B03D10D4B93F9E7
:10D08000093E1BB100210A48FAF712FC0121204693
:10D09000FFF7A2FD28460BB0BDEC028B30BD00BFF0
:10D0A00060C00030000000340000C84200000000F2
:10D0B00044BF0030C862003010B52DED028BC3684C
:10D0C0000446DFED338A1B684269D3ED0A0A9FEDFF
:10D0D000318AF4EEE80A93ED060A1068F1EE10FAD0
:10D0E00060FE880AAFF040FBE36862691B68106865
:10D0F000D3ED0A0A93ED060AF4EEE80AF1EE10FA0F
:10D1000060FE880AAFF0A6FB63691868AFF04AFDBD
:10D1100018B963691868B0F0DBFEE36862691B68E0
:10D12000106893ED080A93ED0C1AD3ED070AB0EEE0
:10D13000C00AAFF045FDE36862691B68106893EDB3
:10D14000080A93ED0C1AD3ED070AB0EEC00AAFF04F
:10D15000ADFD63691868AFF04FFE18B963691868D0
:10D16000B1F04EF900210C48FAF784FB0B488FF020
:10D17000A5F80B4A20460221B2F8BA3F23F4816396
:10D18000A2F8BA3FBDEC028BBDE81040FFF724BD0A
:10D190000000003400007A4344BF00308CAF003000
:10D1A000C88200300C4B10B50446D3F8280B90ED24
:10D1B0000F0A00F1200190F86020B3F05FF80748F3
:10D1C0000368022B02D00821FAF754FB2046052100
:10D1D000BDE81040FFF700BDC8A2003044BF0030DA
:10D1E000F0B5504D04460E461746D5F8280B2DEDE8
:10D1F000028BB0EE408A93B0B2F06CFEDFED4A8A4B
:10D20000F0EEC87AF4EEE87AF1EE10FA07D49FED6A
:10D21000470AD5F8280B28EE000AB2F0BDFED5F873
:10D22000280B90ED0F0AB0EEC00A0FB1B1EE400A24
:10D23000B2F0A2FE002302AA03A9D5F8280B03939B
:10D2400004930593B2F0C4FEDFED397A9DED027AC6
:10D25000B4EEE77AF1EE10FA5FDD022203A90EA820
:10D2600016F0D0FB71683046019116F00BF8019969
:10D2700002460EA815F0DCFFE3680EA91868B3F0AB
:10D2800013FF10B92B48FCF703FEA069B5F028F88E
:10D2900090ED017A90ED006A06A9B7EEC77AD5F84D
:10D2A000280BB7EEC66A20308DED066B8DED087B3E
:10D2B00032F03AFB0AA88DED0A0B8DED0C1B32F013
:10D2C0007DFB1D4B1B68022B1CD0D5F8283BB7EE0D
:10D2D000C00B00211848D3ED0E7AF4EEE87AF1EE97
:10D2E00010FAB8BFD3ED047AF4EEC07AF1EE10FA7A
:10D2F00010D5DFED127AB4EEE70AF1EE10FA09DD8F
:10D30000FAF7D6FA04212046FFF766FC13B0BDEC0D
:10D31000028BF0BDFAF7AEFAF4E72046FFF742FFC2
:10D32000F4E700BFC8A20030000000340000C8428B
:10D3300000009643C832003044BF00300000FA437A
:10D34000294B70B52DED028BD3F8204B0646DFED4F
:10D35000278AD4ED0A0AD3F81C5BF4EEE80A9FEDA5
:10D36000248A94ED060A2846F1EE10FA60FE880A37
:10D37000AFF0FAF9D4ED0A0A284694ED060AF4EE65
:10D38000E80AF1EE10FA60FE880AAFF063FA284668
:10D39000AFF008FC10B92846B0F09AFD94ED080AE9
:10D3A000284694ED0C1AB0EEC00AD4ED070AAFF08F
:10D3B00007FC94ED080A284694ED0C1AB0EEC00A5A
:10D3C000D4ED070AAFF072FC2846AFF015FD10B996
:10D3D0002846B1F015F800210648FAF74BFA012368
:10D3E000BDEC028B337070BDC8A200300000003469
:10D3F00000007A4344BF0030074808B5D0F8C83A67
:10D400009B0704D50121A0F5A040F5F7B9FA034820
:10D41000BDE808400BF012BDC882003060C000308B
:10D4200030B589B00446FDF725FF30B10021204614
:10D4300009B0BDE83040FDF755BF636A02211868A6
:10D44000B6F0ACFAE368186803685B699847014670
:10D450001048FCF707FC63691868B1F035F9236AD6
:10D460001D68636905AC1868AFF0C4FE20460A4920
:10D470008DED020ACDED030A8DED041AFAF750FC8A
:10D48000079B02A92846009394E80C00ACF0DAFD53
:10D4900009B030BDC832003044BF003038B5044652
:10D4A000FDF7E8FE054628B120460021BDE83840DA
:10D4B000FDF718BF636A02211868B6F06FFA2946B3
:10D4C0002046BDE83840FEF76FBD0000002101484E
:10D4D00007F0A0B9A8BA003030B5174D89B09FED5C
:10D4E000170A044605F5E043D3F8280BB2F034FFE1
:10D4F00001462846FCF7B6FB63691868B1F0E4F80A
:10D50000236A1D68636905AC1868AFF073FE204696
:10D510000B498DED020ACDED030A8DED041AFAF7E1
:10D52000FFFB079B02A92846009394E80C00ACF08F
